:020000040800F2
:10000000D83A001081020008B36300087158000854
:1000100049610008691300085587000800000000C6
:10002000000000000000000000000000A101000826
:100030002D1E000800000000FD010008857D00085D
:100040009B0200089B0200089B020008F96600085A
:100050009B0200089B0200089B0200089B0200080C
:100060009B0200089B0200089B0200089B020008FC
:10007000F1160008FD1600080917000815170008FA
:10008000211700082D1700089B020008891300089B
:100090006D1300089B0200089B0200082F1E000839
:1000A0009B0200089B0200089B0200089B020008BC
:1000B0009B02000800000000000000009B020008F6
:1000C0009B0200089B0200089B0200089B0200089C
:1000D0009B020008B1850008FD85000855860008D0
:1000E0009B0200089B0200080000000000000000C6
:1000F0000000000000000000000000000000000000
:10010000000000009B020008000000009B020008A5
:100110000000000000000000FD7E00089B020008B7
:100120009B0200089B0200089B0200089B0200083B
:100130009B0200080000000000000000000000001A
:100140009B0200089B0200089B02000800000000C0
:100150009B0200089B0200089B0200089B0200080B
:100160009B0200089B0200089B02000800000000A0
:100170009B0200089B020008000000000000000035
:100180009B0200089B0200089B020008DFF80CD0CD
:1001900000F0A4FD004800479DBF0008D83A0010B9
:1001A0002C4B1968086800F05AB880F30988BFF32F
:1001B0006F8F4FF0000080F311887047000000003F
:1001C00008480068006880F308884FF0000080F35A
:1001D000148862B661B6BFF34F8FBFF36F8F00DF35
:1001E00000BF00BF08ED00E0DFF80C00016841F43B
:1001F00070010160704700BF88ED00E0EFF30980F7
:10020000BFF36F8F134B1A681EF0100F08BF20ED5D
:10021000108A20E9F04F106009B44FF0500080F3CD
:100220001188BFF34F8FBFF36F8F0EF011F94FF0AE
:10023000000080F3118809BC1968086800F014B840
:100240001EF0100F08BF00F014B880F30988BFF348
:100250006F8F704700070010EFF30580704730C8BC
:10026000B0E8C04FFFF7A1BF30C8B0E8C04FFFF7FC
:10027000E7BFB0EC088AB0EC08CAFFF7E6BF0000A1
:100280000648804706480047FEE7FEE7FEE7FEE730
:10029000FEE7FEE7FEE7FEE7FEE7FEE7317E000849
:1002A0008D0100082DE9F05F0546002092469B462F
:1002B00088460646814640241BE02846414647467C
:1002C000224600F04FFA53465A46C01A914110D3C5
:1002D00011461846224600F036FA2D1A67EB01083F
:1002E0004F4622460120002100F02DFA17EB0009AD
:1002F0004E41201EA4F10104DFDC484631462A4667
:10030000434600F000B830BCBDE8C09F38B5D0E926
:100310000221491E01EB410102EBC1014268C1EB20
:10032000011102EB81010268C1EB011102EB8102B4
:10033000D0E9043101EB410103EB81013023A1F548
:10034000527191FBF3F4174D6C4302EBC41291FB15
:10035000F3F403FB141100921A2902DB124B1A4426
:1003600000920C2291FBF2F3104C6343009C04EBCF
:10037000C313009391FBF2F302FB13110C4A08E044
:10038000491E40F2A324535C6343009C04EBC31357
:1003900000930029F4DC0146684600F001FA009859
:1003A00038BD00003F0C0F008051010067C2030000
:1003B00020F3000810B5431A934209D28318881815
:1003C00003E010F8011D03F8011D521EF9D210BD03
:1003D00040EA01039B0703D009E008C9121F08C0C7
:1003E000042AFAD203E011F8013B00F8013B521E47
:1003F000F9D210BDD2B201E000F8012B491EFBD2A8
:1004000070470022F6E710B513460A46044619461F
:10041000FFF7F0FF204610BD30B505462A460B46D3
:1004200012F8010B13F8014B08B1A042F8D01CB12F
:10043000002802D06D1CF1E7284630BD10B50446F7
:1004400004E00B7800F8013B03B1491C521EF8D2BE
:10045000204610BDCAB2401E10F8011F8A4202D0C9
:100460000029F9D100207047421C10F8011B002917
:10047000FBD1801A704730B504460020034600E0E7
:100480005B1C934203D2E05CCD5C401BF8D030BDD6
:10049000034611F8012B00F8012B002AF9D1184668
:1004A000704730B505460020034600E05B1C9342D0
:1004B00005D2EC5CC85C201A01D1002CF6D130BD0D
:1004C00010B508E00A4602E0A34208D0521C137897
:1004D000002BF9D1401C0478002CF3D1002010BD72
:1004E0000FB400B58DB010A909900B9000914FF09A
:1004F000FF300A9000200C900548069005480790B0
:100500006A4609A80F9900F0A5F90DB05DF814FB33
:10051000710800088F0800082DE9FF5F1D464FF0A5
:10052000FF3BD5E9014691465F464FF00008A969B7
:100530007F1C01988847296A824688470028F6D19F
:10054000BAF1FF3F0CD024F4C064002E19DD600620
:1005500014D5BAF12B0F09D0BAF12D0F0ED103E04B
:10056000584604B000F07EB844F48064A9697F1C4A
:1005700001988847761E8246002E02DDBAF1300FC0
:1005800003D0B9F1000F26D032E0A969761E44F4F9
:1005900000747F1C019888478246002E05DDBAF161
:1005A000780F06D0BAF1580F03D0B9F1000F10D070
:1005B0001EE0B9F1000F02D0B9F1100F18D1A969EE
:1005C000761E24F400747F1C019888478246102010
:1005D00002E0082000E00A20814609E008FB090843
:1005E000A969761E44F400747F1C019888478246EE
:1005F000002E05DD4946504600F018F90028EDDAD6
:10060000E96901988847A00502D46FF00100A8E7C6
:10061000E00725D1600613D5600502D5C8F10000BA
:1006200000E0404629680A1D2A600968220501D5B4
:10063000087015E0220701D5088011E008600FE07E
:100640002868011D29600068210502D580F8008016
:1006500006E0210702D5A0F8008001E0C0F8008084
:1006600038467EE730BCBDE8C09F2DE9F047914693
:100670000F4680460446002614F8015B2DB100F0B9
:1006800081F80068405DC007F6D12B2D02D02D2DDA
:1006900018D0641E4A463946204600F009F927B1B1
:1006A0003968A14201D1C7F8008071054FF00204FA
:1006B0000BD54042002803DD08F016FC0460A007BB
:1006C000BDE8F08746F48066E4E70028F8DA08F031
:1006D0000BFC04606FF00040F2E770B5064608F0CE
:1006E00003FC046805460A2200213046FFF7BDFFDF
:1006F0002C6070BD00F0004230F000400AD0C10D07
:1007000001F56071C0F3160042EA0151C2084007CA
:100710001143704700200146704730B50B46014633
:1007200000202022012409E021FA02F59D4205D390
:1007300003FA02F5491B04FA02F52844151EA2F13A
:100740000102F1DC30BD202A04DB203A00FA02F17C
:10075000002070479140C2F1200320FA03F31943AF
:1007600090407047202A04DB203A21FA02F0002151
:10077000704721FA02F3D040C2F1200291400843B1
:100780001946704700487047B0F3000810B504469A
:10079000FFF7F8FF0068005D00F0010010BD0000E9
:1007A00010B500683C22B0FBF2F302FB1303B0FB70
:1007B000F2F00B60B0FBF2F302FB1303B0FBF2F0BC
:1007C00018224B60B0FBF2F302FB1303B0FBF2F014
:1007D000021D8B600723B2FBF3F403FB142280009D
:1007E00040F2B55300F66C308A61B0FBF3F2B0FB17
:1007F000F3F403FB1400443280084A61C8613B28CB
:1008000002D3920700D0401C0022074C13460A6115
:10081000E25C824203D8801A5B1C0B61F8E7401C43
:10082000C860084610BD0000B4F300083A2800D2A2
:10083000303820F02002412A01D3A2F1370088424B
:1008400001D34FF0FF307047026811441378016004
:1008500018467047D1600449516104491162002172
:100860001161114600F05EBA490800088D070008C2
:10087000426842B1016811F8013B23B1521EC0E940
:100880000012184670470121C160881E70474268F7
:100890005AB1C368016843B983688B4205D0491EC9
:1008A000521CC0E90012002070474FF0FF30704723
:1008B0002DE9F05F82460078002715468B460AF145
:1008C0000104B946302801D09DB113E014F8010BA2
:1008D0000127782803D0582801D045B10AE00DB18E
:1008E000102D07D10027102514F8010B02E0082570
:1008F00000E00A250026B0460EE005FB080005FBD7
:1009000006F1012701EB10461FFA80F8B6F5803F8B
:1009100000D3B94614F8010B2946FFF787FF0028DA
:10092000EBDABBF1000F05D00FB1641E00E05446B6
:10093000CBF80040B9F1000F06D008F0D5FA02213B
:100940000160C81E00F003B848EA0640FAE730BC70
:10095000BDE8C09F2DE9FE4F804681EA0300C00F2D
:100960000C46009021F0004123F00045B8EB020056
:10097000A94105D24046214690461C460B460246F8
:1009800023F00040104347D0270DC7F30A00C3F3FC
:100990000A510290401A019040286BDAC3F3130009
:1009A00040F4801B0098924620B10023D2EB030A4A
:1009B00063EB0B0B01985946C0F140025046FFF71C
:1009C000C2FE06460D4650465946019A00F098F977
:1009D00010EB08006141002487EA115284EAE773B2
:1009E0001A4340D0009A62B3019A012A4FEA075293
:1009F00015DC001B61EB02014FF0004202EA0752D6
:100A0000CDE90042001C41F5801132462B4600F032
:100A100031FB03B000F045B840462146F9E7001B22
:100A200061EB0201001C41F5801300185B412018A6
:100A3000A2F5001747EB030140EAD570B6196D41E6
:100A400011E06D084FEA360645EAC0754FEA0752D5
:100A5000001B61EB0201001C41F5801149084FEABF
:100A600030000019514132462B4603B000F01CB84B
:100A700000F0F1BA0098012240000023D0EB0202FE
:100A800063EBE073009821464FEAE074B8EB000096
:100A900061EB0401E9E783F000435BE781F000418B
:100AA00058E730BCBDE8C08F30BCBDE8C04FFFF791
:100AB000DFBF2DE9FE4F81EA030404F0004421F07A
:100AC000004100944FF0000B23F0004350EA010472
:100AD0005ED052EA03045BD0C3F30A54C1F30A5553
:100AE0002C44A4F2F3340194A0FB0254C1F313018B
:100AF00041F48011C3F3130343F4801301FB024458
:100B000000FB034E840A970A44EA815447EA83575C
:100B1000A4FB076802958D0A05FB07854FEA932C15
:100B200004FB0C542705029D4FEA065847EA163786
:100B3000B5EB08056EEB070C870E920E47EA81179E
:100B400042EA8312A7FB0201B6EB0B0164EB00043F
:100B50002B0D43EA0C335E1844EB1C50DA46514629
:100B6000E7FB0201C5F313044FEA0B3343EA1453C6
:100B70004FEA0432019C43EA0603A4F10C040294F8
:100B8000009CCDE900B400F075FA03B000F003B8A2
:100B900000200146F9E730BCBDE8C08F2DE9F04DDB
:100BA00081EA030404F0004B21F0004514464FF0A5
:100BB000000A23F0004150EA050220D054EA010265
:100BC0001DD0C5F30A570246C5F31303C1F3130042
:100BD000C1F30A5640F4801543F48013A7EB0608CE
:100BE000101BD64608F2FD3873EB050002D308F15E
:100BF000010801E092185B41B8F1000F03DA002010
:100C00000146BDE8F08D00204FF480110646844671
:100C10000EE0171B73EB050705D3121B63EB0503EF
:100C200006434CEA010C49084FEA300092185B4138
:100C300050EA0107EDD152EA030012D082EA040023
:100C400083EA0501084305D0101BAB4106D20122FF
:100C5000002306E000224FF0004302E06FF00102A3
:100C600053101AEB06004CEB085110EB0A0041EB55
:100C70000B01BDE8F04D00F0EEB9C1F30A52C1F32B
:100C8000130140F2FF3341F480119A4202DA00204E
:100C90000146704740F233439A42A2F2334202DCEB
:100CA0005242FFF75FBDFFF74EBD000030B5041E96
:100CB00071F1000404DB4FF00044404264EB010199
:100CC000141E73F1000405DB1C464FF00043524232
:100CD00063EB0403994208BF904230BD064C074DB8
:100CE00006E0E06840F0010394E8070098471034FC
:100CF000AC42F6D3FFF74EFA80F60008C0F60008C3
:100D0000202A06DBCB17203A41FA02F043EAE073CF
:100D100006E041FA02F3D040C2F1200291400843BC
:100D2000194670472DE9F34F8BB04FF0000801F1E1
:100D30000C000C464FF0010B46460DF1080A0190DD
:100D40006269012101989047051E2DD0252D2CD0D8
:100D5000216A8847C0B16269012101989047216AE0
:100D600088470028F7D1411E62690198904700E04A
:100D7000761CA1690B988847216A88470028F7D11B
:100D8000E1690B988847DBE7A1690B98884707461C
:100D9000A84201D1761CD3E7E1690B9888477F1CF4
:100DA00002D1B8F1000F6FD046E1002762693D46DD
:100DB0003946019890472A2804D162690121019897
:100DC00090470125DFF884926269012101989047DC
:100DD000A0F130010A290AD24F45E5DC07EB870173
:100DE00000EB4107303FDFD445F01005ECE7E906A2
:100DF00001D46FF000476C280AD04C2814D0682822
:100E000015D06A280DD074281CD07A281AD01DE07D
:100E100062690121019890476C2802D045F00405D1
:100E200014E045F002050DE045F020050AE0626996
:100E3000012101989047682802D045F0080505E097
:100E400045F400656269012101989047C4E90157A2
:100E500065283DD019DC58287AD00CDC452837D0DD
:100E600004DC252826D0412831D131E046282FD076
:100E700047282CD12CE05B2877D0612828D0632824
:100E80007CD0642823D15AE0D0E06F2848D008DC19
:100E900066281DD067281BD0692821D06E2816D15E
:100EA00027E0702845D0732868D0752847D0782867
:100EB0000DD14DE0A1690B988847054625283FF4E0
:100EC00069AFE1690B9888476D1C3FF46AAFB3E0E6
:100ED00023466A466FF001000B99AFF300809EE055
:100EE00045F040006060A80723464FF0000236D46A
:100EF0003EE0E8077FF447AF2068011D21600068ED
:100F0000290501D506701BE7290701D5068017E7DB
:100F1000A90703D5F117C0E9006111E706600FE7E3
:100F200045F040006060A80723464FF0080216D441
:100F30001EE040F60E0125EA0100606016E045F073
:100F400040006060A80723464FF00A0207D40FE074
:100F500045F040006060A80708D5234610226FF0D6
:100F600001000B99AFF3008059E007E023461022FF
:100F70006FF001000B99FFF7CFFA50E04FF0000936
:100F80004F464B46632802D05B2806D040E0E80677
:100F900001D40120A06001273AE062690121019893
:100FA00090475E2805D14FF00109626949460198D2
:100FB0009047216939B900210A46534643F8212058
:100FC000491C0829FADBB0B3216969B9C11700EBE4
:100FD000D16253110AEB830122F01F02821A012011
:100FE0000B68904003430B606269012101989047B0
:100FF0005D28E8D1B9F1000F09D00020514651F821
:101000002020D24341F82020401C0828F7DB02AB07
:10101000224600976FF001000B99AFF30080002883
:101020000CDA401C08D1BBF1000F05D04FF0FF30A7
:101030000DB000F00DB8FFE74046F9E7E90701D130
:1010400008F1010806444FF0000B79E6CCCCCC0C3B
:1010500030BCBDE8C08F10B5141E73F1000408DA6F
:10106000401C41F1000192185B411A4301D120F06C
:10107000010010BD2DE9F04D92469B4611B1B1FA29
:1010800081F202E0B0FA80F220329046FFF75BFB7B
:1010900004460F4640EA0A0041EA0B0153465A460D
:1010A000084313D0114653EA010019D0C8F1400299
:1010B0005046FFF757FB05460E46504659464246F6
:1010C000FFF741FB084305D0012004E020463946E4
:1010D000BDE8F08D0020054346EAE0762C43374317
:1010E0000A986305E40AA0EB08000022FD0A44EA1E
:1010F00047540A3002D500200146E9E701051019DE
:101100006941DDE9084500196941BDE8F04DA2E7F4
:1011100070B58C1810F8015B15F0070301D110F8B9
:10112000013B2A1106D110F8012B03E010F8016BE6
:1011300001F8016B5B1EF9D12B0705D40023521E69
:101140000DD401F8013BFAE710F8013BCB1A921CD1
:1011500003E013F8015B01F8015B521EF9D5A142CF
:10116000D8D3002070BD00002DE9F04104460027CF
:101170000D46006804F0D0FC0646206804F0C8FC68
:1011800030435DD02068C1682E4E890105D5617E4F
:10119000012902D1217E01290BD0022D1DD020680A
:1011A00004F0BAFCB8B120688168C1F3400169B1AC
:1011B00011E00125244902E08F4232D27F1C0268EF
:1011C000D2435206F8D440210160E8E781683140FB
:1011D00041F010018160012D11D0206804F098FCCD
:1011E00048B120688168C1F3400121B9816831406C
:1011F00041F020018160022D08D0032D04D0042588
:1012000002F0FAFA064617E00C25F9E70825F7E799
:1012100002F0F2FA801B05280ED920688068284267
:101220000AD0606D40F010006065A06D40F00100D4
:10123000A0650120BDE8F081206880682842E7D1E0
:101240000020F7E7C0FFFF7F000040A370B5044611
:10125000006881688268C1F3400112F0010F28D054
:1012600039BB816801F00D01012914D18168124A4E
:101270001140891C816021680320086002F0BCFADB
:10128000054612E002F0B8FA401B02280DD920688A
:101290008068C00709D0606D40F010006065A06DE7
:1012A00040F00100A065012070BD20688068C00783
:1012B000E8D1002070BD0000C0FFFF7FF8B50446F4
:1012C000002000902068816811F0010F41D18168F1
:1012D000214A11422ED18168D5432940491C8160A1
:1012E0001E48806800F0E07000020DD51C481D49C2
:1012F0000068B0FBF1F0401C00EB4000800000E013
:10130000401E00900028FBD102F076FA06461BE052
:10131000816811F0010F03D181682940491C816067
:1013200002F06AFA801B02280ED920680068C043C8
:10133000C00709D0606D40F010006065A06D40F0FE
:101340000100A0650120F8BD20680168C943C907F4
:10135000DED10020F8BD00003F00008000030450F3
:101360000C070020400D0300FEE7000010B5054803
:1013700001F07AFC03480068416941F002014161D3
:1013800010BD00006C310010014801F06DBC000080
:101390006C31001000B58BB000200121CDE90601B1
:1013A0000891059004900090019002900390694686
:1013B0000F4801F06BFB10B101200BB000BD0C48D1
:1013C00001F0A2FE48B10A4801F0D8FB014609A08D
:1013D00007F030FD0FA007F02DFD0221044801F0B9
:1013E000E4FA0028E9D010A007F024FD72B6FEE769
:1013F0006C31001043414E20496E697469616C691B
:101400007A6174696F6E204572726F723A20256C32
:10141000640A000043414E5F73746172745F464119
:10142000494C0D0A0000000043414E5F416374695E
:10143000766174655F4641494C0D0A0010B58AB06B
:101440000023009301934C788DF800408C788DF840
:1014500001408C798DF802405F248DF803408DF8AF
:101460000430C9788DF80510012103908DF806101D
:101470000420CDE904038DF80730069208AB6A46D4
:1014800002A9074801F0A3FA010007D005A007F060
:10149000D1FC0348416A10A007F0CCFC0AB010BD93
:1014A0006C31001048414C5F43414E5F41646454CD
:1014B000784D657373616765206661696C6564204A
:1014C0002C207265745F7374617475733A3078257B
:1014D00078200D0A000000006863616E2D3E4572A1
:1014E000726F72436F64653A2030782578200D0A58
:1014F0000000000000EE900A9FED1B2ADFED1B1A92
:10150000F8EE600A9FED1A0AB3EE031AC0EE822AC3
:1015100062EEA10AC0EE801AB7EE000A31EE800A30
:10152000FCEEC00A10EE900A087010EE100A114985
:10153000884201DC0020704710EE100A0E498842F4
:1015400001DB6420704770EE410A9FED0C1A80EEBB
:10155000810ADFED0B0A20EE200ABCEEC00A10EE75
:10156000100AC0B27047000000F07F45333353408B
:101570008C2EBA3D000098419A99C1416866A640F8
:101580000000C842034610B50020024603E09C5C00
:101590006040521C92B28A42F9D310BD70B58021CE
:1015A0001B4802F016F9054602F026F9194C0122F3
:1015B00094F823102DB10025012914D0022923D03D
:1015C00070BD11B9206684F82320216E401A41F2C3
:1015D00088318842F4D9022084F82300BDE87040A5
:1015E0000DA007F027BC216E401A41F22431643867
:1015F000884209D8607D012802D062750EA001E002
:10160000657512A007F016FC84F8235070BD000029
:1016100000040048140600104457494E5F42757498
:10162000746F6E2070726573732074696D656F7569
:1016300074EFBC815C6E00004477696E5F706F77F9
:1016400065725F6F70656E65640A00004477696E4D
:101650005F706F7765725F636C6F7365640A00001B
:1016600010B540F2AD110448FEF7CBFEBDE81040C6
:101670009F210248FEF7C5BE9C07001049090010D3
:10168000104C86B064200AF0ECFC06F0FBFF607B97
:101690000028F7D00B480DF1080CA4308179457A69
:1016A000037AC2798CE82E0042790179CDE90012E3
:1016B000C37882784178007805F054FA002060738E
:1016C000E0E700001406001070B5002330240CE0A1
:1016D000C55C01EB430604EB151501F81350C55C1E
:1016E00005F00F05303575705B1C9342F0D370BD6B
:1016F000014801F08ABD0000683D0020014801F06A
:1017000084BD0000203D0020014801F07EBD0000A6
:10171000483C0020014801F078BD0000003C00205A
:10172000014801F072BD0000903C0020014801F02A
:101730006CBD0000D83C002030B590F8444004F067
:101740001C050124AC40056C6C6004686360836810
:10175000102B036803D099600068C26030BD9A60A6
:101760000068C16030BD00002DE9F0412A4C207EA8
:1017700041F20205AE1CEF1C012805D0207E022894
:101780000ED0207E38B33EE064200CF065FD0121D0
:10179000284605F01DFB64200CF05EFD012125E0CC
:1017A00064200CF059FD0221284605F011FB14209D
:1017B0000CF052FD40F20131A02000F02FF864201F
:1017C0000CF04AFD0121304605F002FB64200CF0CC
:1017D00043FD012111E064200CF03EFD002128466C
:1017E00005F0F6FA64200CF037FD0021304605F0D4
:1017F000EFFA64200CF030FD0021384605F0E8FADD
:1018000064200CF029FDA17E41F2130001B10121F9
:10181000BDE8F04105F0DCBA140600100A4630B409
:101820000B495A2382240B70A5234B70CC70040AF9
:101830000C714871100A8871CA71802200230A72E3
:1018400007204B72887030BC0A22024803F0BEBFEA
:10185000340A0020F83A002008B5DFF810844FF46D
:10186000967B4FF0070A002598F8030044460928A4
:101870007ED2DFE800F005FEFDFCFBFAF9F8F70088
:10188000FFF772FF5E4658460AF0EBFB94F8202003
:10189000F7A1F94807F0F2FAF7494FF4905005F034
:1018A00017FB30460AF0DDFB207968B15FF00101DB
:1018B00041F2160005F08CFA30460AF0D2FBA07E09
:1018C000A04618B1012102E00021F1E7002141F218
:1018D000130005F07DFA30460AF0C3FBE74E002402
:1018E000371997F8780098B104EB44018819827889
:1018F00000924378725C601CC1B24FF4405000EB20
:10190000041005F07DFA87F8785064200CF0A4FCF0
:10191000641CE4B21E2CE3D398F80600444640BB96
:101920004FF6FF77394643F2E01005F051FA642094
:101930000AF097FB394643F2F01005F049FA6420AB
:101940000AF08FFB39464FF4485005F041FA642005
:101950000AF087FB394643F2102005F039FA64207B
:101960000AF07FFB394643F2202005F031FA01E00E
:1019700050E122E064200AF074FB394643F2302043
:1019800005F026FA64200AF06CFB39464FF4495002
:1019900005F01EFA64200AF064FB394643F2502039
:1019A00005F016FA64200AF05CFB394643F2602029
:1019B00005F00EFA64200AF054FB64200AF051FB93
:1019C000A079A04600287DD0002443F2E019371901
:1019D00097F8960078B106EB4400B0F85A0042BA86
:1019E000601CC1B209EB041005F042FA87F896506A
:1019F0003C200CF031FC641CE4B2032CE7D3A04E75
:101A0000002443F2102900BF06EB840000F5BD70EE
:101A10000AF010FB671CF9B209EB041005F0A0F9FD
:101A2000301980F8AA513C200CF016FCFCB2032CB3
:101A3000EAD300244FF4495906EB840000F5B7704F
:101A40000AF0F8FA671CF9B209EB041005F0F4F893
:101A5000301980F8A7513C200CF0FEFBFCB2032C9F
:101A6000EAD307E071E14DE138E126E120E1D2E07F
:101A70006FE036E098F80E0020B34FF4FA74204679
:101A80000AF0EFFA11200CF0B3F820460AF0E9FA58
:101A900010200CF0ADF820460AF0E3FA12200CF00A
:101AA000A7F820460AF0DDFA02200CF0A1F8204643
:101AB0000AF0D7FA01200CF09BF820460AF0D1FA80
:101AC000032000E004E00CF093F820460AF0C9FA85
:101AD0000AF066F94FF47A700AF0C3FA88F81350E6
:101AE000F8E00DF07FF9616D411AB1F5FA6F29D375
:101AF000606594F820205EA15F4807F0BFF95E4959
:101B00004FF4905005F0E4F9C8200AF0AAFA5D49B4
:101B10004FF4C14005F0F2F8C8200AF0A2FAA07E06
:101B200008B1012100E0002141F2130005F050F955
:101B3000C8200AF096FA207948B1012141F2160036
:101B400005F046F90AF02CF900F02EF9C2E0002168
:101B5000F4E70DF047F9A16D41F28832411A914244
:101B600058D3A06564200AF07CFA404C4FF4C04082
:101B7000A434617805F098F864200AF072FAA1782C
:101B800046F2100005F090F864200AF06AFA217A13
:101B900046F2200005F088F864200AF062FAA17984
:101BA00046F2300005F080F864200AF05AFAE17835
:101BB00046F2500005F078F864200AF052FA2179D4
:101BC00046F2600005F070F864200AF04AFA617984
:101BD00046F2700005F068F864200AF042FAA17A33
:101BE00046F2400005F060F864200AF03AFA254910
:101BF0004FF4C14005F082F864200AF032FA22491D
:101C000046F2900005F07AF864200AF02AFA00BF44
:101C10000AF0C6F85EE00DF0E5F8E16D40F6B83286
:101C2000411A914256D3E06564200AF01AFA0F492E
:101C30001422B03146F2A00006F03CF80B4913A084
:101C4000B03107F0F7F864200AF00BFA07491422C4
:101C5000C4310C4646F2C00006F02CF821460FA015
:101C600007F0E8F864200AF0FCF933E014060010ED
:101C70002564252500000000B80E00104909001059
:101C80009C070010CE060020C80600204457494E8D
:101C90002E73736964203A2573200A004457494E15
:101CA0002E70617373776F7264203A2573200A0077
:101CB00064200AF0D6F9012103E064200AF0D1F98A
:101CC000002141F2160005F083F864200AF0C9F9FA
:101CD00084F803A001200AF0C4F9C5E564200AF0E5
:101CE000C0F90121842000F041F864200AF0B9F91C
:101CF0001C494FF4C14005F001F864200AF0B1F925
:101D0000E57085E764200AF0ACF90E21842000F02C
:101D10002DF864200AF0A5F994F82020AFF2B00164
:101D2000114807F0ABF810494FF4905005F0D0F887
:101D300064200AF096F90B494FF4C14004F0DEFF2D
:101D400064200AF08EF901200AE064200AF089F983
:101D50000621842000F00AF864200AF082F90220AB
:101D6000E07055E7CE060020B80E001030B40A46E9
:101D70000B495A23A5250B704D708225CD70050A9D
:101D80000D7148718B710124CC71130A0B720720FD
:101D90004A72887030BC0A22024803F017BD000066
:101DA000340A0020F83A002070B51F4C607D08B955
:101DB00003206063607D0025012820D1207E616BB7
:101DC00088421CD04FF496700CF046FAA573207E22
:101DD00041F2010602281AD014200CF03DFA00212D
:101DE000304604F0F5FF1E200CF036FA40F20141B7
:101DF000A020FFF713FD0120A073207E6063A0796F
:101E000018B1A07B08B10BF091FDE57470BD3220D4
:101E10000CF022FA0221304604F0DAFF32200CF0F6
:101E20001BFA40F20131E3E71406001070478020EE
:101E300001F0D8BB064910B51F208861081501F0D4
:101E4000D9FD0121BDE81040002001F041BE000095
:101E50000070004072B6FEE7144A117F1448012951
:101E600001D003290FD1036823F4007303600368D2
:101E700043F400630360036823F4006303600368B2
:101E800043F400730360022901D003290BD10168D8
:101E900041F480510160016821F4805101600168C2
:101EA00041F480610160002010777047EC0600204B
:101EB00000200240C107054803D0416941F00401F8
:101EC0004161416941F48031416170470020024025
:101ED00008494A69C0B222F47E7242EAC0004861F1
:101EE000486940F002004861486940F48030486128
:101EF0007047000000200240054910B54C6944F0CD
:101F000001044C610260BFF36F8F436010BD00009D
:101F100000200240094A10B55469402344F480244B
:101F20005461EFF3108272B610C910C05B1E13F03B
:101F3000FF03F9D182F3108810BD00000020024099
:101F400070B5054601F058FC0646134C08E0681CC5
:101F500006D001F051FC801BA84201D3032070BDC4
:101F60002069C003F3D420690C4908400CD00C4907
:101F70004A6802434A60810F01D0A169A1618100D2
:101F800000D02061012070BD2069C00701D0012070
:101F90002061002070BD000000200240FAC3020052
:101FA000EC06002070B586B00C00054628D0154818
:101FB000854225D80026049601F0FEFA1248816970
:101FC00041F0404181614CF2FA31016128460096AE
:101FD00000F01CF80190284600F026F8029005EB6E
:101FE0008400401E00F020F80299401A401C039023
:101FF00004A9684601F010FA002801D001F07CFA2B
:1020000006B070BD000004080020024004490968C1
:1020100004494FF001000968CA431204120C7047CA
:1020200000000140E075FF1F0E4910B509684FF42C
:102030008024CB431A04120C0AD00A045FEA9212DD
:1020400002F10062824205D9A0F10060C00A10BD11
:102050002246F5E71A04120C01D009048C09001B72
:10206000F2E70000E075FF1F064B10B5984207D855
:10207000002303E010C841F823405B1C9342F9D3CE
:1020800010BD000000000408064B10B5984207D8A8
:10209000002303E010F8014BCC545B1C9342F9D3AE
:1020A00010BD0000000004082DE9F04117460D4660
:1020B000044601F081FA0F48844216D2002609E056
:1020C000D5E900232146002001F020FA68B9083440
:1020D0000835761CB6EB570FF2D3F80705D06368C6
:1020E000214600202A6801F011FABDE8F04101F014
:1020F00003BA0000000004082DE9F04FE5B099464E
:1021000014460E0083460CD0A1074FEA940000D07D
:10211000401C00271FFA80FA8DF800703D46E84603
:102120000CE0012065B000F031B86846FEF79CF97C
:102130004044725D13A106F0A1FE6D1CA542F4D3CC
:1021400001215846FFF72EFF524631465846FFF709
:10215000ABFF224649465846FFF796FF8DF8C870F8
:10216000002532AE09E032A8FEF77EF9304419F8B6
:10217000052004A106F082FE6D1CA542F3D30020C9
:10218000D0E70000253032582000000030BCBDE808
:10219000C08F000000B589B014216846FEF731F900
:1021A0000020024607906946134802F0A9FA00226F
:1021B00007A9114802F082FA9DF81F0000F5FA60A5
:1021C000ADF814009DF81D008DF816009DF81E0056
:1021D0008DF817009DF800008DF819009DF801009A
:1021E0008DF81A009DF802008DF81B0005A809F073
:1021F00023FC09B000BD0000A43100102DE9F84F08
:1022000000270446009790F85000DFF8B0930D4681
:10221000B846012811D0012684F85060206803F0E8
:102220007BFC60B1606D40F0200060655FF00107ED
:1022300084F85080384600F0D7B90220FBE769687F
:102240000C20052912D8022907D0032907D0042918
:1022500007D0052907D0062107E0686006E01221B3
:1022600003E0182101E04FF480716960D5E9002195
:10227000236800EA91101844036B01F01F014FF02E
:102280001F0C0CFA01FCC2F3846223EA0C038A409F
:1022900013430363206803F03FFC8246206803F089
:1022A00037FC5AEA00001DD1AA682968206803F0AB
:1022B0003FFC20686969C268C2F3C10252009140C4
:1022C0002A69042A0FD000EB82002B68026EDFF827
:1022D000F0C203F0F84302EA0C020B431A4342F047
:1022E0000041016672E0002103F00CFC400320680D
:1022F0004FF0000172D003F005FC90FAA0F0B0FAA4
:1023000080F1286842036ED090FAA0F0B0FA80F015
:10231000814204D100221146206803F018FC0121FB
:10232000206803F0EFFB400320684FF001015DD00F
:1023300003F0E8FB90FAA0F0B0FA80F128684203BD
:1023400059D090FAA0F0B0FA80F0814204D1002276
:102350000121206803F0FBFB0221206803F0D2FB7F
:10236000400320684FF0020148D003F0CBFB90FA05
:10237000A0F0B0FA80F12868420344D090FAA0F0AF
:10238000B0FA80F0814204D100220221206803F0DB
:10239000DEFB0321206803F0B5FB400320684FF00B
:1023A000030133D003F0AEFB90FAA0F0B0FA80F155
:1023B000286842032FD090FAA0F0B0FA80F0814252
:1023C00004D100220321206803F0C1FB206881684A
:1023D00011F0010F22D0ABE000E004E003F092FB2B
:1023E000C0F384618DE7C0F3846091E703F08AFB5A
:1023F000C0F38461A2E7C0F38460A6E703F082FB28
:10240000C0F38461B7E7C0F38460BBE703F07AFBF5
:10241000C0F38461CCE7C0F38460D0E72A7B2968ED
:1024200050F8B03FC1F3120C23EA0C0302F0180C71
:10243000644A22FA0CF20A4013430360E9684945F2
:1024400076D1286841031BD090FAA0F1B1FA81F14E
:10245000491C01F01F0109294FEA403131D80029F8
:1024600011D090FAA0F1B1FA81F100BF01F10101A0
:1024700001F01F0106FA01F608D1C0F3846109E0FA
:10248000C0F38461E4E7C0F38461EFE790FAA0F160
:10249000B1FA81F101F1010101F01F0146EA816108
:1024A00002D1C0F3846003E090FAA0F0B0FA80F0AB
:1024B00000F1010000F01F0000EB400041EA005174
:1024C00032E000290ED090FAA0F1B1FA81F100BFFC
:1024D00001F1010101F01F0106FA01F605D1C0F377
:1024E000846106E0C0F38461F2E790FAA0F1B1FAEA
:1024F00081F101F1010101F01F0146EA816102D180
:10250000C0F3846003E090FAA0F0B0FA80F000F12C
:10251000010000F01F002C4A00EB400002EB0050CD
:1025200041EA000141F00071AA68206803F000FB55
:1025300026482A6802423FF47BAE25488168254D33
:10254000254B01F0E071AA421BD10D0219D422687B
:102550009A427FF46DAE826841F4000122F0E0728D
:102560000A4382601D481E490068B0FBF1F0401C20
:1025700000EB4000800000E0401E00900028FBD1EE
:1025800056E6184DAA4207D1CD0105D422689A42D9
:10259000F6D141F080710AE06FF00045EA42EFD1D8
:1025A0004A02EDD422689A42EAD141F4800182685D
:1025B00022F0E0720A4382603AE6000000007F40A9
:1025C00000F0FF03FFFF0700000020FE000008806E
:1025D00000030450000052C7000004500C07002004
:1025E000400D0300000084CB18BCBDE8E08F0068FC
:1025F000006C7047F8B54FF0000504002E460095BA
:1026000002D0606D10B107E00120F8BD204600F057
:10261000C9F8A66584F8506020688168C1F34071EC
:1026200019B18168574A1140816020688168C1F3FF
:10263000007189B98168544A114041F0805181602C
:10264000524853490068B0FBF1F04000801C00E0A4
:10265000401E00900028FBD120688168C1F3007102
:1026600041B9616D41F010016165A16D41F0010159
:10267000A165012503F050FA616D01F010010143DD
:10268000606D05D040F01000606501252846F8BD5A
:1026900020F4807040F0020060652068806810F0CF
:1026A000010F0BD13B48806810F0010F06D13A486A
:1026B0006168826822F47C120A438260E168606B80
:1026C000627E0843A16841EA4231084394F8201031
:1026D00040EA0140012904D1A18C304A02EB41417A
:1026E0000843A16A29B101F47071E26A014342EA28
:1026F00001002268D1682A4B19400143D16020684B
:1027000003F00AFA0646206803F002FA304315D1B6
:10271000207E94F83010800340EA41022068C168AE
:1027200044F2020399431143C16094F83800012830
:102730000CD02068016921F00101016120690128A4
:102740002068016B21F00F0111D013E0D4E90F01D3
:102750000843D4E911121143084321680A6940F281
:10276000FC739A43104340F001000861E6E7E26918
:10277000521E11430163606D20F0020040F0010021
:10278000606583E7C0FFFF5FC0FFFF7F0C0700208D
:10279000400D030000000450000304500000FEFF41
:1027A00007C0F0FF10B59EB00446142117A8FDF72E
:1027B00028FE5C216846FDF724FE1C4920688842FB
:1027C00031D14FF480400090800314900224012006
:1027D000CDE90140082003900720CDE904048801D9
:1027E000CDE90640684601F097F908B1FFF732FBE2
:1027F0000F48C16C41F40051C164C16C01F4005137
:102800001C91C16C41F00101C164C06C17A900F0BA
:1028100001001C900B20CDE91740002019904FF0CB
:10282000904000F0EBFE1EB010BD00000000045010
:10283000001002402DE9F041044640690E46082888
:102840000AD02068C068C00708D0606D40F0200042
:1028500060650120BDE8F081082500E0042500F056
:10286000CBFF074614E0701C12D000F0C5FFC01B60
:10287000B04200D866B920680068284208D1606D6F
:1028800040F004006065002084F850000320E1E778
:10289000206800682842E6D0606D40F400706065F2
:1028A000206803F03DF980B1607E70B9206800684F
:1028B00000070AD5606D20F480706065606DC0040B
:1028C00003D4606D40F0010060652068C168082D88
:1028D00005D0490401D40C2101600020BAE7082189
:1028E000FAE7000010B50446006803F015F910B1CE
:1028F0000221084610BD94F8500001280CD0012098
:1029000084F850002046FEF7D9FC01004FF000008B
:1029100004D084F85000ECE7022010BD626D40F650
:1029200001639A4342F480726265626DD20404D5F9
:10293000A26D22F00602A26500E0A06523681C22B9
:102940001A6084F850002068C268920105D5626D53
:1029500022F4005242F4805262658268024B1A40AF
:10296000121D8260C5E70000C0FFFF7F10B504465E
:1029700090F85000012808D0012084F8500003216D
:102980002046FEF7F1FB10B10BE0022010BD2046FF
:10299000FEF75CFC28B9616D21F4885141F001011A
:1029A0006165002184F8501010BD90F82020012AA4
:1029B00007D0022A05D0416A41F4802141620120FA
:1029C0007047006842690A43426100207047F0B5D1
:1029D00090F820500468A468012D05D0022D03D082
:1029E000416A41F480214DE014F0406F01D1E500CF
:1029F00045D5C4F301640125A5401D608D684FF4E1
:102A0000C0739DB1CE6835434E6845EAC605066879
:102A100003EB0417F5514FF4C275076805EB041575
:102A20000E697E51097D012905D009E00E88CD6827
:102A300045EA4655EBE701684E5946F480764E511B
:102A40001179D2F805504FF4C67641EA05210568A0
:102A500006EB0416A9511178D2F801204FF4C47581
:102A600041EA0221026805EB04155151006803EBAD
:102A70000411425842F0010242500020F0BD416A68
:102A800041F4001141620120F0BD000010B590F842
:102A900020300268012B07D0022B05D0416A41F497
:102AA00080214162012010BDD2F8000240F00100F7
:102AB000C2F80002087D00F01F0301209840D2F800
:102AC0001C328343C2F81C32CB69B3B9D2F80C3242
:102AD0008343C2F80C328C894B6864F31F434C6902
:102AE00002EBC404C4F840320C890B6864F31F4342
:102AF0004C6902EBC404C4F84432CB69012B16D1F3
:102B0000D2F80C320343C2F80C320C884B6864F3E1
:102B10001F434C6902EBC404C4F840320C89CB68F3
:102B200064F31F434C6902EBC404C4F844328B695C
:102B3000002BD2F804320FD053EA0003C2F804325B
:102B40000B69002BD2F8143208D00343C2F81432B8
:102B5000096A012904D008E08343EFE78343F5E7DE
:102B6000D2F81C120143C2F81C12D2F8000220F065
:102B70000100C2F80002002010BD7047406A704793
:102B800030B590F82040012C05D0022C03D0416ACA
:102B900041F480215DE00468002955D02469A40730
:102BA00054D04FF4D874056804EB01142D5915F076
:102BB0000405956005682D594ED0ED0855600568EF
:102BC0002C5904F00204D4604FF4DA74056804EB65
:102BD00001142D5905F00F05156105682D59C5F330
:102BE0000725956105682C59240C54614FF4DC725B
:102BF000046802EB0112A4581C700468A458240A4B
:102C00005C700468A458240C9C700468A258120ECE
:102C1000DA704FF4DE72046802EB0112A4581C71E2
:102C20000468A458240A5C710468A458240C9C719C
:102C30000468A258120EDA71006881B1016941F08E
:102C400020010161002030BDE468A8E7416A41F439
:102C500000114162012030BD6D0D1560AFE7C16804
:102C600041F02001C160EDE72DE9F05F0546006805
:102C700000244669D0F804908768D0F80CB0D0F8EA
:102C800010A0D0F81880F10748D0F90714D001211E
:102C90008160B80703D5284600F063FA0CE0780796
:102CA00002D54FF4006407E0380702D54FF4805492
:102CB00002E0284600F054FAF80516D529684FF4CA
:102CC00080708860B80503D5284600F04CFA0CE007
:102CD000780502D544F4005407E0380502D544F4E1
:102CE000804402E0284600F03DFAF80316D5296832
:102CF0004FF480308860B80303D5284600F035FAD9
:102D00000CE0780302D544F4004407E0380302D510
:102D100044F4803402E0284600F026FA300707D554
:102D20005FEACB6004D52968102044F40074C860C1
:102D300070074FF0080707D55FEA0B7004D52868C5
:102D4000C760284600F060F9B00706D52868C0685B
:102D5000800702D0284600F059F9700607D55FEACF
:102D6000CA6004D52968102044F480640861B00664
:102D700007D55FEA0A7004D528680761284600F085
:102D8000BFF9F00606D528680069800702D02846FA
:102D900000F0B7F9B00308D55FEAC96005D5296826
:102DA00010204860284600F0ADF9F00307D55FEA2F
:102DB000097004D528684760284600F0D7F9300428
:102DC00046D55FEA497040D5F00504D55FEAC87082
:102DD00001D044F00104B00504D55FEA887001D544
:102DE00044F00204700504D55FEA487001D544F050
:102DF0000404300529D518F0700F26D008F07000B3
:102E0000402815D006DC102809D020280AD0302808
:102E100016D10AE050280ED0602811D10EE044F0FF
:102E200008040DE044F010040AE044F0200407E038
:102E300044F0400404E044F0800401E044F4807471
:102E40002868816921F07001816129680420486047
:102E5000002C05D0686A204368622846FFF78DFE83
:102E600000F000B830BCBDE8C09F70B5040003D0CE
:102E700094F8200010B104E0012070BD204600F05D
:102E800081F82068016841F00101016000F0B4FCA4
:102E90000546052604E000F0AFFC401B0A2811D8C7
:102EA00020684068C007F6D02068016821F0020160
:102EB000016000F0A1FC05460BE000F09DFC401B0A
:102EC0000A2806D9606A40F40030606284F8206005
:102ED000D2E7206840688007EFD4207E0128206870
:102EE00001683DD021F080010160607E01282068EA
:102EF000016838D021F040010160A07E01282068DF
:102F0000016833D021F020010160E07E01282068B3
:102F100001682ED041F010010160207F0128206857
:102F2000016829D021F008010160607F0128206834
:102F3000016824D021F004010160D4E902010843B2
:102F4000D4E90412114308436168491E084321680B
:102F5000C86100206062012084F82000002070BD5C
:102F600041F08001C0E741F04001C5E741F0200198
:102F7000CAE721F01001CFE741F00801D4E741F0A2
:102F80000401D9E710B586B0044614216846FDF760
:102F900038FA1B49206888422FD11A48816D41F0C8
:102FA00000718165816D01F000710591C16C41F086
:102FB0000101C164C06C694600F0010005904FF446
:102FC000C050009002200190002002900320039046
:102FD00009200490C00600F011FB002205211320F7
:102FE00000F0D6FC132000F0C5FC002206211420BE
:102FF00000F0CEFC142000F0BDFC06B010BD0000B7
:1030000000640040001002407047000010B58EB010
:10301000002001460A9003AA224801ABFFF7B0FD49
:1030200000283CD104980090B0F5102F12D11E4812
:103030009DF8041041709DF805108170BDF80610D0
:1030400049BAC170BDF8081049BA4171BDF80A10FB
:1030500049BA017114480499A438026C91421ED0F7
:10306000016400F1800400230AAA694620680BF07D
:10307000BFFC012813D00AAA0BA920680BF0C0FDE1
:10308000012801D009A008E000230AAA69462068A7
:103090000BF0AEFC012802D00EA005F0CBFE0EB066
:1030A00010BD00006C310010B80600105175657538
:1030B000652072656365697665206661696C656423
:1030C00020756E65787065637465646C792E0D0A81
:1030D000000000004661696C656420746F206F76A3
:1030E0006572777269746520717565756520776999
:1030F0007468206E657720646174612E0D0A00008B
:10310000704770477047000070B5044690F8200083
:10311000012804D0606A40F40020606218E00220B8
:1031200084F820002068016821F00101016000F0AE
:1031300063FB05460EE000BF00F05EFB401B0A2863
:1031400008D9606A40F400306062052084F82000ED
:10315000012070BD20684068C007EDD1606270BD7D
:10316000704770477047704770477047704710B599
:1031700090F825100022022905D00421C16380F8AF
:103180002420012010BD01680B6823F00E030B60A2
:1031900001680B6823F001030B6090F84410046C85
:1031A00001F01C03012101FA03F3636080F825108C
:1031B00080F82420104610BD10B590F8251000248A
:1031C000022903D00421C16301241AE001680A68BE
:1031D00022F00E020A6001680A6822F001020A6009
:1031E00090F84410036C01F01C02012101FA02F274
:1031F0005A6080F82510002180F82410816B01B1FD
:103200008847204610BDC06B7047F0B4016C0C6855
:1032100001680D6890F8442002F01C06042202FAAE
:1032200006F3234211D06B070FD50B689B0603D41E
:103230000B6823F004030B6090F8441001F01C01AC
:103240008A40016C4A60016B1DE0022303FA06F715
:1032500027424FF0000C4FF0010218D0AF0716D5EF
:103260000C68A40605D40C6824F00A040C6080F8ED
:10327000252090F8441001F01C018B40016C4B603C
:1032800080F824C0C16A00291AD0F0BC084708237E
:10329000B340234214D02B0712D50B6823F00E0342
:1032A0000B6090F84410036C01F01C0102FA01F16C
:1032B0005960C26380F8252080F824C0416BE2E7A2
:1032C000F0BC704770B568B12B4C036814212B4AD1
:1032D000A34209D22A4C1C44B4FBF1F18900C0E995
:1032E00010210BE0012070BD234C64421C44B4FB50
:1032F000F1F189004164204908390164022180F814
:1033000025101C6847F6F0718C43D0E9021529435B
:10331000D0E904563543294385692943C5692943C2
:10332000056A2943214319608168B1F5804F19D09E
:10333000036C0F21934202D152F8A83F02E00E4ADB
:10334000A032136890F8444004F01C04A1408B4361
:10335000136090F84430416803F01C0399401368EF
:10336000194311600021C163012280F8252080F8F3
:103370002410084670BD000008040240000002400E
:10338000F8FFFDBF70B5044690F824000025012821
:103390000CD0012084F8240094F825600020012E30
:1033A00006D084F824000225284670BD022070BD96
:1033B000022684F82560E0632068066826F001068E
:1033C00006602046FEF7B8F9206B002820680168E7
:1033D00002D041F00E0106E021F0040101602068F6
:1033E000016841F00A0101602068016841F00101B3
:1033F0000160D9E770B5044600F0FEF90546601C8F
:1034000002D004480078044400F0F6F9401BA042C2
:10341000FAD370BDE00600202DE9F05F0546324882
:103420008946017801290CD00126804606704CF2AD
:10343000503B5846FEF784FD07004FF0000A03D0CA
:103440004EE0022000F054B851464046C8F804A0AF
:10345000264C226892050AD52168490505D52168C0
:1034600021F480612160032109E0067708E02268E9
:10347000520504D5216821F4806121600221017781
:103480002868012807D04FF0FF31C9F8001040F23A
:10349000FA3BAE681DE06868FEF70CFD5846FEF783
:1034A0004FFD0746606920F00400606116E0304679
:1034B0006968FEF70DFD4CF25030FEF741FD070044
:1034C000606920EA0B00606102D0C9F8006005E085
:1034D000761CD5E902010844B042E8D8FEF7BCFCEE
:1034E00088F800A03846ADE7EC0600200020024036
:1034F00030BCBDE8C09F00000348416941F0004175
:103500004161002070470000002002402DE9FF5F6C
:10351000254C0646904620789A4601280BD001207B
:1035200020704CF2503B5846FEF70AFD07004FF062
:10353000000904D02AE0022004B000F039B848465F
:10354000C4F80490194D2968490504D5286820F469
:10355000806028600220207726B1012E09D0022E3B
:1035600007D00CE0424653460198FEF7C5FC012601
:1035700012E041460198FEF7CDFC022E0AD05846D3
:10358000FEF7DEFC4FEA0007FEF766FC84F80090C9
:103590003846D1E74FF480265846FEF7D1FC07465F
:1035A0006869B0436861EFE7EC0600200020024044
:1035B00030BCBDE8C09F0000064900204A69002ACF
:1035C00007DA054A8A60054A8A604969002900DAF3
:1035D000012070470020024023016745AB89EFCDF1
:1035E00070470000044910B50A68024202D0086022
:1035F000FFF7F6FF10BD0000140401402DE9F04F65
:10360000DFF8AC9100230325A9F1040B85B04FF03E
:10361000010C0F2709F1040AABF1040EBFE000BF53
:103620000CFA03F6324075D00C7904F00304012C37
:1036300001D0022C1BD1846800945C0005FA04F8C8
:103640000494009C24EA08040094D1F80C80049CA3
:1036500008FA04F8009C48EA0408C0F808804468A6
:10366000B4430E79C6F300169E40264346600C799B
:10367000E443A4070AD0C4684FEA430805FA08F6F1
:10368000B4438E6806FA08F62643C6600C7904F047
:103690000304022C10D1DC0800EB84040294246A99
:1036A0005E074FEAD66807FA08F6B4430E6906FAD1
:1036B00008F62643029C266204684FEA430805FA8E
:1036C00008F6B4430E7906F0030606FA08F6264318
:1036D00006604C6814F4403F60D0364C266E46F0CD
:1036E00001062666246E23F0030604F0010400940C
:1036F000314C34440294A4689E074FEA167807FAC6
:1037000008F6B443B0F1904F05D02C4EB04204D12E
:10371000012612E042E000260FE0294EB04201D11E
:1037200002260AE0274EB04201D1032605E0264ECC
:10373000B04201D1042600E0072606FA08F6264327
:10374000029CA660D9F800604C46D1F804809643EC
:103750005FEAC82800D516432660DAF800405646CE
:10376000D1F8048094435FEA882800D5144334607C
:10377000DBF800405E46D1F8048094435FEA883865
:1037800000D514433460DEF800407646D1F804805A
:1037900094435FEAC83800D5144334605B1C0A6860
:1037A00032FA03F47FF43CAF05B000F00FB800002C
:1037B00008040140001002400000014000040048DD
:1037C00000080048000C00480010004830BCBDE86C
:1037D000C08F0069084000D001207047426921EA8B
:1037E00002030A4043EA0241816170470AB18161E4
:1037F0007047816270470000014880687047000090
:10380000E006002070B5040011D021684CF6CC40D1
:103810000860216845F255500860D4E90001416014
:103820002168A0688860FFF7E7FF05460DE00120EA
:1038300070BD00BFFFF7E0FF401B312805D92068AD
:10384000C068400701D0032070BD2068C0684007F1
:10385000F0D120680269E1688A4201D0016102E08A
:103860004AF6AA210160002070BD00684AF6AA212C
:10387000016000207047000002488168027811440E
:1038800081607047E006002010B50024032000F09E
:103890009FF80F2000F008F808B1012401E000F0C3
:1038A0004FF8204610BD000030B505461F4887B0D0
:1038B000816D41F010018165806D06A900F0100056
:1038C000009001A800F028FB0498B0B100F044FB80
:1038D00040001749174AB0FBF1F11748491E026032
:1038E000416040F2E7320021C0E90321816081613B
:1038F00001F055FA040003D015E000F02DFBE8E7D5
:103900000D4801F07FFA04000DD1362000F032F8A6
:10391000102D07D200222946362000F039F807483A
:10392000056000E0012407B0204630BD00100240D1
:1039300040420F0000100040C8310010E406002093
:103940000B4882B0016E41F001010166016E01F089
:1039500001010091816D41F080518165806D0022EF
:1039600000F0805000900F21901E02B000F010B8BF
:1039700000100240002809DB00F01F0201219140E5
:103980004009800000F1E020C0F8001170470000FD
:10399000F0B40E4B1B680C46C3F30223C3F10705BA
:1039A000042D00D90425191D072901D2002300E0A8
:1039B000DB1E012606FA05F1491E214099409E4072
:1039C000761E16403143F0BC05F06CBA0CED00E0F9
:1039D000064900F0070208684FF6FF03184040EA66
:1039E0000220034A10430860704700000CED00E01D
:1039F0000000FA051649B0F5007F0868C0F34120C1
:103A000009D0022805D0086820F4C06040F4806026
:103A10000860002070470128FBD0086820F4C060CF
:103A200040F4007008600B483222006850430A4A94
:103A3000B0FBF2F0401C00E0401E4A69520501D57F
:103A40000028F9D148694005E3D5032070470000FC
:103A5000007000400C07002040420F000D4908682C
:103A600020F4804008600C483222006850430B4A22
:103A7000B0FBF2F0401C00E0401E4A69920501D5FF
:103A80000028F9D14869800501D50320704700203E
:103A900070470000007000400C07002040420F00FB
:103AA0000248016841F480410160704700700040A5
:103AB0000248006800F4C0607047000000700040D9
:103AC0000248016841F48071016070470070004055
:103AD00010B50C460E49002848690FD0C043800538
:103AE00001D5FFF7DDFF0B48016821F004010160FB
:103AF000012C0AD040BF20BF20BF10BD8005F2D5E9
:103B0000FFF7ACFF0028F8D1EDE730BF10BD000093
:103B10000070004010ED00E02DE9F84F044600274A
:103B20000088A84D3E46000515D5606C60B1B0F523
:103B3000000F04D0B0F5400F2BD001270AE0E86851
:103B400040F48030E86024E00021201D02F09AFC5F
:103B500007001ED03E46206880033AD5A86D4FF07E
:103B60000008C00009D4A86D40F08050A865A86D79
:103B70004FF0010800F080500090DFF84CA2DAF816
:103B8000001041F48071CAF80010FFF735FE81463D
:103B900010E0D5F88800616C20F440000843C5F8B7
:103BA0008800D8E7FFF728FEA0EB0900022801D91A
:103BB000032705E0DAF80000C005F3D5002F7DD01B
:103BC0004FEA0706B8F1000F03D0A86D20F080502F
:103BD000A8652078C00707D0D5F88800216A20F0B2
:103BE00003000843C5F888002078800707D5D5F87A
:103BF0008800616A20F00C000843C5F8880020782E
:103C0000400707D5D5F88800A16A20F030000843A6
:103C1000C5F888002078800607D5D5F88800E16AC5
:103C200020F440600843C5F888002088800507D547
:103C3000D5F88800E16B20F440200843C5F88800DF
:103C40002088400507D5D5F88800216C20F4401065
:103C50000843C5F888002078400607D5D5F88800C5
:103C6000216B20F440500843C5F8880020780006F6
:103C700007D5D5F88800616B20F440400843C5F8AB
:103C800088002088C00507D5D5F88800A16B20F4EE
:103C900040300843C5F8880020684FF000670003F3
:103CA0004FF0806850D5D5F88800A16C20F04060B6
:103CB0000843C5F88800A06CB84200E005E03BD19D
:103CC000E86840F48010E8603EE0D5F8900010F419
:103CD000407014D0A16D814211D0D5F89000D5F874
:103CE000901020F4407041F48031C5F89010D5F860
:103CF000901021F48031C5F89010C5F89000C007ED
:103D000011D0FFF779FD074641F2883907E000BF7F
:103D1000FFF772FDC11B494501D9032652E7D5F8CB
:103D200090008007F4D5D5F89000A16D20F4407084
:103D30000843C5F8900045E7404505D10121201D05
:103D400002F0A0FB00B106462068400317D5D5F865
:103D50008800E16C20F040600843C5F88800E06C02
:103D6000B84204D1E86840F48010E86007E04045BC
:103D700005D10121201D02F085FB00B106462088F7
:103D8000400411D5D5F88800216D20F0405008433B
:103D9000C5F88800206DB0F1805F05D10221201D9B
:103DA00002F070FB00B106462088000406D555F8E5
:103DB000880F616D20F0804008432860304600F095
:103DC00005B80000001002400070004018BCBDE8BB
:103DD000E08F00002DE9F0470F4605006BD0494EFB
:103DE000306800F00700B84209D2306820F00700C0
:103DF00038433060306800F00700B8425BD1287863
:103E0000414C80070AD5A868A16801F0F0018842FA
:103E100004D9A16821F0F0010143A1602878C0070E
:103E20002CD06868032811D0022812D0216898B1DC
:103E3000490500293FDAA16821F003010143A1608F
:103E4000FFF7DAFC804641F2883910E021688901E9
:103E5000EFE721688903ECE78907EAE7FFF7CCFC85
:103E6000A0EB0801494502D90320BDE8F087A0680E
:103E7000696800F00C00B0EB810FEFD12878800763
:103E80000AD5A868A16801F0F001884204D2A168AF
:103E900021F0F0010143A160306800F00700B84252
:103EA0000BD9306820F0070038433060306800F0EC
:103EB0000700B84201D00120D7E72878400705D590
:103EC000A068E96820F4E0600843A0602878000753
:103ED00006D5A068296920F4605040EAC100A060BE
:103EE00000F05EF8A168094AC1F30311515C01F0CA
:103EF0001F01C8400649086006480068BDE8F04751
:103F0000FFF7D2BC0020024000100240D8F20008A7
:103F10000C070020E40600200F2202600C4A936880
:103F200003F003034360936803F0F0038360936836
:103F300003F4E063C36092684FF4E06303EAD202E3
:103F400002610448006800F0070008607047000044
:103F500000100240002002400548064900688968B8
:103F6000054AC1F30221515C01F01F01C8407047AE
:103F70000C0700200010024018F30008054806490D
:103F800000688968054AC1F3C221515C01F01F0134
:103F9000C84070470C0700200010024018F30008CA
:103FA00070B52549002318468A68CC6812F00C02C7
:103FB00004F00306214C4FEA640509D00C2A05D011
:103FC000042A32D0082A00D1284670BD012E10D113
:103FD0000B681B0704D4D1F89430C3F3032302E029
:103FE0000B68C3F30313164E56F82330DAB10C2ACC
:103FF000EBD1C86800F00300022818D0032818D0BD
:104000001846CA68CB68C2F30212C3F306234343BF
:10401000521CB3FBF2F2C868C0F34160401C400080
:10402000B2FBF0F070BD184670BD204670BD204652
:10403000E7E72846E5E70000001002400024F4000E
:10404000E8F200082DE9F84304006FD0FA4DA868A3
:1040500000F00C06E86800F003072078C00664D57D
:1040600076B10C2E01D1012F0AD0A0690028286852
:104070007AD040F001002860FFF7BEFB80465DE08B
:104080002868800702D5A0690028DED0216A286848
:10409000000703D5286800F0F00004E0D5F894008C
:1040A000F02202EA1010814216D9084602F080FA86
:1040B00000283BD1286840F0080028602868216A61
:1040C00020F0F000084328606868E16920F47F4030
:1040D00040EA0120686016E0286840F00800286087
:1040E0002868216A20F0F000084328606868E169C8
:1040F00020F47F4040EA0120686026B9206A02F07F
:1041000057FA0028D5D1FFF74BFFA968CB4AC1F376
:104110000311515C01F01F01C840C9490860C9483A
:104120000068FFF7C1FB00287ED12EE0CAE000BF87
:10413000FFF762FBA0EB0800022876D8286880070A
:10414000F6D5286840F0080028602868216A20F029
:10415000F000084328606868E16920F47F4040EA85
:104160000120686011E0FFE720F001002860FFF700
:1041700043FB804606E000BFFFF73EFBA0EB0800D4
:104180000228DAD828688007F6D42078C00740D003
:10419000082E18D00C2E01D1032F14D06068B0F572
:1041A000803F17D0B0F5A02F286817D020F48030BA
:1041B0002860286820F4802028606068E0B1FFF75C
:1041C0001BFB804614E02868800322D56068002825
:1041D00078D01EE0286840F48030EDE740F480207D
:1041E0002860F7E7FFF708FBA0EB08006428A4D8D5
:1041F00028688003F6D50CE0FFF7FEFA804605E05C
:10420000FFF7FAFAA0EB0800642896D82868800324
:10421000F6D4207880073BD5042E11D00C2E01D186
:10422000022F0DD0E06801E0AAE1FFE00028286835
:104230001ED040F480702860FFF7DEFA07460CE0DD
:10424000286840050CD5E0680028C1D008E000BF10
:10425000FFF7D2FAC01B022893D828684005F7D58B
:104260006868217C20F0F85040EA016068600FE047
:1042700020F480702860FFF7BFFA074605E000BF12
:10428000FFF7BAFAC01B0228B1D828684005F7D456
:104290002078000729D560690028D5F8940012D04D
:1042A00040F00100C5F89400FFF7A6FA074604E0C5
:1042B000FFF7A2FAC01B022899D8D5F8940080070E
:1042C000F6D512E02BE120F00100C5F89400FFF7CD
:1042D00093FA074605E000BFFFF78EFAC01B0228DD
:1042E00085D8D5F894008007F6D42078400766D5A5
:1042F000A86D0027C00008D4A86D40F08050A865C4
:10430000A86D012700F0805000904F480168C90552
:1043100012D40168814641F480710160FFF76CFAA4
:10432000804605E0FFF768FAA0EB080002287DD878
:10433000D9F80000C005F5D5A068012816D00528D9
:10434000D5F8900017D020F00100C5F89000D5F8FE
:10435000900020F0040000BFC5F89000A06841F272
:104360008839C0B1FFF748FA80460FE0D5F89000D1
:1043700040F00100F0E740F00400C5F89000F5E7D8
:10438000FFF73AFAA0EB080149454FD8D5F890005D
:104390008007F5D50EE0FFF72FFA804606E000BF54
:1043A000FFF72AFAA0EB080149453FD8D5F890005D
:1043B0008007F5D41FB1A86D20F08050A865207843
:1043C000800628D5606A0028D5F8980012D040F001
:1043D0000100C5F89800FFF70FFA074605E000BF97
:1043E000FFF70AFAC01B022820D8D5F898008007EA
:1043F000F6D510E020F00100C5F89800FFF7FCF9B1
:10440000074604E0FFF7F8F9C01B02280ED8D5F8DC
:1044100098008007F6D4A06AF0B3022816D00C2EBC
:104420007DD0286820F08070286000E0A7E0FFF7CA
:10443000E3F90446A6E0000000100240D8F20008AC
:104440000C070020E406002000700040E868E26AE3
:1044500000F00301914228D1216B00F070020901A4
:104460001039914221D1626B00F4FE41B1EB022F71
:104470001BD194F8382000F07841B1EBC26F14D111
:10448000A18F00F4C00249084905A1F5001191422D
:104490000BD194F8401000E06AE04908490600F0AA
:1044A000C060A1F1007181424BD00C2E73D02868FE
:1044B000400170D4286820F080702860FFF79CF9D4
:1044C000064604E0FFF798F9801B022857D82868B1
:1044D0008001F7D4F4E90B016FF00F0202EB011138
:1044E0000843218A5204490802EB4151A26841EA7B
:1044F00002210843217D4FF07E42490802EB4161D1
:104500000843217B40EAC160E968244A114008431E
:10451000E860286840F080702860E86800E03AE0D1
:1045200040F08070E860FFF767F9044605E000BFDF
:10453000FFF762F9001B022821D828688001F7D50F
:1045400027E02868800124D4286840F08070286023
:10455000E86840F08070E860FFF74EF9044604E038
:10456000FFF74AF9001B022809D828688001F7D50F
:104570000FE000BFFFF740F9001B022802D903201B
:10458000BDE8F88328688001F4D4E868044908404D
:10459000E8600020F4E70120F2E700008C809D0134
:1045A000FCFFEEFE2DE9F05F044690F820009346F4
:1045B0008A46012825D0012684F82060022084F84C
:1045C00021002168CA20486221685320486220687F
:1045D000816821F4806181602068C16801F08001F8
:1045E00061F49061C1602068C0684FF00007400628
:1045F0004FF0FF081AD4FFF7FFF805464FF47A7919
:1046000010E0022000F03CB8FFF7F6F8401B4845E8
:1046100008D92168C1F82480032084F8210084F897
:104620002070EFE72068C0684007EDD52168C1F829
:1046300014A02068816821F0070141EA0B01816024
:104640000E48016841F4801101600C48083001688F
:1046500041F4801101602068816841F480418160EB
:104660002068816841F4806181602168C1F82480FC
:1046700084F8216084F820700020C3E70004014022
:1046800030BCBDE8C09F704710B50B4904464FF4DD
:10469000801008602068C168490508D5C16801F02C
:1046A000800161F49061C1602046FFF7ECFF0120BA
:1046B00084F8210010BD00001404014010B500680A
:1046C0000B4641680D480140080CD870C1F3042422
:1046D0005C7001F03F049C70C1F34231197052B913
:1046E00001F0A4FFD870587801F0A0FF58709878B6
:1046F00001F09CFF9870002010BD00003FFFFF00FC
:1047000010B50B460168896A596001680969C1F3EF
:104710000E019960006801680D480140C1F3054031
:104720001870C1F306245C7001F07F049C70890D41
:10473000D97052B901F07AFF1870587801F076FFFD
:104740005870987801F072FF9870002010BD00003A
:104750007F7F7F0010B504004FF0010044D094F833
:10476000210028B9002084F82000204600F040F8FD
:10477000022084F821002168CA2048622168532061
:104780004862204601F068FF00282DD1206881682A
:10479000164A11408160216888686268A3691043E5
:1047A00022691A43104388602168E0680861206824
:1047B0000169228941EA02410161204601F070FF4E
:1047C000002811D12168CA6C22F00302CA64626910
:1047D000E16911432268D36C1943D1642268FF2137
:1047E0005162012184F8211010BD0000BFFF8FFF2E
:1047F00010B598B004465C216846FBF702FE0F49ED
:104800002068884218D14FF4003000904012169072
:104810006846FFF781F908B1FDF71CFB084850F81E
:10482000901F41F400410160002205210320FFF7A1
:10483000AFF80320FFF79EF818B010BD0028004025
:104840000010024070B5044690F820000B46012885
:104850001BD0012684F82060022084F82100B2B128
:104860009878D97840EA014558781978000240EAEA
:10487000413005432168CA204862216853204862BC
:10488000204601F0E9FED0B120E0022070BD58784A
:10489000C10603D500F0EF000A305870D87801F057
:1048A000CEFE0504587801F0CAFE45EA0025987846
:1048B00001F0C5FE0543187845EA4035DAE70848B7
:1048C000054020684560204601F0EAFE2268FF218D
:1048D000516208B984F82160002184F8201070BD6D
:1048E0003FFFFF002DE9F041044690F8200090467C
:1048F0000D46012811D0012784F82070022084F889
:1049000021002168CA20486221685320486220465D
:1049100001F0A2FE002618B129E00220BDE8F081D6
:104920002068B8F1000F80684FEA406024D000286A
:1049300000DBEE70A8782978EA7840EA01406978CF
:10494000090241EA82510843184908402168086079
:104950002068816821F480218160D5E90301084342
:1049600021688A6810438860204601F099FE226819
:10497000FF215162A0B115E0002800DBEE7028781D
:1049800001F05DFE0304687801F059FE43EA00235C
:10499000A87801F054FE0343E87843EA8050D3E757
:1049A00084F8217084F82060B8E700007F7F7F00E2
:1049B00070B504460068C16821F0A001C160FEF72F
:1049C0001BFF05464FF47A7607E000BFFEF714FFA1
:1049D000401BB04201D9032070BD2068C06880062A
:1049E000F4D5002070BD70B5040009D0606A0025C0
:1049F00040B125616561A56294F85D0040B10CE0AD
:104A0000012070BD6068B0F5827FF4D0E561F2E707
:104A100084F85C50204600F057F8022084F85D00CE
:104A20002068016821F040010160E1684FF4E06214
:104A3000914201D9002001E04FF48050B1F5706F30
:104A400002D0914200D0A562A188228901F482712E
:104A500002F404421143227C02F002021143227D3F
:104A600002F001021143228B02F400721143227FF3
:104A700002F03802114394F8202002F08002114322
:104A8000228D02F40052114322681160A1690422B0
:104A900002EA114194F8242000F4805002F0100240
:104AA000114394F8342002F008021143A28902F461
:104AB000706211430143206841602566012084F83B
:104AC0005D00002070BD000010B586B004461421C2
:104AD0006846FBF796FC1349206888421FD11248AC
:104AE000816D41F480418165816D01F480410591C2
:104AF000C16C41F00201C164C06C694600F0020063
:104B000005904FF460400090022001900120029037
:104B100003200390052004900448FEF76FFD06B0C3
:104B200010BD0000003800400010024000040048A2
:104B30002DE9F05F044690F85C0000270A9E1D46B0
:104B400092468B464FF0010901280ED0012084F8CF
:104B50005C00FEF751FE804694F85D006168012814
:104B60000CD0B1F5827F07D102E0022000F011B92C
:104B7000A16809B9042801D0022700E1BBF1000FA8
:104B800024D0BAF1000F21D005B394F85D000428B9
:104B900002D0052084F85D0000202066C4F840A003
:104BA000A4F84650A4F84450C4F838B0E587A58767
:104BB000E0642065E0684FF4E061884201D8012D8F
:104BC00006D92068426822F4805205E00127D6E029
:104BD0002068426842F480524260206802685206AF
:104BE00003D4026842F040020260E06888426068D4
:104BF00045D908B1012D3AD1A06B21680088C86061
:104C0000A06B801CA063E08F401EE0872FE020682F
:104C1000816889070FD5E18F69B1B9F1010F0AD118
:104C2000A16B0988C160A06B801CA063E08F401E4F
:104C3000E0874FF0000920688168C9070FD0B4F8F9
:104C4000461061B1C068216C0880206C801C206413
:104C5000B4F84600401EA4F846004FF00109FEF7E4
:104C6000CBFDA0EB0800B04201D3701C75D1E08FE2
:104C70000028CCD1B4F846000028C8D176E008B1AD
:104C8000012D6CD1E08F0128A06B08D92168008824
:104C9000C860A06B801CA063E08F801E07E02168C5
:104CA00000780873A06B401CA063E08F401EE08773
:104CB00055E02068816889071AD5E18FC1B1B9F143
:104CC000010F15D1E18F0129A16B07D90988C160B6
:104CD000A06B801CA063E08F801E06E00978017342
:104CE000A06B401CA063E08F401EE0874FF00009DE
:104CF00020688168C90728D0B4F8461029B3B4F8F1
:104D00004610012914D9C068216C0880206C801CD1
:104D10002064B4F84600801EA4F84600B4F84600AB
:104D2000012810D82068416841F4805141600AE0B0
:104D3000007B216C0870206C401C2064B4F8460095
:104D4000401EA4F846004FF00109FEF755FDA0EB08
:104D50000800B04202D3701C01D018E0BEB1E08F51
:104D60000028A6D1B4F846000028A2D14246314618
:104D7000204601F0A5FD10B101272020206601206A
:104D800084F85D00002084F85C003846EEE60327D6
:104D9000F5E730BCBDE8C09F70477047704710B55D
:104DA000040003D094F83D0010B107E0012010BDCD
:104DB000002084F83C00204600F022F8022084F80D
:104DC0003D00211D206803F09FF8012084F8480071
:104DD00084F83E0084F83F0084F8400084F84100E5
:104DE00084F8420084F8430084F8440084F84500C5
:104DF00084F8460084F8470084F83D00002010BD88
:104E00007047000090F83D10012901D00120704743
:104E1000022180F83D100168CA6842F00102CA60B0
:104E200000680B49884205D0B0F1804F02D0094993
:104E3000884207D18168084A1140062906D0B1F599
:104E4000803F03D0016841F00101016000207047FC
:104E5000002C01400040014007000100704770B580
:104E60000446006801694FF00005C943890715D45D
:104E7000C168C943890711D4E91E01610120207767
:104E8000206880698007204602D0FFF7E7FF04E032
:104E900000F0A7F8204600F0A5F825772068016902
:104EA000C943490717D4C168C943490713D46FF0F0
:104EB00004010161022020772068806910F4407F9E
:104EC000204602D0FFF7CAFF04E000F08AF820462F
:104ED00000F088F8257720680169C943090716D4CE
:104EE000C168C943090712D46FF0080101610420A9
:104EF00020772068C0698007204602D0FFF7AEFF08
:104F000004E000F06EF8204600F06CF82577206889
:104F10000169C943C90617D4C168C943C90613D476
:104F20006FF010010161082020772068C06910F43B
:104F3000407F204602D0FFF791FF04E000F051F8D7
:104F4000204600F04FF8257720680169C943C9075A
:104F500008D1C168C943C90704D1891E016120462F
:104F600000F042F820680169C943090609D4C16804
:104F7000C943090605D46FF0800101612046FFF79F
:104F80000CFF20680169C943C90509D4C168C94338
:104F9000090605D46FF4807101612046FFF7FCFE1D
:104FA00020680169C943490609D4C168C943490653
:104FB00005D46FF040010161204600F01FF8206821
:104FC0000169C94389060BD4C168C943890607D45E
:104FD0006FF0200101612046BDE87040FFF7DEBEA2
:104FE00070BD70477047000000680349884201D1D6
:104FF000FEF742BC70470000001000407047704749
:10500000704770B50446806FE66F216889684FF07D
:105010001005090618D5212816D12068083050E857
:10502000001F21F0800140E80012002AF5D1E06E57
:1050300038B1FEF79CF820B1E06EFEF7E4F82028C6
:1050400021D0204603F0F1F820688068400618D58A
:10505000222E16D12068083050E8001F21F04001B0
:1050600040E80012002AF5D1206F38B1FEF77FF832
:1050700020B1206FFEF7C7F8202804D0204603F0A7
:10508000AFF8002070BDC4F88050032070BD000050
:1050900000680549884206D1012101628215034951
:1050A000034800F0D5BA7047004400401E000010CD
:1050B000F83A00202DE9F04102680446D0691168F1
:1050C000936840F60F0528424FF0000505D186068B
:1050D0007ED58E067CD5616E1BE1994F03F00106EB
:1050E0000F40374374D0C70709D0CF0507D5012734
:1050F0001762D4F8802042F00102C4F880208207B1
:105100000AD5DA0708D0276802223A62D4F880204C
:1051100042F00402C4F8802042070AD5DA0708D01A
:10512000236804221A62D4F8802042F00202C4F8F4
:10513000802002070CD501F02002324308D02368FA
:1051400008221A62D4F8802042F00802C4F88020B5
:1051500002050BD54A0109D523684FF400621A6293
:10516000D4F8802042F02002C4F88020D4F88020B7
:10517000002A35D0800605D5880603D5616E09B1B1
:1051800020468847D4F8800021688968490602D4FF
:1051900010F0280F26D0204603F022F820688068FF
:1051A00040061AD52068083050E8001F21F0400161
:1051B00040E80012002AF5D1206F70B16149816387
:1051C000206FFDF7F9FF00280AD0206F816B01E006
:1051D0000EE02046BDE8F04108472046FFF758FFA3
:1051E000BDE8F0812046FFF753FFC4F88050F7E791
:1051F000276E2026012F7BD1C70679D5CF0677D51C
:105200001020106220688068400641D5216F086830
:1052100040680004000CE3D0B4F858208242DFD983
:10522000A4F85A000868006880062AD4206850E86C
:10523000001F21F4807140E80012002AF6D1206896
:10524000083050E8001F21F0010140E80012002A58
:10525000F5D12068083050E8001F21F0400140E8F7
:105260000012002AF5D1E6672566216851E8000F93
:1052700020F0100041E80002002AF6D1206FFDF76F
:1052800076FFB4F85800B4F85A10401A81B22AE0F8
:10529000B4F85800B4F85A10401A81B2B4F85A0061
:1052A00000289DD000299BD0226852E8000F20F4EE
:1052B000907042E80003002BF6D12068083050E8D7
:1052C000002F22F0010240E80023002BF5D1E66711
:1052D00025666566226852E8000F20F0100042E85B
:1052E0000003002BF6D12046FFF789FE78E7FFE7A1
:1052F000C70209D55B0207D54FF480101062204623
:10530000BDE8F041FFF77CBE020606D50A0604D5CB
:10531000A16E00297FF45DAF62E74006E6D548063E
:10532000E4D52046026852E8001F21F0400142E81F
:105330000013002BF6D18667856600F097FA4FE7D9
:10534000200100049980000810B5040002D0A06F6D
:1053500010B107E0012010BD002084F87400204641
:1053600000F026F82420A0672068016821F00101E0
:105370000160204602F066FF0128ECD0606A10B19F
:10538000204602F0F7FD2068416821F49041416019
:105390002068816821F02A0181602068016841F05D
:1053A000010101602046BDE8104002F047BE000048
:1053B0002DE9F04F9DB00446142117A8FBF721F802
:1053C0005C216846FBF71DF8974A2168974D00203D
:1053D000022780264FF003084FF007094FF0100A0C
:1053E000914257D101218346089000916846FEF70B
:1053F00093FB08B1FCF72EFD286E40F48040286630
:10540000286E00F480401C90E86C40F00100E864D5
:10541000E86C18AA00F001001C904FF4C0601790CF
:1054200002205D4682E8210317A94FF09040FEF765
:10543000E5F8804F7E4838600220C7E90105C7E9DA
:1054400003567D61BD61FD6138463D62FDF73AFF5F
:1054500008B1FCF7FFFC2767BC62764F74484837F9
:1054600014383860C7E903567D61BD61FD610220D3
:105470003D62C7E9010A3846FDF724FF08B1FCF791
:10548000E9FCE766002206212520BC62FEF780FACF
:10549000252062E0684A914264D10020099000977B
:1054A0006846FEF739FB08B1FCF7D4FCA86D40F460
:1054B0000030A865A86D00F400301C90E86C40F046
:1054C0000100E864E86C19AA00F001001C900C20AF
:1054D000CDE91707002582E82003BB4617A94FF046
:1054E0009040FEF78BF8DFF84C81514908F19008A5
:1054F00014314046C8F80010C0E90175C0E90356F0
:10550000C8F81450C8F81850C8F81C50C8F82050F3
:10551000FDF7D8FE08B1FCF79DFC464FC4F870803B
:10552000D837C8F82840C7F808A0C7E903567D61F6
:105530003F48BD61FD6128303D62C7E9000B384638
:10554000FDF7C0FE08B1FCF785FCE76600220521E7
:105550002620BC62FEF71CFA2620FEF70BFA1DB0CF
:1055600000F072B8354A9142F9D104210091834686
:105570000A906846FEF7D0FA08B1FCF76BFCA86DFC
:1055800040F48020A865A86D00F480201C90E86C91
:1055900040F00200E864E86C022700F002001C9072
:1055A0004FF44060CDE9170719AA5D4682E8200351
:1055B00017A92348FEF722F81D49DFF8888028390B
:1055C0004046C8F80010C0E90175C0E90356202123
:1055D000C8F81450C8E90651C8F82050FDF772FE0B
:1055E00008B1FCF737FC174F1148C4F870804837F2
:1055F0003C38C8F828403860C7E903567D61BD6172
:10560000FD6102203D62C7E9010A3846FDF75AFEF6
:1056100008B1FCF71FFCE766002206212720BC62C8
:10562000FEF7B6F9272098E7003801400010024045
:1056300058000240003C0020004400400048004068
:1056400000040048203D002030BCBDE8C08F0000B1
:1056500030B4C36F202B20D1E1B1DAB190F87430AF
:10566000012B1AD0012380F87430002303660C4C00
:105670000368A3420BD05B681B0208D5046854E89A
:10568000003F43F0806344E80035002DF6D130BC84
:1056900002F0D8BE012030BC70470220FBE70000BA
:1056A0000080004010B5044696B028211448FAF74F
:1056B000A8FE282213491248FAF77CFE12492068F6
:1056C00088421AD10020149028220E496846FAF721
:1056D00071FE0E4C002314AA6946A06809F088F9EF
:1056E00001280AD014AA0AA9A06809F089FA00239F
:1056F00014AA6946A06809F07BF916B010BD000035
:10570000200300101E00001000440040940600100A
:10571000704700002DE9F8430446806F1F46164687
:105720000D4620284FD1CDB1C6B194F874000128A0
:1057300049D0012084F874004FF00008C4F880803C
:105740002120A067FEF758F8A4F850608146A4F81D
:105750005260A068B0F5805F03D004E00120BDE88E
:10576000F883206928B12E465FF0000584F8748024
:1057700010E00026FAE78021204602F0B5FEB8B915
:10578000C6B116F8010B21680885B4F85200401E16
:10579000A4F85200B4F852004B464FF000020097B4
:1057A0000028E8D14FF04001204602F09DFE30B1C4
:1057B0000320D4E735F8020BC0F30800E3E720200C
:1057C000A0670020CBE70220C9E7000070B50446BF
:1057D000806F202841D169B362B394F87400012826
:1057E0003BD0012084F87400E164A4F85020A4F8B0
:1057F00052200025C4F880502120A067E06ED8B167
:105800001749C162E16E174813460863E16E1648F6
:105810004863E06E85632668E16C06F12802E06E5D
:10582000FDF7B0FD40B11020C4F8800004F8745FAB
:1058300020206060012070BD21684020086284F84B
:1058400074502068083050E8001F41F0800140E8A3
:105850000012002AF5D1002070BD022070BD0000AA
:1058600095810008D7810008AD8000087047704717
:10587000FEE700000026DFF898A1664CDFF898915B
:1058800037460125B046052006F0EBFB761CB6B284
:10589000FBF784FE642E07D320215046FDF79EFFC0
:1058A00000265E48FDF7E1FF607DA16B884201D0D4
:1058B000607DA063607D012802D0607D78B11EE02C
:1058C000207D012809D0012211464846FDF78EFFB0
:1058D00065740720E07084F81B8025750FE00022B6
:1058E00001214846FDF782FF0920E07084F8168008
:1058F0000321C4E90C5184F81B8084F81480A0793A
:10590000012804D0A079022801D040460EE0A079F9
:1059100002280AD0E079022807D0207A022804D091
:10592000607A022801D0257601E002202076207ED0
:10593000022803D0207E00283ED047E07F1CBFB263
:105940004FF400614846FDF744FF70B30020A07299
:10595000B8B1002204214846FDF748FF012006F0B7
:1059600051F8012208215046FDF740FF00224FF474
:1059700080514846FDF73AFF29A003F05BFA84F80E
:10598000178010215046FDF724FF88B10020E072F7
:1059900080B1012006F03EF82BA003F04BFAB7F5DA
:1059A000FA5F13D3A573002710E0FFE70120CEE7CD
:1059B0000120ECE7A57309E010215046FDF709FF2F
:1059C000A0B10020E07298B184F80E8020790128FF
:1059D00012D0002280214846FDF708FF0022102146
:1059E0004846FDF703FFC4F84C804CE70120E9E787
:1059F000002006F00FF8E7E7012280214846FDF776
:105A0000F5FE012210214846FDF7F0FEE5643AE775
:105A100000040048140600100008004894310010EB
:105A200053595354454D5F4C4556454C5F322061A8
:105A300063747561746F725F706F7765725F6F709A
:105A4000656E65640A0000006761735F706F77655B
:105A5000725F6F70656E65640A00000030B50021EA
:105A6000254B264C4FEA010001EB410203EBC20536
:105A700003F832006870A870A88044F8220004EB94
:105A80008202491C10719071D071C9B210721E2926
:105A9000EAD31B4A002100BF42F8310002EBC103E8
:105AA000491C18719871C9B2D8710329F4D3144BE9
:105AB0000021183301EB4102491C43F8220003EB9B
:105AC0008202C9B210719071D071107250720329A4
:105AD000F0D30B4B00213C3301EB4102491C43F84E
:105AE000220003EB8202C9B210719071D071107262
:105AF00050720329F0D330BDE80B001048030010AA
:105B0000B004001000EB8100006E00F0F840704718
:105B10008068C0F3C00070478068C0F380007047A1
:105B2000C06810F4406F01D000207047012070471A
:105B3000042303EAD15310B518444369C1F3045157
:105B400007248C40A3438A401343436110BD00EBFC
:105B50008100016E21F00041114301667047000091
:105B600008B5012269460348FCF77EFA024900980D
:105B7000086008BD00EC0108F406001030B58BB0D9
:105B8000214914226846FAF715FC1F4914221431E2
:105B900005A8FAF70FFC00210C4608466A46135C7C
:105BA000FF2B01D0012102E0401C1428F7DB00206C
:105BB00005AA135CFF2B01D0012402E0401C14282D
:105BC000F7DB29B1142269461048FAF7F3FB07E026
:105BD00014210E48FAF715FC0DA10C48FAF758FCF1
:105BE0000A4D143534B1142205A92846FAF7E2FB10
:105BF0000BB030BD14212846FAF703FC06A1284655
:105C0000FAF746FCF4E7000000DC0108C4060010C7
:105C100042415453555256006169726C696E657306
:105C20000000000008B5012269460448FCF71CFA90
:105C300003A0009903F0FEF808BD000000E401088D
:105C400056657273696F6E203078253034780D0A8E
:105C50000000000030B587B018216846FAF7D1FB84
:105C6000184817490024C0E9001484600425C46062
:105C7000C0E90445047644760121C16180F82040E2
:105C80008462C46280F83040446380F83840FCF796
:105C9000B1FC08B1FCF7DEF80B480090062001903B
:105CA00002907F200594CDE9030569460548FCF77D
:105CB000A5FA002801D0FCF7CDF807B030BD0000F0
:105CC00000000450AC39002040002019104810B5E5
:105CD0000E4901600221416000214FF430228160B1
:105CE000C0E903124FF400124261017601224276AC
:105CF0008176C27601774277FDF7B7F8002803D0A6
:105D0000BDE81040FCF7A6B810BD000000640040DC
:105D10006C3100101D4808B5816C41F001018164AF
:105D2000806C002200F00100009005210C20FDF79E
:105D30002FFE0C20FDF71EFE002205210D20FDF791
:105D400027FE0D20FDF716FE002205210E20FDF78F
:105D50001FFE0E20FDF70EFE002205210F20FDF78D
:105D600017FE0F20FDF706FE002205211020FDF78B
:105D70000FFE1020FDF7FEFD002205211120FDF78A
:105D800007FEBDE808401120FDF7F4BD00100240F9
:105D900070B5384806F0D4F9374C364A01212061F5
:105DA0001032084606F000FA324A4FF4007560617E
:105DB000603A0C21284606F097F92E4A2060483AAE
:105DC0001221284606F090F92A4A6060303A2821CC
:105DD000402006F089F9274AA060183A52211E2077
:105DE00006F082F9E060803C207908B1012800D1FA
:105DF000E064FFF733FEFBF733FC00F0F7FE00F042
:105E00009DFC00F0E3FCFFF7ABFE00F03BFDFFF76D
:105E100009FF1A4A00211A4806F012FA174A60666A
:105E200024320021174806F00BFA144AA0664832C3
:105E30000021154806F004FA104AE0666C32002191
:105E4000124806F0FDF90D4A2067903200211048F3
:105E500006F0F6F9074A6067A83A00210D4806F0F7
:105E6000EFF9044AA067843A00210B4806F0E8F9EC
:105E7000E06770BDB8F20008940600105CF10008FD
:105E8000755800088116000849DE0008759B000857
:105E90008DBB0008D99D0008417E00082DE9F04324
:105EA00087B014216846FAF7ACFA4448C16C41F057
:105EB0000401C164C16C01F004010591C16C41F0A1
:105EC0000101C164C16C01F001010591C16C41F097
:105ED0000201C164C16C01F002010591C16C41F085
:105EE0000801C164C06C364E00F008000590002225
:105EF00041F693413046FDF779FC00224FF4807162
:105F00003046FDF773FCDFF8BC90012204214846BF
:105F1000FDF76CFC002241F278014846FDF766FC73
:105F20004FF0904700224FF400413846FDF75EFCE9
:105F3000DFF89480012204214046FDF757FC41F62A
:105F40009750009001250024CDE901546946304660
:105F50000394FDF753FB41F27C000090CDE901541E
:105F6000694648460394FDF749FB48F2100000904B
:105F7000CDE90154694638460394FDF73FFB042000
:105F80000090CDE90154694640460394FDF736FB85
:105F9000802000904FF44410CDE901046946484642
:105FA000FDF72CFB002205211720FDF7F1FC17203F
:105FB000FDF7E0FC07B0BDE8F083000000100240F0
:105FC0000008004800040048000C00480A4810B5CA
:105FD000084901600421416040F6FF71C1608160A1
:105FE000FDF710FC002803D0BDE81040FBF732BFDE
:105FF00010BD00000030004094310010104810B572
:106000000E49016000217F22C0E90112FF22C0E990
:10601000032141618161C161FEF79CFB08B1FBF77F
:1060200019FF042200210648FEF7BCFA002803D01D
:10603000BDE81040FBF70EBF10BD00000028004077
:10604000A4310010124810B5104901604FF482715C
:10605000416000214FF4E062C0E9021202220261B5
:1060600001224261520282611022C0E90721072207
:106070004162C0E90A1201634163FEF7B4FC0028E3
:1060800003D0BDE81040FBF7E5BE10BD003800406E
:10609000103A00200D4810B50B4901604FF4E13172
:1060A0004160002181600C22C160C0E9041281615D
:1060B000C16101624162FFF747F9002803D0BDE8E2
:1060C0001040FBF7C7BE10BD00380140743A0020F5
:1060D0000D4810B50B4901604FF416514160002185
:1060E00081600C22C160C0E904128161C16101625A
:1060F0004162FFF729F9002803D0BDE81040FBF703
:10610000A9BE10BD00440040F83A00200D4810B56B
:106110000B4901604FF4E1314160002181600C22A4
:10612000C160C0E904128161C16101624162FFF78F
:106130000BF9002803D0BDE81040FBF78BBE10BD63
:10614000004800407C3B0020FEE700002DE9F04FB6
:1061500087B005007DD02868020FC0F30751C0F357
:106160000733C0F3032CC0F3031472D0DFF830926E
:106170008A4A0127A9F2AD1B4FF00008A9F2E510E9
:10618000102967D31039CEB28DF800808DF80160E8
:106190001E2E6DD200F2844A012C1FD0022C67D132
:1061A00006EB46010AEBC104A08820B16078984252
:1061B00004D0A4F80480637084F802C06868C4F84E
:1061C0000900A868C4F80D00507E6074A088002102
:1061D00040F00402A2800846A37853E029790329FD
:1061E00001D9002101E00229FBD8815500210B468D
:1061F000C45C8C4200D921465B1CDBB21E2BF7D35A
:1062000011B1012900D002219346917106EB460499
:106210004846211809EB0600A1F8008081F80280A9
:1062200035F8052F0A80AA788A7080F87870FDF713
:10623000E3FA01465B4840F8241000EB8400077144
:1062400080F805802888ADF80200A8788DF8040051
:1062500001E00DE04BE08DF805800AEBC4002979E0
:1062600081716979C171A9790172E9788BF8191086
:1062700007B000F09BB800BF07FA00F50D43401CC3
:10628000A9B2C0B28342F7D8491C8A4201D1A7758E
:1062900002E0A07D0128EBD1A11D10220DF10A0022
:1062A000FAF788F83D488DF8096080308DF808804D
:1062B0004068B8B100231A4602A908F0DDFA9DF83B
:1062C0000910DDF80A3001EB41020BEB82020BEB07
:1062D00001001360DDF80E305360DDF8123093607A
:1062E00080F8867120461821FAF78BF8C0E702295A
:1062F000BED3891E8DF80070CCB28DF8014029798B
:10630000022900D00021254E26360023315519469A
:1063100016F801C09C4500D9435C491CC9B2032949
:10632000F6D3C3B30220D07135F8056FADF8026023
:10633000FDF762FA01461C4840F8341000EBC40037
:1063400009EB4401077180F8058009EB0400A1F80E
:106350005A6080F896708DF808709DF801008DF8ED
:1063600009002888ADF80A000C48803040680028F1
:10637000BCD000231A4602A908F07EFA9DF8091045
:10638000BDF80A300BEB41020BEB0100A2F86831BB
:1063900080F8A4716CE7FFE70020C4E71406001042
:1063A0004909001048030010B004001030BCBDE8DB
:1063B000C08FFEE710B596B004462C2104A8FAF76A
:1063C00020F815A12046FAF727F800280ED00FACC8
:1063D00010AB11AA12A98DE81E0013AB14AA10A1CC
:1063E000801DFAF77DF8062802D0002016B010BDF7
:1063F0001498A0F26C7009901398401E089012989F
:10640000079011980690109805900F98049004A892
:10641000F9F77CFFEAE700002B54494D453A0000AC
:1064200025642D25642D25642C25643A25643A25A0
:1064300064000000084810B5417C012909D0807B28
:10644000002808D007F072FABDE81040012005F0DE
:1064500008BEFBF701FA10BD140600100EB5084C7B
:10646000206840B10022694608F02EFB012802D1C5
:106470006846FFF76BFE012005F0F3FDF0E7000032
:10648000940600102DE9F041444C05468846E0682A
:106490000026810728680DD0E16801F003018142E0
:1064A00016D1A8B1E0686968C0F30210401C8842A8
:1064B0000ED120E0012804D0022805D0032807D1FE
:1064C00008E02168890701E021684905002907DB08
:1064D00001265FE02168890302D421684903F5E7BA
:1064E000E1686A686FF00F0321F0730103EB021299
:1064F00011430143E160206820F080602060FDF7D7
:106500007BF9074605E000BFFDF776F9C01B0228BE
:1065100037D820680001F7D4B8F1000F18D0B8F1CF
:10652000010F1DD0287D4FF07E41400801EB4060F7
:10653000A96840EA01202169194A114008432061F5
:10654000206840F080602060FDF756F907461AE0A9
:10655000A868297B000240EAC1602169114AECE782
:10656000288A1149400801EB4050A96840EA0120FF
:1065700021690E4AE1E700BFFDF73EF9C01B022882
:1065800001D9032606E020680001F5D52069A96934
:10659000084320613046BDE8F08100000010024051
:1065A000FF80FFF9FF80FF070000E0FFFF809FFFF3
:1065B000F8B51C4D06460024A86DC00002D5FDF7B5
:1065C00077FA0DE0A86D40F08050A865A86D00F046
:1065D00080500090FDF76CFAA96D21F08051A965FB
:1065E000B0F5007F04D0802E07D94FF003040AE0F5
:1065F000802E08D9A02E01D804E001D1022402E0A7
:10660000702E00D101240848016821F007012143C0
:106610000160006800F00700A04201D00120F8BD31
:106620000020F8BD0010024000200240010901EBEB
:10663000810100F00F0000EB4100C0B27047002262
:10664000014602E00A39C9B2521C0A29FAD21007DF
:1066500041EA1060704700002DE9F04104460068EF
:106660000025C168490617D4691EC160FDF7C4F84A
:1066700006464FF47A78032708E000BFFDF7BCF820
:10668000801B404502D9032584F821702068C0682A
:10669000400601D4032DF1D12846BDE8F081000069
:1066A0002DE9F041064613480025016821F08001DC
:1066B0000160041F20684FF00307800607D43046AE
:1066C000FEF776F990B186F8217003250EE0206878
:1066D00020F0200020603046FEF76AF910B186F8FD
:1066E00021700325206840F0200020602846BDE886
:1066F000F08100000C2800400148FDF7C5BF0000F4
:10670000A431001070B500242546661E0A48FCF727
:10671000E9F831460848FCF78DF818B90648FBF748
:1067200066FF04440448FCF721F96D1C0A2DEDDBDB
:106730000A20B4FBF0F070BDAC390020214910B53F
:106740000A782148FF2A00D1002202704B783C22AF
:10675000FF2B1BD043708C786423FF2C18D08470DF
:10676000CC78FF2C16D0C4700C790A23FF2C13D0E0
:1067700004714C79FF2C11D044718B790124FF2BCB
:106780000ED08371CB79FF2B0CD00CE04270E2E786
:106790008370E5E7C370E7E70371EAE74371ECE76D
:1067A0008471EFE71E23C3710B7AFF2B05D00372B0
:1067B000497AFF2903D0417210BD0472F8E7427292
:1067C00010BD000000FC0108B8060010F0B5254817
:1067D0008AB0254D016806918488ADF81C40837904
:1067E0008DF81E30D0F807100891B0F80B20ADF8E6
:1067F0002420417B002006AE375CFF2F16D0401CC2
:106800000728F9DB06982860AC80AB71174B002095
:1068100008AC255CFF2D16D0401C0628F9DB089833
:1068200018609A801248FF2917D017E011A3D3E906
:106830000003CDE901032860BDF80800A8809DF899
:106840000A00A871E2E70DA2D2E90002CDE9010237
:106850001860BDF808009880E4E70121C1720AB011
:10686000F0BD000000F40108CE060020C80600209C
:10687000B806001020240000001500002024120497
:106880000015000008B5012269460548FBF7ECFB3E
:1068900004480099016004A002F0CCFA08BD000091
:1068A00000D4010860060010776966696F7234478A
:1068B0005F666C6167203078253034780D0A0000FF
:1068C000F8B515460E460B460092044600224FF4DA
:1068D000C05100F019F888B93346002280212046C3
:1068E000009500F085F848B9334600224FF4C061A6
:1068F0002046009500F008F8002804D0206E40F0F3
:10690000200020660320F8BD2DE9FE4F4FF0000A5D
:10691000984617460E4604460C9D8DF804A0FCF7D9
:106920006BFF411BA8EB0105FCF766FF8146206861
:106930004FF4C06B0C3002902A480068C0EBC000D6
:1069400000EB8000000D6843009043E05E4506D1F7
:106950002FB9029800788DF804009DF80400B8F172
:10696000FF3F37D0FCF748FFA0EB0900A84203D255
:1069700015B1009858B32BE02068416821F0E00180
:1069800041606068B0F5827F0BD1A068B0F5004F20
:1069900002D0B0F5806F04D12068016821F0400179
:1069A0000160A06AB0F5005F09D12068016821F498
:1069B000005101602068016841F40051016001202C
:1069C00084F85D0084F85CA0032000F00DB8002579
:1069D000401E0090206880683040B842B6D1002048
:1069E000F3E700000C0700201EBCBDE8E08F0000AC
:1069F0002DE9F8431E46914688460446089DFCF75B
:106A0000FBFE401B351AFCF7F7FE074625480068D9
:106A1000C0F3CB30684338E0701C37D0FCF7ECFE95
:106A2000C01BA84203D215B1009860B32CE02068C7
:106A3000416821F0E00141606068B0F5827F0BD1D0
:106A4000A068B0F5004F02D0B0F5806F04D1206887
:106A5000016821F040010160A06AB0F5005F09D132
:106A60002068016821F4005101602068016841F448
:106A700000510160012084F85D00002084F85C0072
:106A80000320BDE8F8830025401E0090206881683F
:106A900038EA010004D000214945BDD10020F0E7CB
:106AA0000121F9E70C07002038B50748074C012100
:106AB000006800902046FBF775FA012269462046DF
:106AC000FBF7F2FA38BD0000F406001000EC0108F4
:106AD00000B595B028210AA8F9F793FC14220C49B7
:106AE0006846F9F767FC0A491422143105A8F9F73A
:106AF00061FC0AAB282269460648FBF7FDFA08B19B
:106B000005A000E00CA002F095F915B000BD000052
:106B1000C406001000DC01084661696C65642074DD
:106B20006F2073617665207769666920746F2066CF
:106B30006C6173680A0000005769466920636F6ED4
:106B400066696720736176656420746F20666C6186
:106B50007368207375636365737366756C6C790A0B
:106B600000000000F0B589B0DDE90E45DDE91067F1
:106B70008DF80000DDE912CE8DF801108DF808C007
:106B800000208DF802208DF804408DF809E08DF882
:106B900005508DF80A008DF803308DF806608DF8E9
:106BA0000B0003908DF8077004AB1022694605486E
:106BB000FBF7A2FA002802D003A002F03BF909B0CB
:106BC000F0BD000000FC01084661696C656420743A
:106BD0006F207361766520506172616D65746572B6
:106BE00020746F20666C6173680A000038B506482F
:106BF000064C009001212046FBF7D4F9012269469A
:106C00002046FBF751FA38BD0115052500E40108BF
:106C1000064808B5C06C009001210548FBF7C2F991
:106C2000012269460348FBF73FFA08BD140600102D
:106C300000E4010800D401087CB5154C0D465A212A
:106C40002170A52161700021A1708221E170010AEB
:106C50002171607110EE100AF9F74CFDCDE90001C9
:106C6000A01D2A460BA102F009F9801DC0B2FF2128
:106C70002154401CC0B22154401CC2B2D01EA0708E
:106C800002B02146BDE870400648FEF79FBD0000F7
:106C9000340A0020434F3A20253032642320253324
:106CA0002E326600F83A002010B5114C5A2222709C
:106CB000A52262700022A2708222E270020A227172
:106CC00060710A46A01D0BA102F0D8F8801DC0B269
:106CD000FF212154401CC0B22154401CC2B2D01E1E
:106CE000A0702146BDE810400348FEF76FBD0000CC
:106CF000340A002025346400F83A00207FB5164C91
:106D00000B465A212170A52161700021A1708221BA
:106D1000E170010A21716071022606250822694688
:106D20001846FAF7D1FC002069460A5C62556D1CD2
:106D3000401CEDB21028F8DBFF2161556D1CE8B254
:106D40002154401CC2B2901B401EA055214603484E
:106D5000FEF73CFD7FBD0000340A0020F83A002019
:106D60007CB5154C0D465A212170A521617000217A
:106D7000A1708221E170010A2171607110EE100A88
:106D8000F9F7B8FCCDE90001A01D2A460BA102F0DD
:106D900075F8801DC0B2FF212154401CC0B221549F
:106DA000401CC2B2D01EA07002B02146BDE87040A7
:106DB0000648FEF70BBD0000340A002048323A2096
:106DC00025303264232025332E326600F83A002025
:106DD0000A4609495A230B70A5234B708223CB70B6
:106DE000030A0B714871100A88710523CA710822C1
:106DF0008B700248FEF7EABC340A0020F83A002003
:106E00007CB5134C5A26069D2670A5266670002672
:106E1000A6708226E670060A26716071CDE90035FB
:106E200013460A46A01D0BA102F028F8801DC0B22F
:106E3000FF212154401CC0B22154401CC2B2D01EBC
:106E4000A07002B02146BDE870400848FEF7BEBC05
:106E5000340A00202530326423202533642020208A
:106E6000253364202020253364000000F83A0020F8
:106E700010B5114C5A232370A52363700023A3700F
:106E80008223E370030A2371134660710A46A01D32
:106E90000AA101F0F3FF801DC0B2FF212154401C64
:106EA000C0B22154401CC2B2D01EA0702146BDE821
:106EB00010400648FEF78ABC340A002050723A207F
:106EC000253032642320253464000000F83A002085
:106ED00010B5114C5A222270A52262700022A270B5
:106EE0008222E270020A227160710A46A01D0BA183
:106EF00001F0C4FF801DC0B2FF212154401CC0B26C
:106F00002154401CC2B2D01EA0702146BDE81040E2
:106F10000348FEF75BBC0000340A00202573000024
:106F2000F83A00202DE9FE43002100914FF48070D3
:106F3000ADF800003B480291DFF8EC80D0F80E205D
:106F40000192408AADF8080036487E244FF00109CE
:106F5000808842BAADF80A20324A401C90808DF8F1
:106F6000021005228DF8032088F800404046009B5F
:106F700040F8013F019B4360029B8360A8F105003C
:106F80002A4B01701B784370812383700323C370E5
:106F900001711230A0F11201F9F70CFA122511213A
:106FA00008F10100FAF7EEFA88F81200294608F114
:106FB000010004F0F1FD401C80B21DA108F8004062
:106FC000401C86B2324608F5E17001F057FF85B2E9
:106FD000002408F5E17709E018F80420781919A1D0
:106FE00001F04CFF2844641C85B2A4B2B442F3D330
:106FF000781916A216A101F041FF164916A001F05A
:1070000019FF062316A21CA11248CDF8009006F025
:1070100041FD10B1002000F041B818A001F00AFFB6
:107020000120F8E7BA060020050000200E06001037
:1070300041542B4D495053454E443D302C25642C32
:10704000220000002530325800000000220D0A0006
:1070500025730000C701002025730D0A0000000001
:107060002B4D49505552433A202272746370222CA2
:10707000302C3230000000004F4B000053656E642E
:107080005F47656E6572616C5F726573706F6E737A
:10709000655F6661696C0D0A0000000006BCBDE812
:1070A000F88300002DE9FE430022324900924FF49C
:1070B00000700292ADF80000D1F80E000190488AED
:1070C000ADF808004888DFF8B08043BAADF80A3060
:1070D000401C48808DF803207E2488F800404046FC
:1070E000009940F8011F01994160029981604FF0B9
:1070F00001090D250C2108F10100FAF743FA88F87F
:107100000D00294608F1010004F046FD401C80B244
:107110001AA108F80040401C86B2324608F5E1701A
:1071200001F0ACFE85B2002408F5E1770AE000BF6B
:1071300018F80420781916A101F0A0FE2844641C58
:1071400085B2A4B2B442F3D3781913A213A101F00B
:1071500095FE062312A218A11848CDF8009006F05B
:1071600099FC10B1002000F037B815A001F062FEC4
:107170000120F8E7BA0600200500002041542B4DFD
:10718000495053454E443D302C25642C22000000CC
:107190002530325800000000220D0A00257300003F
:1071A0002B4D49505552433A202272746370222C61
:1071B000302C3230000000004F4B0000C70100208F
:1071C0004D495053454E445F48656172745F666136
:1071D000696C0D0A0000000006BCBDE8F8830000E1
:1071E0002DE9FE43754900244FF0F0080C2281F888
:1071F00000804A7025460226224623468B55761C7F
:10720000F6B2571C8F55761CF6B201EB060C00EB5C
:107210004202B61CB2F86821ACF80020FAB2F6B20D
:10722000032AEBD301F80680761CF2B208268E54AE
:10723000521CD7B20022CB557F1CFFB2561CCE5534
:107240007F1CFFB201EB070C00EB82023F1DD2F85E
:107250006E21CCF80020F2B2FFB2032AEBD301F882
:1072600007807F1CFAB206268E54521CD6B200222A
:107270008B55761CF6B2571C8F55761CF6B201EB77
:10728000060C00EB8202361DD2F87A21CCF80020E1
:10729000FAB2F6B2032AEBD301F80680761CF0B2FC
:1072A00005220A54464A401CC0B212780A54454A84
:1072B000401CC0B212780A54401CC2B24248444F2B
:1072C0004FF07E080068060E8E54521CD2B2060C97
:1072D0008E54521CD2B2060A8E54521CD2B288541A
:1072E0003A49009342F202600293ADF80000D1F8EF
:1072F0000E000190488AADF80800521C8889D6B269
:1073000042BAADF80A20401C88818DF8036007F866
:107310000480641C38190099016001994160029948
:1073200081600C34381932462449F9F743F8344463
:10733000601E81B2781CFAF725F93855A1B2781C85
:1073400004F02AFC401C80B2402207F80080401C58
:1073500086B207F10D011F48F9F72CF832461EA13D
:1073600007F5E17001F08AFD284485B2002407F595
:10737000E17809E03A5D08EB05001CA101F07EFD13
:107380002844641C85B2A4B2B442F3D308EB0500D0
:1073900018A219A101F072FD02200090062317A285
:1073A0001AA11B4806F076FB10B1002000F044B88B
:1073B00018A001F03FFD0120F8E700007B05002048
:1073C000330600103406001040060010BA060020F4
:1073D00005000020A10B001041542B4D495053458E
:1073E0004E443D302C25642C2200000025303258BC
:1073F00000000000220D0A00257300002B4D4950AB
:1074000053454E443A20302C373300004F4B000098
:10741000C70100204D495053454E445F507265737B
:10742000737572655F434F5F48325F446174615F9B
:107430006661696C0D0A000006BCBDE8F8830000B7
:107440002DE9F0438FB00025424C00954FF0010923
:107450000295ADF80090D4F80E000190608AADF866
:107460000800208841BAADF80A10401C20802E2068
:107470008DF80300302103A8F8F7C3FF6069CDF849
:107480002900208BADF82D00A07E8DF82F008DF8FF
:107490003050D4F81B00CDF83100D4F81F00CDF8DF
:1074A000350094F82300DFF8B0808DF839007E2491
:1074B00088F800404046009940F8011F019941605A
:1074C0000299816008F10D002E2203A9F8F772FFDE
:1074D0003B253A2108F10100FAF754F888F83B00FF
:1074E000294608F1010004F057FB401C80B21BA1A3
:1074F00008F80040401C86B2324608F5E17001F001
:10750000BDFC85B2002408F5E17709E018F80420F5
:10751000781917A101F0B2FC2844641C85B2A4B20A
:10752000B442F3D3781914A214A101F0A7FC0623E6
:1075300013A219A11948CDF8009006F0ABFA18B1C2
:1075400000200FB0BDE8F08315A001F073FC01200E
:10755000F7E70000BA0600200500002041542B4D3B
:10756000495053454E443D302C25642C22000000E8
:107570002530325800000000220D0A00257300005B
:107580002B4D49505552433A202272746370222C7D
:10759000302C3236000000004F4B0000C7010020A5
:1075A00053656E645F436C6F75645F5265676973A2
:1075B0007465725F6661696C0D0A0000F8B50120A0
:1075C0000346009014A214A114A006F063FA164812
:1075D00005F084F8154C0228E06202D000F090FB20
:1075E00002E0FAF7D7FDE0620025A573104800F02D
:1075F00023F80F2608B1A57626700D48FFF7F0FD99
:1076000008B1A57626704FF400710A4804F076FBA5
:10761000BDE8F840FFF748BA4F4B000041542B43F8
:10762000434C4B3F0D0A00001E01001014060010D1
:107630009C070010E80900102DE9FE435149F02293
:1076400000270A700A224A703E4602253A463B4607
:107650004B55541C6D1C02EB42024C556D1C00EB4B
:10766000820201EB050CD2F80080CCF80080D2F841
:107670000480CCF804809268CCF80820E2B20C3583
:107680001E2AE5D34048424C4FF07E080068020EA7
:107690004A556D1C020C4A556D1C020A4A556D1C58
:1076A00048553A49009342F202600293ADF8000057
:1076B000D1F80E000190488AADF8080048896D1C89
:1076C00042BAADF80A20401C4881280A8DF8020011
:1076D0008DF8035004F807807F1CE01900990160C1
:1076E00001994160029981600C37E0192A462549C9
:1076F000F8F760FE781985B2681E81B2601CF9F750
:1077000041FF6055A9B2601C04F046FA401C80B2EB
:1077100040F2B91204F80080401C87B221461D488F
:10772000F8F748FE3A461CA104F5E17001F0A6FB0B
:10773000304486B2002504F5E17809E0625D08EB8B
:1077400006001AA101F09AFB30446D1C86B2ADB25E
:10775000BD42F3D308EB060016A217A101F08EFB81
:1077600002200090062315A218A1194806F092F9EC
:1077700010B1002000F03EB816A001F05BFB012024
:10778000F8E70000D303002040060010BA060020EE
:1077900005000020E809001041542B4D4950534585
:1077A0004E443D302C25642C2200000025303258F8
:1077B00000000000220D0A00257300002B4D4950E7
:1077C00053454E443A20302C343431004F4B0000A6
:1077D000C70100204D495053454E445F54656D70BC
:1077E000657261747572655F446174615F66616939
:1077F0006C0D0A0006BCBDE8F88300002DE9F041DD
:10780000ADF5627D80464FF461716846F8F7F9FD89
:107810004046F8F729FE84B21748E31C17A1026816
:10782000684601F02BFB064687B26D460DEB07005C
:1078300022464146F8F7BEFD381980B27C21295412
:10784000401C80B20D212954401C80B20A212954C9
:10785000401C82B269460F48FDF7B8FF6A463146C0
:107860000DA001F0E7FA424621460DA001F0E2FA30
:107870000DF5627DBDE8F0815C06001041542B439C
:10788000495053454E443D25642C25642C302C3002
:107890002C0000007C3B0020252E2A7300000000F5
:1078A000252E2A730D0A00002DE9F041ADF5007D6B
:1078B0000D4680464FF400716846F8F7A2FD1A485D
:1078C0002B461AA10268684601F0D8FA044687B22E
:1078D0006E460DEB07002A464146F8F76BFD781916
:1078E00080B20D213154401C80B20A213154401C19
:1078F00082B269461348FDF769FF6A46214612A025
:1079000001F098FA002406E018F8041010A001F025
:1079100091FA641CA4B2AC42F6D30FA001F08AFA2B
:107920000DF5007DBDE8F0815C06001041542B434D
:10793000495053454E443D25642C25642C302C3051
:107940002C0000007C3B0020252E2A730000000044
:1079500025303258000000000D0A00002DE9FE43DA
:1079600000224149009209200292ADF80000D1F8AE
:107970000E000190488AADF80800C888DFF8EC8056
:1079800043BAADF80A30401CC8808DF802200A20A6
:107990008DF803007E2488F800404046009940F8A6
:1079A000011F0199416002998160314940464FF0C1
:1079B00001090A6840F80D2F898881802D48172514
:1079C0000068010E88F81310010C88F81410010AE1
:1079D00088F8151088F81600162108F10100F9F74B
:1079E000D1FD88F81700294608F1010004F0D4F809
:1079F000401C80B220A108F80040401C86B23246EC
:107A000008F5E17001F03AFA85B2002408F5E17753
:107A10000AE000BF18F8042078191CA101F02EFA22
:107A20002844641C85B2A4B2B442F3D3781919A2D5
:107A300019A101F023FA194919A001F0FBF9062355
:107A400019A21FA11548CDF8009006F023F828B11F
:107A50001CA001F0EFF9002000F04CB81FA001F0CD
:107A6000E9F90120F8E70000BA060020050000202F
:107A7000AC0600104006001041542B4D49505345B0
:107A80004E443D302C25642C220000002530325815
:107A900000000000220D0A0025730000C70100202D
:107AA00025730D0A000000002B4D49505552433AF2
:107AB000202272746370222C302C323000000000BF
:107AC0004F4B000053656E645F73656E736F726C2D
:107AD000696E655F4F4B0D0A0000000053656E64D0
:107AE0005F73656E736F726C696E655F6661696CFA
:107AF0000D0A000006BCBDE8F88300002DE9FE4336
:107B000000224349009240F203100292ADF80000B7
:107B1000D1F80E000190488AADF8080008893D4C64
:107B200043BAADF80A30401C08818DF802200C22BF
:107B30008DF803207E2525702146009B41F8013FEA
:107B4000019B4B60029B8B60012004F2C231F02349
:107B500008704B70887030480078304BC8701888B7
:107B6000060A0E714871987888711879C8712C4886
:107B70000068030E0B72030C4B72030A8B72C872FF
:107B8000A1F2B530F8F716FC19261821601CF9F798
:107B9000F9FC60763146601C03F0FEFF401C80B2A9
:107BA00020A12554401C87B23A4604F5E17001F04B
:107BB00065F986B2002504F5E17809E0625D08EB1D
:107BC00006001DA101F05AF930446D1C86B2ADB219
:107BD000BD42F3D308EB060019A21AA101F04EF939
:107BE00019491AA001F026F902200090062319A2D3
:107BF0001EA1154805F04EFF28B11DA001F01AF98D
:107C0000002000F053B822A001F014F90120F8E799
:107C1000BA060020050000202C060010B206001055
:107C20004006001041542B4D495053454E443D30C1
:107C30002C25642C22000000253032580000000062
:107C4000220D0A0025730000C701002025730D0ACC
:107C5000000000002B4D49505552433A20227274C7
:107C60006370222C302C3233000000004F4B000098
:107C70004D495053454E445F73797374656D6C651F
:107C800076656C5F6368616E67655F4F4B0D0A00D8
:107C90004D495053454E445F73797374656D6C65FF
:107CA00076656C5F6661696C0D0A000006BCBDE814
:107CB000F8830000F0B40D460F4914465A220A70AA
:107CC000A5224A7000228A708222CA70020A0A71B2
:107CD000022348710622002005E02E5C8E54521CBF
:107CE000401CD2B2C0B2A042F7D3D01A401EC85432
:107CF000F0BC0248FDF76ABD340A0020F83A0020C3
:107D000030B589B00546142102A8F8F77AFB0024A3
:107D100069462846079403F0D1FE9DF805008DF8CA
:107D200008009DF806008DF809009DF807008DF801
:107D30000A000594BDF800000694A0F5FA608DF8DD
:107D40001F009DF802008DF81D009DF803008DF8BE
:107D50001E0001208DF81C00002202A90848FCF733
:107D6000C1FD08B1FAF776F8002207A90448FCF72C
:107D700069FD002801D0FAF76DF809B030BD0000A8
:107D8000A431001010B54FF0E020006907F01CF896
:107D9000012803D0BDE8104006F06ABC10BD000009
:107DA00000B597B044216846F8F72BFB142111A8C1
:107DB000F8F727FB4FF40070FBF71CFE08B172B612
:107DC000FEE7FBF77DFE194850F8901F21F01801DF
:107DD00001600E20012100900802CDE90210102060
:107DE000CDE9040102200A90CDE90B0108210D9193
:107DF0000721CDE90E1010906846FCF723F908B171
:107E000072B6FEE70F20119003201290902013907D
:107E1000002014900146159011A8FBF7DBFF002805
:107E200001D072B6FEE717B000BD0000001002409E
:107E30000248016841F470010160704788ED00E07C
:107E400000251C4C4FF4C8770126207E01282CD138
:107E50006D1CC102ADB21848FBF7BBFC012800D075
:107E60000020A07230B1002003F0CCFDE67513A015
:107E700000F0E0FF10211748FBF7ABFC78B10020C1
:107E8000E07270B1012003F0C5FD13A000F0D2FF35
:107E9000BD420AD3A67315A000F0CCFF04E0012078
:107EA000EEE7BD4201D3A6730025642004F0D9F8A3
:107EB000CBE70000140600100008004861637475E9
:107EC00061746F725F706F7765725F636C6F7365FB
:107ED000640A0000000400486761735F706F776593
:107EE000725F6F70656E65640A0000006761735FA2
:107EF00073746172745F726561640A000148FCF713
:107F0000AEBF0000C831001070B50268164B4FF0CC
:107F10008046984201D0B04203D122F070044A68F2
:107F20002243124C124D984205D0B04203D0A042D9
:107F300001D0A84203D122F44076CA6832434E6988
:107F400022F08002324302608A68C2620A6882625A
:107F5000984203D0A04201D0A84201D1096901632F
:107F60000121416170BD0000002C01400040014032
:107F70000044014090F82410C90706D001684A68FF
:107F8000836A22F400321A434A6090F82410890769
:107F900006D501684A68C36A22F480321A434A60EF
:107FA00090F82410490706D501684A68036B22F44B
:107FB00080221A434A6090F82410090706D5016808
:107FC0004A68436B22F400421A434A6090F8241036
:107FD000C90606D501688A68836B22F480521A4369
:107FE0008A6090F82410890606D501688A68C36BF8
:107FF00022F400521A438A6090F82410490611D5E1
:1080000001684A68036C22F480121A434A60016CCA
:10801000B1F5801F06D101684A68436C22F4C002A2
:108020001A434A6090F82410090606D501684A6888
:10803000806C22F4002202434A607047F8B50026A3
:108040000446C0F88060FBF7D7FB0546206800684F
:108050006FF07E47000708D52B4600224FF4001131
:108060002046009700F040FA60B920680068400799
:108070000AD52B4600224FF480012046009700F0DD
:1080800033FA08B10320F8BD2020A067E067266618
:1080900084F874600020F8BD10B5806A0021A0F853
:1080A0005A10A0F85210FCF7F3FF10BD70B5846AA7
:1080B000A06FE56F216889684FF00006090606D5B4
:1080C000212804D1A4F85260204600F0AEF82068C0
:1080D0008068400606D5222D04D1A4F85A602046B7
:1080E00000F07EF8D4F8800040F01000C4F8800062
:1080F0002046FCF7CDFF70BD10B50146806A0968C7
:10810000096889062DD40021A0F85A10016851E8A9
:10811000002F22F4807241E80023002BF6D1016881
:10812000083151E8002F22F0010241E80023002B22
:10813000F5D10168083151E8002F22F0400241E8F2
:108140000023002BF5D12021C167016E012908D140
:10815000026852E8001F21F0100142E80013002BD2
:10816000F6D1016E012902D0FDF79CFA10BDB0F8DE
:108170005810FCF744FF10BD10B5806A016E01294C
:1081800002D0FDF7C5FA10BDB0F858104908FCF749
:1081900036FF10BD10B50146806A09680968890676
:1081A00016D40021A0F852100168083151E8002FC0
:1081B00022F0800241E80023002BF5D1026852E84A
:1081C000001F41F0400142E80013002BF6D110BD22
:1081D000FDF74CFB10BD10B5806AFDF748FB10BDE4
:1081E000016851E8002F22F4907241E80023002B2F
:1081F000F6D10168083151E8002F22F0010241E870
:108200000023002BF5D1016E012908D1026852E844
:10821000001F21F0100142E80013002BF6D12021AD
:10822000C1670021016641667047026852E8001F7D
:1082300021F0C00142E80013002BF6D12021816714
:10824000704700002DE9F04104460168806822690A
:10825000E3691043626900251A431043714F0A68AD
:10826000714B1A4002430A6020684168E26821F4B9
:108270004051114341602168A069B94201D0226A8E
:1082800010438A6822F4306202438A606749236897
:1082900067488B420DD1D0F8880010F0030006D05B
:1082A000012847D0022843D0032830D144E00121DF
:1082B0002EE060498B420BD1D0F8880010F00C0002
:1082C00034D0042836D0082832D00C281FD133E00F
:1082D00059498B420BD1D0F8880010F0300025D0DE
:1082E000102827D0202823D0302810D124E0BB42EA
:1082F0000DD1D0F8880010F4406017D0B0F5806F31
:1083000018D0B0F5006F13D0B0F5406F14D0102125
:108310004A4A00264FF40040BB422FD171B10229D6
:108320000FD004290FD0082973D10FE00021EFE707
:108330000221EDE70421EBE70821E9E7FBF70CFE5A
:1083400003E0104602E0FBF72BFEE8B3626802EBA5
:10835000420181425DD8B0EB023F5AD8010E0302C0
:108360005008181871410023F7F79CFF344AA0F514
:10837000407191424DD82168C8604BE0E3694FF6E7
:10838000EF77834228D1092943D2DFE801F00508BD
:108390000B420D4242421000FBF7DEFD06E0FBF708
:1083A000EDFD03E0104602E0FBF7FAFD60B141008D
:1083B000606801EB5001B1FBF0F0A0F11001B9428F
:1083C00027D84FF6F07100E024E00140C0F34200EE
:1083D00001432068C1601DE009291AD2DFE801F0DD
:1083E00005080B190D1919191000FBF7B5FD06E06A
:1083F000FBF7C4FD03E0104602E0FBF7D1FD48B1F6
:10840000616800EB5100B0FBF1F0A0F11001B9423E
:1084100005D9012566662846A666BDE8F08180B2CA
:10842000A9E7000000800040F369FFEF0038014039
:108430000010024000440040004800400024F400C6
:10844000FFFC0F0070B54165A0F8582000250446D8
:10845000C0F880502220E067206FD8B11F49C16268
:10846000216F1F4813460863216F1E484863206F21
:108470008563666D216832462431206FFAF782FFEA
:1084800040B11020C4F8800004F8745F2020A06080
:10849000012070BD84F87450206940B1216851E812
:1084A000000F40F4807041E80002002AF6D12068F5
:1084B000083050E8001F41F0010140E80012002A96
:1084C000F5D12068083050E8001F41F0400140E835
:1084D0000012002AF5D1002070BD0000F9800008CC
:1084E00079810008AD8000082DE9F0479A461746CB
:1084F0000E4604464FF000094FF02008089D4AE060
:10850000681C48D0FBF778F9A0EB0A00A8422AD8EB
:108510004DB32068016849073DD5C069C0430005D7
:1085200039D421684FF400600862206850E8001FC9
:1085300021F4D07140E80012002AF6D120680830FA
:1085400050E8001F21F0010140E80012002AF5D197
:10855000C4F87880C4F87C80C4F8808084F8749073
:108560000320BDE8F087216851E8000F20F4D070A7
:1085700041E80002002AF6D12068083050E8001FC8
:1085800021F0010140E80012002AF5D1C4F87880FA
:10859000C4F87C80E2E72068C06936EA000004D0B5
:1085A0000020B842ACD00020DBE70120F9E7000052
:1085B00010B5104C2068C169C943C90614D41021F4
:1085C00001622046FCF71DFD206F006840680A4AE2
:1085D000C0F11E0000211154104604F00BF91E22B8
:1085E00005492046FDF734F8BDE810400148FCF786
:1085F00061BD0000743A002000000010114810B561
:108600000068C169C943C90616D4102101620D482A
:10861000FCF7F7FC0C48006840680C494042C0B2C7
:108620000870072802D90748FDF73CF84FF480721C
:1086300007490448FDF70CF8BDE810400148FCF775
:1086400039BD0000F83A0020903C0020EC060010F4
:108650001E00001010B505F0F9FBBDE81040014800
:10866000FCF728BD7C3B002070B505460C4608464B
:10867000F7F7FAFE82B221462846BDE87040FDF7C2
:10868000A5B8000070B58AB028216846F7F7B9FE92
:10869000284800226946806806F016FA012819D198
:1086A00025A000F0C7FB00246E46264D04E0315D96
:1086B00025A000F0BFFB641C28788442F7DB24A0CF
:1086C00000F0B8FB684603F0E1FB0028684603D0E1
:1086D00004F0B0F90AB070BD03F000FC0028684651
:1086E00002D004F0E1F9F5E703F0BCFB002868468E
:1086F00002D004F073F9EDE703F02CFC0028684683
:1087000002D004F03DFBE5E703F010FC00286846CA
:1087100002D004F0CFFADDE703F030FC0028684611
:1087200002D004F0EFFBD5E703F0ECFB0028D1D03A
:1087300000F0C8FB94060010727842756666657298
:108740003A200000EC0600102530325820000000CE
:108750000A000000FEE70000F0B5B3B006460022B4
:1087600000924FF40070ADF8000020480292214CB6
:10877000016801911E498088ADF8080008887E25AF
:1087800043BAADF80A30401C08808DF803202570EC
:108790002046009940F8011F0199416002998160CB
:1087A0000D270C21601CF8F7EDFE60733946601C44
:1087B00003F0F2F9401C80B22554401C84B26EB123
:1087C000C8216846F7F71DFE6A462146094800F0B1
:1087D000FFFF6846FFF712F833B0F0BD33B0214613
:1087E000BDE8F0400348FFF75FB80000C80600206E
:1087F000BC060020050000202DE9F04180466648B7
:10880000F025B2B000240C220570427002262246E8
:1088100023468355761CF6B2571C8755761CF6B254
:1088200000EB060C01EB4202B61CB2F86821ACF872
:108830000020FAB2F6B2032AEBD38555761CF2B2C9
:1088400008268654521CD7B20022C3557F1CFFB2A3
:10885000561CC6557F1CFFB200EB070C01EB8202D1
:108860003F1DD2F86E21CCF80020F2B2FFB2032AED
:10887000EBD3C5557F1CFAB206268654521CD6B2DD
:1088800000228355761CF6B2571C8755761CF6B22B
:1088900000EB060C01EB8202361DD2F87A21CCF8EF
:1088A0000020FAB2F6B2032AEBD38555761CF1B25A
:1088B00005224254394A491CC9B212784254384AF6
:1088C000491CC9B212784254491CCAB235497E27A4
:1088D00009680D0E8554521CD2B20D0C8554521CE1
:1088E000D2B20D0A8554521CD2B2314D815400933C
:1088F00042F20260ADF800002B480293521C01685E
:1089000001912A498088ADF808000888D6B242BA99
:10891000ADF80A20401C08808DF803602F55641CB8
:1089200028190099016001994160029981600C3415
:10893000281932461849F7F73DFD3444601E81B2CC
:10894000681CF8F71FFE2855A1B2681C03F024F933
:10895000401C80B240222F54401C84B205F10D010E
:108960001448F7F727FDB8F1000F0ED0C82168466C
:10897000F7F747FD6A462146284600F029FF68467A
:10898000FEF73CFF32B0BDE8F08132B02146BDE8D1
:10899000F0410748FEF788BF7B0500203306001032
:1089A0003406001040060010C8060020C60600204D
:1089B00005000020A10B0010F0B5BFB00646002452
:1089C0000C940120ADF830002F480E9401680D91F1
:1089D0002E498088ADF83800088842BAADF83A20B0
:1089E000401C08802E208DF8330030216846F7F7B0
:1089F00008FD27487E252E220168CDF81D108188AC
:108A0000ADF8211080798DF8230022488DF824409C
:108A1000214C0168CDF825104168CDF82910007A65
:108A20008DF82D00257020460C9940F8011F0D99F6
:108A300041600E99816004F10D006946F7F7BAFCB8
:108A40003B273A21601CF8F79DFD84F83B0039462E
:108A5000601C03F0A1F8401C80B22554401C84B275
:108A60006EB1C8210CA8F7F7CCFC0CAA21460A4825
:108A700000F0AEFE0CA8FEF7C1FE3FB0F0BD2146EF
:108A80000548FEF711FFF8E7C8060020BA060020E7
:108A9000CE060020D5060020050000202DE9F0417B
:108AA000464A8046ADF5627DF020107000250A2010
:108AB0005070022428462B461355461C641C00EBBC
:108AC00040001655641C01EB80001719D0F800C057
:108AD000C7F800C0D0F804C0C7F804C08068B86008
:108AE000F0B20C341E28E7D33548384E7E27006894
:108AF000010E1155641C010C1155641C010A11551D
:108B0000641C1055009342F20260ADF800002D483D
:108B100002932D4A016801918088ADF80800108801
:108B2000641C41BAADF80A10401C1080200A8DF870
:108B300002008DF8034077556D1C70190099016093
:108B400001994160029981600C35701922461B49D8
:108B5000F7F730FC281984B2601E81B2701CF8F758
:108B600011FD3055A1B2701C03F016F8401C80B204
:108B700040F2B9123754401C84B231461448F7F71A
:108B800019FCB8F1000F10D04FF461716846F7F787
:108B900038FC6A462146304600F01AFE6846FEF769
:108BA0002DFE0DF5627DBDE8F0810DF5627D21465B
:108BB000BDE8F0410548FEF777BE0000D303002072
:108BC00040060010C8060020C40600200500002052
:108BD000E8090010F0B5B3B0064600210091092065
:108BE000ADF80000294802912A4C02680192284AF7
:108BF0008088ADF8080010887E2543BAADF80A30A9
:108C0000401C10808DF802100A208DF8030025709A
:108C10002046009940F8011F019941600299816046
:108C20001D49204617270A6840F80D2F8988818042
:108C30001A480068010EE174010C2175010A617582
:108C4000A0751621601CF8F79DFCE0753946601C84
:108C500002F0A2FF401C80B22554401C84B26EB1C9
:108C6000C8216846F7F7CDFB6A462146094800F05F
:108C7000AFFD6846FEF7C2FD33B0F0BD33B021460C
:108C8000BDE8F0400348FEF70FBE0000C806002014
:108C9000C006002005000020AC06001040060010B1
:108CA000F0B5B3B006460021009140F20310ADF8D4
:108CB000000031480291324C026801922F4A8088AC
:108CC000ADF8080010887E2543BAADF80A30401C84
:108CD00010808DF802100C228DF80320257021469B
:108CE000009B41F8013F019B4B60029B8B60254933
:108CF0000120F02308704B70887023480078C870FA
:108D0000224803881F0A0F714B7183788B71007999
:108D1000C8711F480068030E0B72030C4B72030AE4
:108D20008B72C87204F10D00F7F744FB1927182164
:108D3000601CF8F727FC60763946601C02F02CFFB7
:108D4000401C80B22554401C84B26EB1C8216846D4
:108D5000F7F757FB6A462146094800F039FD684697
:108D6000FEF74CFD33B0F0BD33B02146BDE8F04016
:108D70000348FEF799BD0000C8060020C206002087
:108D800005000020C70300202C060010B2060010CA
:108D900040060010F0B5B3B00646002200924FF432
:108DA0007F40ADF8000020480292214C01680191FB
:108DB0001E498088ADF8080008887E2543BAADF8C2
:108DC0000A30401C08808DF8032025702046009949
:108DD00040F8011F01994160029981600D270C2123
:108DE000601CF8F7CFFB60733946601C02F0D4FEBC
:108DF000401C80B22554401C84B26EB1C821684624
:108E0000F7F7FFFA6A462146094800F0E1FC684698
:108E1000FEF7F4FC33B0F0BD33B02146BDE8F040BE
:108E20000348FEF741BD0000C8060020BC06002034
:108E3000050000200FB4054B10B503A9044A0298A1
:108E400000F01CF910BC5DF814FB000089BD00089F
:108E5000300700200FB41CB50A46521ECDE90002AF
:108E600007A9054B6A46069800F008F9009A002108
:108E700011701CBC5DF814FBB19700080FB4084BCF
:108E800010B504A902AA039800F0F8F8044602A954
:108E9000002000F098FC204610BC5DF814FB000098
:108EA000C79700080907090E002804DB00F1E0203D
:108EB00080F80014704700F00F0000F1E02080F807
:108EC000141D7047BFF34F8F05480168054A01F430
:108ED000E06111430160BFF34F8F00BFFDE7000069
:108EE0000CED00E00400FA05004870476007001030
:108EF00002E008C8121F08C1002AFAD17047704763
:108F0000002001E001C1121F002AFBD170470000C0
:108F10002DE9FF5FDDE90220010DDDF838B00243E5
:108F200018D044F61050A1F2FF3141430D140F98B0
:108F3000012820D0A5EB0B00401C5FEA000A4FF08F
:108F40000004474EDFF81C91A046504616D5CAF1E2
:108F5000000728E00F98012443A2012808D000212F
:108F600000980F9BC0E90021C0E9024300F082B8DD
:108F70006FEA0B01F4E7CBF10000DEE7074612E0F1
:108F8000F80707D02246334640464946F7F791FD99
:108F9000804689462246334610461946F7F789FD32
:108FA00004460E467F10002FEAD1DDE90201BAF136
:108FB000000F42464B4602DAF7F77BFD01E0F7F778
:108FC000EDFD04460E460022284BF7F76FFE03D84E
:108FD0004FF0FF30014607E00022254B2046314686
:108FE000F7F7B8FCF7F749FE102409E0002C0ADB7C
:108FF0000A220023F7F756F9019B30321A55641EF6
:1090000050EA0102F2D1641C019AC4F11103144424
:109010000F9A012A03D0012208430DD10AE0084328
:1090200004D000204FF0110B0F9080E7A3EB0B054D
:109030006D1E0DE05B4504DD4FF0000205F10105FA
:1090400004E003DA4FF00002A5F10105002AECD09C
:1090500000980F99C0E90231C0E9004586E7000099
:10906000000024400000F03F300000000000F0430A
:109070000000E03F3FBCBDE8C09F00002DE9FF4F6E
:1090800095B09B468946064600250FE2252877D1F4
:1090900000242746F84A0121059400E0044316F80D
:1090A000013F203B01FA03F01042F7D130782A2823
:1090B00011D06FF02F033078A0F13002092A16D8B2
:1090C000059A44F0020402EB820203EB42021044D0
:1090D000761C0590EFE759F8042B0592002A03DA75
:1090E000504244F40054059044F00204761C307859
:1090F0002E2816D116F8010F44F004042A280DD0AA
:109100006FF02F023078A0F13003092B09D807EB5C
:10911000870302EB4303C718761CF3E759F8047B77
:10912000761C30786C280FD006DC4C2817D06828C5
:109130000DD06A2814D104E0742810D07A280FD1F9
:109140000DE044F400140AE044F4801401E044F417
:1091500040147278824202D104F58014761C761C89
:10916000307866280BD013DC582877D009DC00282B
:1091700075D04528F6D04628F4D047281AD19DE16D
:1091800018E0632835D0642879D0652812D195E19C
:10919000702873D008DC6728F1D069286FD06E285A
:1091A0000DD06F2806D1B5E073282CD0752875D066
:1091B000782874D05A46179990476D1C75E1C4F30E
:1091C0000250022809D003280DD0D9F80010042835
:1091D0000DD00D6009F1040967E1D9F80010EA1714
:1091E000C1E90052F6E7D9F800100D80F2E70D70E2
:1091F000F0E719F8041B8DF8001000208DF801002D
:10920000EA46012003E059F804AB4FF0FF30610754
:109210004FF0000102D40DE008F101018846B94287
:109220000FDA8045F8DB1AF808100029F4D108E0BD
:1092300008F1010188468142FADB1AF8081000297A
:10924000F6D105985B46A0EB080721463846179AE9
:1092500000F097FA284400EB080507E04DE029E10B
:109260000DE01AF8010B5A4617999047B8F101081A
:10927000F7D25B4621463846179A13E142E00A22AC
:109280000092C4F302524FF0000A022A08D059F8A3
:1092900004CB032A4FEAEC710AD00DE029E02AE062
:1092A00009F1070121F00702F2E802C1914609E045
:1092B0000FFA8CFC4FEAEC71042A03D14FFA8CFCB4
:1092C0004FEAEC71002907DA0A460021DCF1000CB4
:1092D00061EB02012D2202E0220504D52B228DF83C
:1092E0000420012203E0E20701D02022F7E79046A4
:1092F00059E00A2102E010220DE010214FF0000A8F
:1093000000910BE010224FF0000A44F004040827FB
:10931000009203E008224FF0000A0092C4F30252C8
:10932000022A05D059F804CB0021032A08D009E00D
:1093300009F1070121F00702F2E802C1914605E0B8
:109340001FFA8CFC042A01D10CF0FF0C4FF000082E
:10935000220728D5702806D0009B83F0100353EA1B
:109360000A0305D00EE040228DF80420012208E017
:109370005CEA010206D030228DF804208DF8050049
:1093800002229046009B83F0080353EA0A030AD1A5
:109390005CEA010201D1620705D530228DF8042074
:1093A0004FF001087F1E582804D034A003900EA867
:1093B00002900DE036A0F9E753466046009AF6F7B2
:1093C00071FF84460398825C0298401E02900270EE
:1093D0005CEA0100F0D1029806A9081A00F1200AFF
:1093E000600702D524F4803400E00127574502DDF0
:1093F000A7EB0A0000E0002000EB0A0100900598AE
:109400004144401A0590E00306D45B462146179A72
:10941000059800F0B6F90544002706E001A85A4671
:10942000C05D179990476D1C7F1C4745F6DBE00334
:109430000CD55B462146179A059800F0A2F9054421
:1094400004E030205A46179990476D1C0099481E39
:1094500000900029F5DC08E0029802995A4600784D
:10946000491C0291179990476D1CBAF10001AAF1AD
:10947000010AF1DC65E100000928010030313233D6
:109480003435363738396162636465660000000040
:10949000303132333435363738394142434445462A
:1094A0000000000000F05BF90544761C30780028CD
:1094B0007FF4ECAD19B0284600F04EB9620700D435
:1094C000062709F1070222F0070CFCE80223E14617
:1094D00003F000485FEA080C02D00FF2702C0DE098
:1094E0005FEA045C02D50FF2682C07E05FEAC47CF7
:1094F00002D00FF2602C01E0AFF2700C4FF0FF3899
:1095000023F00043CDF850C065280CD006DC452878
:1095100009D046281DD047283DD13DE0662818D007
:1095200067287ED138E00021112F01DB112000E0F7
:10953000781CCDE9000106A90EA8FFF7E9FCDDE9DA
:109540000F010E9A03910021009207F1010A049184
:109550004DE04FF000400097CDE9011006A90EA89C
:10956000FFF7D6FCDDE90F0203920E9B1199002252
:10957000DDF80CA00093049211B9791C00EB010AEC
:10958000B7EB0A0004D4C0F1FF3007F1010A0490E0
:10959000AAEB0700019044E0012F00DA0127002127
:1095A000112F01DD112000E03846CDE9000106A9A8
:1095B0000EA8FFF7ADFCDDE90F010E9A0391002123
:1095C00004910092BA4621070CD40399514500DA60
:1095D0008A46BAF1010F05DD009AAAF10101515C3A
:1095E000302908D0B84202DA10F1040F06DA01215E
:1095F000CDE9011015E0AAF10101E9E7002805DC39
:10960000049901440491AAEB000102E0411C514578
:1096100000DD8A460499401A401C01904FF000403A
:109620000290200704D40198504501DBCDF8048056
:1096300000208DF84F0002980DF14F07B0F1004F58
:1096400025D02B200E9002984FF0020800280CDA4B
:10965000404202902D200E9007E00A210298F7F771
:109660005CF83031029007F8011DB8F10001A8F153
:109670000108F2DC02980028EFD1791E0E980870DC
:10968000307800F0200040F0450007F8020D12A8E5
:10969000C01B00F107081498007800B1012000EB0E
:1096A0000A01019801EBE07105984144401A401EFF
:1096B0000590E00306D45B462146179A059800F012
:1096C00060F805441498007818B15A4617999047E5
:1096D0006D1CE00324D55B462146179A059800F0DF
:1096E00050F805441CE00498002807DBDDE903017D
:1096F000884203DD0098405C179901E017993020FB
:109700005A469047049805F10105401C04900198C1
:10971000401E019004D12E205A46179990476D1C87
:10972000BAF10001AAF1010ADDDC05E017F8010B2E
:109730005A46179990476D1CB8F10001A8F101082D
:10974000F4DC5B462146179A0598ABE62D00000035
:109750002B0000002000000030BCBDE8C08F2DE9C8
:10976000F041044600251E461746880404D405E04F
:1097700039462020B0476D1C641EF9D52846BDE847
:10978000F0812DE9F041044600251E469046C803AD
:1097900001D5302700E02027880404D505E04146A4
:1097A0003846B0476D1C641EF9D52846BDE8F081E7
:1097B0004A68002A06D00A68531C0B60107048687B
:1097C000401E486070470A68531C0B601070704759
:1097D0002DE9F04116460D460746002407E03A5DA4
:1097E00006EB440004A1FFF749FB641CA4B2AC42A1
:1097F000F5D3BDE8F08100002530325800000000AC
:1098000070B505464FF6FF7000224AF201040DE0E4
:10981000AB5C58400023C6074FEA500000D06040C0
:109820005B1CDBB2082BF6D3521C92B28A42EFD3F8
:1098300070BD00002DE9FF5FF9F7DEFF8046394873
:10984000007E002863D00025A946414636A0FFF7D8
:10985000F1FA3BA0DFF8CCB000683A4E00244FF09C
:10986000010A0BF1980B039004EB4407364856F8B5
:109870002710A8EB0102824237D3214633A0FFF71D
:10988000D9FA06EB87010020087181F805A0384954
:109890000A19B9F1000F82F8A70101F2AD1202EB2B
:1098A000840201EB84011066C1F86E0101D14FF012
:1098B0000109C5F10A010DEB0500631C2DA2FFF79C
:1098C000C9FA0544022C07D2C5F10A010DEB0500C7
:1098D00029A2FFF7BFFA054403A99BF804200B5DFA
:1098E0000AFA03F18A438BF8042006EB87004079DB
:1098F000002858460DD003A902790B5D0AFA03F13E
:109900008A438BF80420641CE4B2032CACD300F02F
:1099100035B803AA0179135D0AFA03F211438BF8F3
:109920000410F0E714060010636865636B20434F72
:109930002063757272656E745F6D732025640A0012
:1099400000010200EC040010C02709006368656391
:109950006B20434F2025642063757272656E742DF1
:10996000636F756E745F6D732025640A00000000DC
:109970009C070010256400002C0000003FBCBDE8DF
:10998000C09F00002DE9F04F85B0F9F735FF014683
:10999000039037A0FFF74EFA3B48007E002861D0C5
:1099A0003AA00025DFF8E0900068394EA8462C4622
:1099B0000DF1100B4FF0010A09F19809CDF81000D4
:1099C00004EB4407039856F82710421A31488242A4
:1099D00037D3214630A0FFF72DFA06EB8701002090
:1099E000087181F805A035490A19B8F1000F82F80D
:1099F000AA0101F2AD1202EB840201EB8401D066F0
:109A0000C1F87A0101D14FF00108C5F10A010DEB4F
:109A10000500631C2AA2FFF71DFA0544022C07D299
:109A2000C5F10A010DEB050026A2FFF713FA054464
:109A30001BF8043099F805200AFA03F18A4389F8E3
:109A4000052006EB87001BF80430407999F80520C3
:109A50000AFA03F148B18A43641CE4B289F805208C
:109A6000032CADD305B000F02FB80A43F4E7000093
:109A7000636865636B2068322063757272656E740B
:109A80005F6D732025640A001406001004050600AB
:109A9000C8040010C0270900636865636B20683242
:109AA0002025642063757272656E742D636F756E08
:109AB000745F6D732025640A000000009C0700108D
:109AC000256400002C00000030BCBDE8C08F000001
:109AD000F8B5F9F791FE2249097E002937D021A176
:109AE0001F4A0968009100211F4F204C01236D4639
:109AF00012F1980254F83160861BBE4217D304EB72
:109B0000C10C00268CF804608CF80530DFF860C0CA
:109B10000CEB410CACF85A6015F801C0167903FA49
:109B20000CFE26EA0E06167144F8310003E004EB41
:109B3000C106767966B115F801C0167903FA0CFCF6
:109B400026EA0C06491CC9B216710329D2D3F8BD06
:109B500015F801E0167903FA0EFC46EA0C06F1E767
:109B60001406001004050600C0270900B004001008
:109B70004909001000250E4F2C4641F65836642046
:109B800002F06FFAB54202D900F014F800256435EE
:109B9000B44209D9FCF7B6FD054978641F31F7F7DF
:109BA000A9FC87F8200000246434F8F743F9E6E7BD
:109BB0001406001070B5114C207E012540B1207CA8
:109BC00050B101280BD002280CD0032810D10CE092
:109BD00000F016F8A57770BD00F012F807E0FFF767
:109BE00077FF05E0FFF7CEFE02E0FFF723FEA57743
:109BF000207C401C00F00300207470BD140600108F
:109C00002DE9F047F9F7F8FD0021DFF874901D4DBC
:109C10001D4A4FF0030A012301EB4106AAEBD104D0
:109C200055F826C0E4B2A0EB0C0801F00707C845C0
:109C300012D305EB86084FF0000C88F804C088F8B2
:109C4000053012F804C003FA07F82CEA080C02F8F1
:109C500004C045F8260003E005EB8606767956B188
:109C6000165D03FA07F7BE43491CC9B216551E29F3
:109C7000D2D3BDE8F087165D03FA07F73E43F3E75A
:109C8000C027090048030010AC06001070B5204C36
:109C9000208800281CD1A4F19E0188791D4A022841
:109CA00009D10020A2F2E5131D5C022D11D0401C49
:109CB000C0B21E28F8D3C879022809D1144800215F
:109CC0007838435C022B0ED0491CC9B20329F8D363
:109CD00070BD4FF20A032380431C00EB40006380F9
:109CE000105CA080E7E74FF20C002080481C02EBDC
:109CF0004105608095F85A2012B1FF2085F85B007D
:109D000015F85B3F04A0FFF795F82878A08070BD98
:109D1000B20600104909001073656E736F725F64BC
:109D200077696E5F646174615F6275666665722EE5
:109D300070726573737572655F646174615B2564CD
:109D40005D5B305D5B315D2025642025640D0A007C
:109D5000002808D0002A06D0002904D00023436040
:109D60000360C0E90212704710B54FF0FF3220B116
:109D700019B103684468A34201D1104610BD0368BD
:109D8000C268D25C0A7001688268491CB1FBF2F3B8
:109D900002FB13110160002010BD70B5C0B1C46892
:109DA000B4B18368A3B14268521CB2FBF3F503FB64
:109DB00015220568954206D105686D1CB5FBF3F6C2
:109DC00003FB165303604368E1544260002070BDFA
:109DD0004FF0FF3070BD00002DE9F04FE0488BB030
:109DE0000068016841F0100101604FF40072DD4924
:109DF000DB48FBF72DFCDC4C2079C0B10128FAD1FF
:109E00006079112881F04E84DFE810F033044A04B1
:109E100079049304A704A307C807EF04BF0435051A
:109E200020056C07190850088B08E0070C052078FE
:109E30001C282FD2DFE800F00E1E3044576D80FD45
:109E40002E95A5B7C8FCFBFAF9F8F7F6F52E2E2EDD
:109E50002EC6F4F301252B46C4A2C4A1C4A00095CC
:109E600003F018FE20B1C4A0FEF7E4FF2570C2E79E
:109E7000C3A00DE040F6B83002F0F3F8012302224F
:109E8000C2A1C6A003F098FD08B1C7A027E0C9A0F1
:109E9000FEF7D0FF002052E14FF4FA6002F0E1F843
:109EA00001230222C6A1C9A003F086FD18B1CAA0F1
:109EB000FEF7C0FF2BE0CBA0FEF7BCFF01203EE188
:109EC000012003460090A9A2A8A1CAA003F0E2FDC8
:109ED00020B1CBA0FEF7AEFF042030E1CBA0FEF70F
:109EE000A9FF02202BE10120034600909FA29FA121
:109EF000C9A003F0CFFD9B4802F0F0FBE06202280E
:109F000005D0FDF7FDFE02F0C3FC0D2017E1032094
:109F100015E10325012395A294A1C2A0009503F0A9
:109F2000B9FD20B1C6A0FEF785FF062049E0C8A014
:109F3000FEF780FF257045E00320009001238BA2EF
:109F40008AA1C8A003F0A6FD20B1CDA0FEF772FF44
:109F5000092000E0072020705FF0C80002F081F8BF
:109F600049E703200090012380A280A1C8A003F04C
:109F700091FD20B1CDA0FEF75DFF0A20EBE7D0A058
:109F80000EE001200346009078A278A1D24803F0A9
:109F900081FD20B1D1A0FEF74DFF0B20DBE7D3A060
:109FA000FEF748FFD6E70120034600906FA26FA19D
:109FB000D34803F06FFD00283CD0D2A0FEF73AFF53
:109FC0000C2020706420C9E7D24801AEC1788579A1
:109FD0004379027986E82E008178009143780278EF
:109FE000CDA1DA48FEF74AFFD84AD9A102F16400B0
:109FF000FEF744FF012003460090D4485BA25BA11A
:10A00000643003F047FDA8B1D049D7A0FEF712FF96
:10A0100001220421D948F9F7E9FB0D20D1E71BE320
:10A020000BE386E27CE28CE078E06EE047E035E02E
:10A0300015E004E0D2A0FEF7FDFE0720C1E70320F3
:10A040000090012349A249A1D1A003F023FD08B14A
:10A05000D3A000E0D7A0FEF7EDFE05207BE70220AD
:10A0600000900523D8A241A1DBA003F013FD20B18D
:10A07000E4A0FEF7DFFE0E2061E0E7A0FEF7DAFEC7
:10A0800001200090052339A238A1E9A003F002FDC8
:10A0900010B1EBA0FEF7CEFE0F2050E001200346EA
:10A0A000009032A231A1EAA003F0F4FC18B1112013
:10A0B0002070EFA026E00D202070F0A022E0607854
:10A0C000401CC1B261700A2904D300202070EFA0A7
:10A0D000FEF7B0FE6078642804D32349002048705E
:10A0E000FEF7F0FE012000900223F0A2EFA1F3A002
:10A0F00003F0D0FC18B10D202070F5A002E0042080
:10A100002070F7A0FEF796FE75E60120034600904A
:10A1100016A216A1F6A003F0BDFCBDE740F6B830CC
:10A1200001F09FFFFDF78CF920B110202070002076
:10A13000A07660E60120A076801EE06313202070E8
:10A1400059E60025A573FCF7ADFF10B1A5760F20E9
:10A1500020700120044D0026A073A435D6E1000034
:10A160007C3B00201E010010140600104F4B000025
:10A1700041540D0A0000000041545F4F4B0D0A008E
:10A1800041545F6661696C0D0A0000002B43504921
:10A190004E3A2052454144590000000041542B439F
:10A1A00050494E3F0D0A00004350494E5F4F4B0D42
:10A1B0000A0000004350494E5F6661696C0D0A0059
:10A1C0002B43455245473A20302C310041542B4314
:10A1D000455245473F0D0A0043455245475F4F4BA7
:10A1E0000D0A000043455245475F6661696C0D0AE0
:10A1F0000000000041542B4346554E3D310D0A00EE
:10A200004346554E5F4F4B0D0A0000004346554EE6
:10A210005F6661696C0D0A0041542B43434C4B3F10
:10A220000D0A000041542B4D5545434F4E464947BA
:10A230003D226175746F636F6E6E222C310D0A00C2
:10A240004D5545434F4E4649475F4F4B0D0A000061
:10A250004D5545434F4E4649475F6661696C0D0A4F
:10A260000000000041542B4D4449414C5550434699
:10A27000473D226175746F222C310D0A00000000E9
:10A280004D4449414C55504346475F4F4B0D0A00E2
:10A2900041542B4D5154544346473D2263616368FA
:10A2A0006564222C302C310D0A0000004D515454AD
:10A2B0004346475F4341434845445F4F4B0D0A00C7
:10A2C0004D5154544346475F4341434845445F66BC
:10A2D00061696C0D0A000000C0F300084D51545430
:10A2E000434F4E4E455F4F4B0D0A00004D515454A5
:10A2F000434F4E4E455F6661696C0D0A00000000D9
:10A3000064F400084D5154545355425F4F4B0D0AAD
:10A3100000000000CE0600202F6B317663634C4AAC
:10A32000767355792F253032582530325825303202
:10A3300058253032582530325825303258253032A1
:10A34000582F757365722F67657400001005001033
:10A3500041542B4D5154545355423D302C222573BA
:10A36000222C310D0A0000004D5154545355425FC8
:10A370004F4B3A2025730D0A00000000000C0048E6
:10A380004D5154545355425F6661696C0D0A00008B
:10A3900041542B4D515454444953433D300D0A0010
:10A3A00041542B4D515454444953435F4F4B0D0A74
:10A3B0000000000041542B4D515454444953435F15
:10A3C0006661696C0D0A00002B4D49504F50454E97
:10A3D0003A20302C3000000041542B4D49504F5052
:10A3E000454E3D302C22544350222C2234372E31FE
:10A3F00030392E37332E313637222C31303030324F
:10A400000D0A00004D49504F50454E5F5443505F78
:10A4100049505F4F4B0D0A004D49504F50454E5F1C
:10A420005443505F49505F6661696C0D0A0000003B
:10A4300041542B4D4950434C4F53453D300D0A007C
:10A440004D49504F50454E5F6661696C0D0A0000E2
:10A4500041542B4D49504346473D22656E636F641E
:10A46000696E67222C302C312C310D0A000000005F
:10A470004D49504346475F4F4B0D0A004D495043ED
:10A4800046475F6661696C0D0A0000004D49504304
:10A490004C4F53455F6D61785F7265747269657387
:10A4A0002C746F2041542C25640D0A002B4D49500B
:10A4B000434C4F53453A20300000000041542B4D8F
:10A4C0004950434C4F53453D302C300D0A0000009D
:10A4D0004D4950434C4F53455F4F4B0D0A00000010
:10A4E0004D4950434C4F53455F6661696C0D0A00FE
:10A4F00041542B4353510D0A00000000207E0028D8
:10A500007FF4B5AC642001F0ACFD6436E87900EB73
:10A510004001C1EBC010B6EBC00FBFF4A8ACEDE733
:10A52000FDF7ECFA18B10020A0760F20207014205F
:10A5300005E601F0A3FD81464E46B046EC4F2546A8
:10A5400001F09CFD0446297E002021B9397AC1EB37
:10A5500001114900A984297E012902D0297E0229FE
:10A5600001D1397AA984397899B9A98CA4EB090267
:10A5700001EB4103C3EBC111B2EBC10F09D30022C0
:10A5800010214FF09040F9F731F9FDF717F8A14687
:10A590000120FA79A11B02EB4203C3EBC212B1EB1B
:10A5A000C20F0ED3002210214FF09040F9F71EF990
:10A5B000FCF778FD18B10020A8760F2024E026468D
:10A5C0000120797AA4EB080201EB4103C3EBC1112E
:10A5D000B2EBC10F0BD3002210214FF09040F9F7DE
:10A5E00005F9FDF7BBF90028E5D1A04601202A7E38
:10A5F000E96B8A420AD0297EBEA0FEF71BFCFFF75A
:10A6000045FB287EE8631320287030E488B10120E0
:10A610000346AFF2A842AFF2AC410090BCA003F0F9
:10A6200039FA012210214FF09040F9F7DFF8F7F7DF
:10A6300001FC0A2001F015FD82E701231A46AFF262
:10A64000D441BBA003F0B8F920B1192020704FF419
:10A65000967083E4BAA009E001231A46AFF2F441F0
:10A66000BDA003F0A9F90028EFD1BFA0FEF7E2FBDF
:10A67000EBE7AFF2045003F083F9AFF21050019012
:10A680004FF47A7000904FF48073BC4A012101A806
:10A6900003F010FF08B9BAA02EE0022000F0E9BFD5
:10A6A000BBA003F06DF9BEA001904FF4FA7001F069
:10A6B000D8FC4FF4FA6000904FF48073AF4A012148
:10A6C00001A803F0F7FEB0B14FF47A75284601F007
:10A6D000C8FCB7A0FEF7AEFBBB4E0022802130467F
:10A6E000F9F784F8284601F0BCFC012280213046AD
:10A6F000F9F77CF81BE0B5A0FEF79CFBCDE7B8A00E
:10A7000003F03EF9AFF29C5001904FF47A70009044
:10A710004FF48073994A012101A803F0CBFE08B1E0
:10A72000B3A0FBE3B8A0FEF785FB0320B6E701204A
:10A73000B4E7BAA003F024F999A001904FF4FA60AD
:10A7400000904FF480738D4A012101A803F0B2FEFE
:10A7500008B1B5A0E5E7B9A012E3BCA003F010F979
:10A76000AFF2F85001904FF47A7000904FF480737C
:10A77000824A012101A803F09DFE08B1B8A0D0E7EC
:10A78000BEA0FEF757FB082088E7C2A003F0F8F848
:10A79000C3A00190C7A00290CCA00390D0A00490C9
:10A7A000D5A0059040F6B83000904FF48073734AFE
:10A7B000052101A803F07EFE052814D2DFE800F091
:10A7C0000305070C0E00D3A086E0D8A000E0DEA0B1
:10A7D000FEF730FB092061E7E1A033E0E7A0FEF7D8
:10A7E00029FB0A205AE7EDA09BE700254FF47A7673
:10A7F0004FF48077EFA003F0C3F8AFF29060CDE99B
:10A8000000603B465D4A012101A803F053FE20B1E0
:10A810006D1C032DEEDBEBA083E7EFA0FEF70AFB38
:10A8200010203BE75EA001904FF47A7000904FF447
:10A830008073524A012101A803F03CFE08B17AA0BE
:10A84000ECE77EA0FEF7F6FA0B2027E7E6A003F080
:10A8500097F8AFF2E86001904FF47A7000904FF4EF
:10A860008073464A012101A803F024FE08B1E1A04B
:10A8700057E7E6A0ACE7E078032801D0FBF77EF9C4
:10A880001B49E6A00C31FEF7D5FA1949E7A02031A3
:10A890000D46FEF7CFFA164829460C3003F08EF924
:10A8A000E7A00190E9A00290EBA00390EEA0049035
:10A8B000F2A0059040F6B83000904FF480732F4A14
:10A8C000052101A803F0F6FD05280ED2DFE800F00F
:10A8D00003080A0C0E00EEA0FEF7ACFA0720DDE636
:10A8E000EFA075E7F4A073E7F6E1F9E1F6E1000007
:10A8F000B806001053797374656D5F4C6576656CAE
:10A900005F4368616E6765643A2025640A00000051
:10A9100041542B4D4C504D4346473D22736C656569
:10A92000706D6F6465222C322C300D0A000000001F
:10A9300041542B4D474E53534C4F433F0D0A00009B
:10A9400041542B4D474E53534C4F433D305F66614E
:10A95000696C0D0A0000000041542B4D474E5353C3
:10A960004C4F430D0A00000041542B4D474E5353AA
:10A970004C4F435F6661696C0D0A0000B905002009
:10A98000574946495F41545F4F4B0D0A0000000094
:10A9900041542B524553544F52450D0A00000000BC
:10A9A0002B494E49543A444F4E452C30000000008C
:10A9B000574946495F524553544F52455F554E4B98
:10A9C0004E4F574E0D0A00000008004857494649AF
:10A9D0005F524553544F52455F4F4B0D0A000000E4
:10A9E00041542B43574D4F44453D300D0A00000064
:10A9F000574946495F43574D4F44455F554E4B4E6F
:10AA00004F574E0D0A000000574946495F43574DC6
:10AA10004F44455F4F4B0D0A0000000041542B523C
:10AA200053540D0A00000000574946495F525354E1
:10AA30005F554E4B4E4F574E0D0A00005749464941
:10AA40005F5253545F4F4B0D0A00000041542B548A
:10AA50004350444154414D4F44453D300D0A0000A0
:10AA6000574946495F544350444154414D4F444532
:10AA70005F554E4B4E4F574E0D0A00005749464901
:10AA80005F544350444154414D4F44455F4F4B0D3B
:10AA90000A00000041542B4357535441540D0A00FF
:10AAA0007770615F73746174653D434F4D504C45E1
:10AAB000544544007770615F73746174653D444927
:10AAC00053434F4E4E454354454400007770615FF9
:10AAD00073746174653D5343414E4E494E470000C7
:10AAE0007770615F73746174653D4153534F43499F
:10AAF00041544544000000007770615F73746174D5
:10AB0000653D345741595F48414E445348414B4598
:10AB100000000000574946495F4357535441545F72
:10AB2000434F4D504C455445440D0A005749464942
:10AB30005F4357535441545F444953434F4E4E452E
:10AB4000435445440D0A0000574946495F43575353
:10AB50005441545F5343414E4E494E470D0A000045
:10AB6000574946495F4357535441545F4153534FEC
:10AB70004349415445440D0A0000000057494649E5
:10AB80005F4357535441545F345741595F48414ED6
:10AB9000445348414B450D0A0000000057494649BF
:10ABA0005F4357535441545F554E4B4E4F574E0DD4
:10ABB0000A00000041542B44504D3D312C300D0A09
:10ABC00000000000574946495F44504D5F554E4BC9
:10ABD0004E4F574E0D0A0000574946495F44504DAD
:10ABE0005F4F4B0D0A00000041542B435751415019
:10ABF0000D0A0000574946495F43575141505F5580
:10AC00004E4B4E4F574E0D0A000000005749464923
:10AC10005F43575141505F4F4B0D0A00574946491A
:10AC20002E535349443A2025730A00005749464998
:10AC30002E50617373776F72643A2025730A000097
:10AC40002B43574A41503A31000000004552524FC1
:10AC5000523A2D31340000002B43574441503A30D2
:10AC60002C444541555448002B43574A41503A30F3
:10AC70002C57524F4E475057440000002B43574A21
:10AC800041503A302C54494D454F55540000000076
:10AC9000574946495F43574A41505F4F4B0D0A00A1
:10ACA000574946495F43574A41505F4552524F52B8
:10ACB0003A2D31340D0A0000574946495F43574A3F
:10ACC00041505F2B43574441503A302C4445415545
:10ACD00054480D0A00000000CCA022E5D3A020E5D6
:10ACE000DAA075E5012000F09DFEDEA002F048FE2E
:10ACF000642001F0B6F9E0A00190AFF2B00002903C
:10AD0000E0A0002540F6B8364FF480770390E0A02D
:10AD100002F036FE3B46E74A032101A8009603F005
:10AD2000C9FB40B16D1C032DF1DB01280DD00228B9
:10AD30000DD0E1A0F5E4DF4800F0A4FF0546014690
:10AD4000E3A0FEF777F8A56461E0E8A0E9E4EEA0EF
:10AD5000E7E4F4A002F014FEAFF6F0300190AFF299
:10AD6000081002904FF4FA6000904FF48073D14ABB
:10AD7000022101A803F09EFB30B1022809D0F2A005
:10AD8000FEF758F8042089E4F5A0FEF753F80620F2
:10AD900084E4F8A0FEF74EF805207FE4FBA002F063
:10ADA000EFFDAFF6384001904FF47A7000904FF409
:10ADB0008073C04A012101A803F07CFB08B1F7A011
:10ADC000DEE7FCA0FEF736F80F2067E4FD4F002514
:10ADD0004FF47A764FF48078FBA002F0D1FDFDA00D
:10ADE000CDE900604346B34A012101A803F062FBAC
:10ADF00078B1FAA0FEF71EF830466D1C03F02CFA6D
:10AE0000062DE9DBF7F7C6F9E06201F041FD0C2001
:10AE1000ECE3A848FBF7CEFA0146E062B8420AD953
:10AE2000F6A0FEF707F8E06AFCF76AFF01F030FDD4
:10AE3000062DE7DAEBE7F5A0FDF7FCFFDCE7FDA068
:10AE40000190FEA000254FF4FA794FF4967A4FF462
:10AE50007A774FF4807802900120FDF7ADFD4846E7
:10AE600001F0FFF84346934A022101A8009703F03E
:10AE700021FB060011D06D1C2946F3A0FDF7DAFF77
:10AE8000504601F0EEF8052DE6DB012E0CD0F6A0C1
:10AE9000FDF7D0FF0020A07649E4F9A0FDF7CAFF36
:10AEA0000120A0760D20E4E3FAA0F1E7E1A00190F3
:10AEB000E2A000254FF4FA794FF4967A4FF47A77AE
:10AEC0004FF4807802900120FDF764FF484601F0BE
:10AED000C8F84346774A022101A8009703F0EAFA2E
:10AEE000064694F8220058B1F1A0FDF7A3FF01F047
:10AEF000CFFC0120A076002084F822000E20B8E3C9
:10AF00006D1C2946EFA0FDF795FF504601F0A9F80A
:10AF1000052DD8DB012E02D0F2A0B9E724E2F7A07C
:10AF2000B6E701F0ABF8002108900790CDE90510D5
:10AF30008346AFF6C8500190C0A00290F6A00390DF
:10AF4000F8A00490F7A0DFF8E4A3099001F096F8C8
:10AF50000546207E002628B99AF80800C0EB0010AC
:10AF60004000A084207E012802D0207E022802D149
:10AF70009AF80800A0849AF80000D046002840D132
:10AF8000A18C089801EB4102281AC2EBC111B0EB69
:10AF9000C10F37D3012000F045FD00274FF47A762A
:10AFA0004FF480792FA002F0EBFC4B46414A04217C
:10AFB00001A8009603F07EFA30B1642001F051F848
:10AFC0007F1C032FEEDB10E3002000F02BFD002799
:10AFD0004FEA0709F7F7DEF8E062D5490120FDF7EF
:10AFE0005DFD4FF48073334A042101A8009603F0FD
:10AFF00061FA28B17F1C012805D0022804D099E10C
:10B000009AE1F3E1B4E1A1E1A2E100005749464928
:10B010005F43574A41505F2B43574A41503A302CC7
:10B0200057524F4E475057440D0A00005749464962
:10B030005F43574A41505F2B43574A41503A302CA7
:10B0400054494D454F55540D0A0000005749464993
:10B050005F43574A41505F554E4B4E4F574E0D0A76
:10B060000000000041542B434C5244504D534C506F
:10B070004558540D0A0000002B4349505354415287
:10B08000543A00004552524F523A2D3733360000A1
:10B0900041542B43495053544152543D31302E3981
:10B0A000302E302E31342C31303030322C300D0AED
:10B0B00000000000B9050020574946495F43495048
:10B0C00053544152545F554E4B4E4F574E0D0A004C
:10B0D000574946495F43495053544152545F4F4B7F
:10B0E0002C204944203D2025640D0A00574946493B
:10B0F0005F43495053544152545F4552524F523A64
:10B100002D31340D0A000000574946495F4349502C
:10B1100053544152545F4552524F523A2D373336B1
:10B120000D0A000041542B434950534E54503D31B9
:10B130002C226E74702E6E7473632E61632E636E98
:10B14000222C3132330D0A00574946495F4349509A
:10B15000534E54505F554E4B4E4F574E0D0A000004
:10B16000574946495F434950534E54505F4F4B0D2A
:10B170000A000000574946495F434950534E545016
:10B180005F616761696E0D0A0000000041542B5435
:10B190005A4F4E453D300D0A0000000057494649C0
:10B1A0005F545A4F4E455F554E4B4E4F574E0D0A0A
:10B1B00000000000574946495F545A4F4E455F4FC3
:10B1C0004B0D0A008085746741542B54494D453D11
:10B1D0003F0D0A002B54494D453A00005749464956
:10B1E0005F54494D455F554E4B4E4F574E2C207284
:10B1F00065747279696E670D0A0000005749464907
:10B200005F54494D455F4F4B0D0A000054494D4571
:10B2100020696E76616C6964202865706F63683A96
:10B2200020256C64292C207265747279696E670D13
:10B230000A0000002B54524454433A004552524FE6
:10B24000523A2D3400000000574946495F52656765
:10B2500069737465725F5265747279202564206623
:10B2600061696C65640D0A00574946495F5265671C
:10B2700069737465725F554E4B4E4F574E0D0A0001
:10B28000574946495F52656769737465725F4F4BF2
:10B290000D0A0000574946495F5265676973746536
:10B2A000725F4552524F523A2D340D0A0000000091
:10B2B000574946495F756E697874696D655F4F4B94
:10B2C0000D0A0000574946495F756E697874696DCB
:10B2D000655F5265747279202564206661696C65CA
:10B2E000640D0A00574946495F756E697874696D47
:10B2F000655F554E4B4E4F574E0D0A005749464914
:10B300005F756E697874696D655F4552524F523A48
:10B310002D340D0A000000004552524F523A2D3193
:10B32000000000002B54525854433A00B806001055
:10B330009C070010DCA00CE0E5A0FDF77BFD0120E0
:10B34000A07606460895032F0DDA0EE0E8A000E08F
:10B35000F1A0FDF76FFD84F81A90642000F081FEE3
:10B36000032FFFF637AEF64880E198F80000E8BBFF
:10B37000A18C079801EB4102281AC2EBC111B0EB76
:10B38000C10F53D3012000F04DFB00274FF47A7614
:10B390004FF48079AFF2343002F0F2FA4B46E94ACA
:10B3A000042101A8009603F085F830B1642000F074
:10B3B00058FE7F1C032FEDDB17E1002000F032FB6D
:10B3C0000027B946F6F7E6FEE062DF490120FDF707
:10B3D00013FA4FF48073DB4A042101A8009603F0AE
:10B3E00069F840B17F1C012812D000E01EE002285D
:10B3F00010D0D6A00FE0DFA0FDF71CFD0120A07645
:10B40000142000F02EFE01260795032F0CDA0DE024
:10B41000E1A000E0EBA0FDF70DFD84F81A90642098
:10B4200000F01FFE032FCDDBF1481FE198F8070065
:10B43000A5EB0B0100EB4002C2EBC010C246B1EB22
:10B44000C00F52D3012000F0EDFA00274FF4967997
:10B450004FF47A764FF48078AFF2F83002F090FA39
:10B46000484600F0FEFD4346B64A042101A8009676
:10B4700003F020F830B1484600F0F3FD7F1C032FA5
:10B48000EADBB2E0002000F0CDFA0027B34601204D
:10B49000FDF762F94E46484600F0E3FD4346A94AEF
:10B4A000012109A8CDF800B003F004F84FF4FA70B8
:10B4B00000F0D7FD94F8210060B1CEA0FDF7BAFCF2
:10B4C0000120A0760020AB4684F821000126032F3E
:10B4D00009DA0AE0CEA07F1CFDF7ACFC304600F094
:10B4E000C0FD032FD3DBD3A0C0E0DDE905124FF090
:10B4F0000009AB1A69EB01009AF809104FF47A724F
:10B5000011FB02F1CA17591A904150D3012000F0E3
:10B5100089FA00274FF47A764FF48078AFF2BC4076
:10B5200002F02EFA4346874A042101A8009602F051
:10B53000C1FF30B1642000F094FD7F1C032FEDDBD0
:10B5400053E0002000F06EFA5FF00007F6F722FEED
:10B55000E0620120FDF73EFB43467A4A042101A840
:10B56000009602F0A7FF30B17F1C012811D00228FD
:10B5700011D0C0A010E0C7A0FDF75CFC0120A076B0
:10B58000CDE905950646206D401C2065032F0CDA99
:10B590000DE0C7A000E0CEA0FDF74CFC84F81A90A7
:10B5A000642000F05EFD032FD0DBD1485EE0207EFA
:10B5B000E16B884260D0012000F034FA00254FF49E
:10B5C0007A764FF48077AFF2645002F0D9F93B46B7
:10B5D0005C4A042101A8009602F06CFF68B1642067
:10B5E00000F03FFD6D1C032DEDDB00E041E0C1A04C
:10B5F000FDF720FC0BB000F001BA002000F012FAB9
:10B60000B84600254F46217EAFF61850FDF712FCD4
:10B61000FEF73CFBF6F7BEFDE0620120FDF740FBC4
:10B620004346484A042101A8009602F043FF30B186
:10B630006D1C01280ED002280ED0BCA00DE0C3A0C6
:10B64000FDF7F8FB0120A0760646207EE063032D7F
:10B650000BDA11E0C4A000E0CCA0FDF7EBFBA7766D
:10B66000642000F0FEFC032DCDDBD148FDF7E2FBAA
:10B6700012E46071FEF7BFBB206D642806DB0D206D
:10B680006071CCA0C4F85090FDF7D4FB36B1207E99
:10B6900010B9D5A002F074F9F6F7CCFB0A2000F03F
:10B6A000E0FC53E40020E4E7574946495F53656EE8
:10B6B000645F54656D70657261747572655F446135
:10B6C00074615F554E4B4E4F574E0D0A00000000FF
:10B6D000574946495F53656E645F54656D70657286
:10B6E00061747572655F446174615F4F4B0D0A0050
:10B6F000574946495F53656E645F54656D70657266
:10B7000061747572655F446174615F4552524F5256
:10B710003A2D340D0A000000574946495F53656EC3
:10B72000645F54656D70657261747572655F4461C4
:10B7300074615F4552524F523A2D310D0A0000009C
:10B74000F4F40008B90500209C0700105749464949
:10B750005F53656E645F50726573737572655F43A6
:10B760004F5F48325F446174615F554E4B4E4F5797
:10B770004E0D0A00574946495F53656E645F50722B
:10B780006573737572655F434F5F48325F446174E0
:10B79000615F4F4B0D0A0000574946495F53656E84
:10B7A000645F50726573737572655F434F5F4832B3
:10B7B0005F446174615F4552524F523A2D340D0A15
:10B7C00000000000574946495F53656E645F507240
:10B7D0006573737572655F434F5F48325F44617490
:10B7E000615F4552524F523A2D310D0A0000000060
:10B7F000A8F40008574946495F53656E645F486581
:10B80000617274626561745F4F4B0D0A0000000045
:10B81000574946495F53656E645F4865617274625B
:10B820006561745F4E6F74207265636569766564E7
:10B830000D0A0000574946495F53656E645F4865CD
:10B8400061727462656174204641494C45442061CF
:10B8500066746572203320726574726965732E2078
:10B86000476F746F20574946495F524553544F52B2
:10B87000450D0A00574946495F53656E645F73651D
:10B880006E736F726C696E655F554E4B4E4F574EBF
:10B890000D0A0000574946495F53656E645F736542
:10B8A0006E736F726C696E655F4F4B0D0A0000001E
:10B8B000574946495F53656E645F73656E736F7277
:10B8C0006C696E655F4552524F523A2D340D0A0035
:10B8D000574946495F53656E645F73656E736F7257
:10B8E0006C696E655F4552524F523A2D310D0A0018
:10B8F0003CF5000841542B434C5244504D534C509E
:10B90000455854206661696C65642061667465728F
:10B9100020726574726965732C20736B6970207373
:10B92000656E64696E670D0A00000000574946495C
:10B930005F53656E645F73797374656D6C6576656E
:10B940006C5F554E4B4E4F574E0D0A0057494649B6
:10B950005F53656E645F73797374656D6C6576654E
:10B960006C5F4F4B0D0A0000574946495F53656EA7
:10B97000645F73797374656D6C6576656C5F455251
:10B98000524F523A2D340D0A0000000057494649E3
:10B990005F53656E645F73797374656D6C6576650E
:10B9A0006C5F4552524F523A2D310D0A0000000093
:10B9B00080F500085265616368656420313030208D
:10B9C0006D696E757465732C20737769746368692B
:10B9D0006E6720746F20574946495F756E697874A9
:10B9E000696D650D0A00000041542B5345544450C5
:10B9F0004D534C504558540D0A00000030BCBDE872
:10BA0000C08F000002464FF400610148F7F7EEBE18
:10BA100000080048024610210148F7F7E7BE000081
:10BA20000004004880F001024FF480710148F7F7EC
:10BA3000DDBE000000080048F0B50023044640F2D7
:10BA4000B2761D460AE0304600F0F8F910B103F571
:10BA5000B77301E003F26D13761CB6B22088B042D2
:10BA6000F1D8144EA6F10C07A078401EA8420ADDBA
:10BA7000208800F0E3F908B1705D00E0785D6D1C8E
:10BA80000344ADB2F0E7E0785B1E0B49184448432D
:10BA90006179C1EB4112C2EB012100EB0110A179E8
:10BAA000C1EB011100EB8100E1790844A0F5E14010
:10BAB000F0BD000050F10008805101000B46F0B5C8
:10BAC00030494FF46166B0FBF1F2B0FBF1F401FBD9
:10BAD0001401B1FBF6F406FB14173C24B7FBF4F792
:10BAE00000251D60B1FBF6F05D609F71B1FBF6F7BC
:10BAF00006FB1711B1FBF4F604FB16110830C0B2B7
:10BB0000D9715871172802D918385871012540F297
:10BB1000B551B2FBF1F040F2B27404EB8000B2FB1D
:10BB2000F1F401FB142180B2294418808CB200F09A
:10BB300085F94FF4B7756E1E06E0401C80B2611A9D
:10BB400018808CB200F07AF908B1294600E031463D
:10BB500018888C42F1D200F071F908B10A4A01E06C
:10BB6000094A0C3A641CA0B203E0001B491C80B2D5
:10BB700099709978545C8442F7D3C9B2491C997082
:10BB8000D870F0BD8051010050F10008FAF752FC66
:10BB90005A2002F061FBF9E7F0B50D460646002495
:10BBA0001FE0305D7E2802D07D280BD017E03719CA
:10BBB0002A1B791CB81C521E00F04BFA7D20305510
:10BBC000022007E037192A1B791CB81C521E00F00E
:10BBD00040FA01206D1C641C7870ADB2A4B2641CE4
:10BBE000A4B2AC42DDD32846F0BD00002DE9F041FF
:10BBF000C2B020A1F4F710FC002837D01FA1F4F741
:10BC00000BFC040032D01DA1A01CF4F705FC08B108
:10BC1000801C05E01AA12046F4F7FEFB002825D081
:10BC2000071B002F22DDB7F5007F1FDC00263546FD
:10BC3000E846409612E0605D90B161194A787AB1A9
:10BC40008DF8000148788DF801011022002140A8EC
:10BC5000F4F70BFD08F80600AD1C761CBD42EADBCC
:10BC6000002E03DDB1B2684600F07EFC42B0BDE8B4
:10BC7000F08100002B54524454433A0037450000F1
:10BC80000D0A000010B506A1F4F7C6FB20B1BDE80F
:10BC900010400A30F4F721BD4FF0FF3010BD000016
:10BCA0002B43495053544152543A000010B502F00E
:10BCB000B5F8C72002F064F802F074F806490020D5
:10BCC00048604FF480510548F4F79BFBBDE81040F5
:10BCD00003A0FDF7AFB80000F0060010C03E002042
:10BCE000573235464C41534820636F6D706C657414
:10BCF0006520656D70746965640D0A002DE9F05F5B
:10BD00001D4C83460E466068DFF8708030444FF06B
:10BD10000109B0F1807F0FD3002005464FF4805A0F
:10BD200047466060280302F003F802F03BF807F88A
:10BD300005906D1C5545F5D36068050B3044401ED9
:10BD4000070B0AE018F8050030B9280301F0F0FFEE
:10BD500002F028F808F805906D1CBD42F2D9324671
:10BD60005946606802F038F802F01CF86068304408
:10BD7000606000F005B80000F0060010C03E002032
:10BD800030BCBDE8C09F000013B54FF6FF73012221
:10BD900069460248F9F7BEFC00981CBD743A0020C1
:10BDA000114810B5C07809281BD2DFE800F014163E
:10BDB000181A1A1A050A0F000CA0FDF73BF8062006
:10BDC00010BD11A0FDF736F8072010BD15A0FDF736
:10BDD00031F8082010BD002010BD012010BD022048
:10BDE00010BD092010BD0000140600104457494E34
:10BDF0005F53544154455F44454255475F5357494B
:10BE00005443480A000000004457494E5F535441D0
:10BE100054455F5741524E494E475F53574954432B
:10BE2000480A00004457494E5F53544154455F53FC
:10BE300045545F5357495443480A000081070CD1C9
:10BE40006421B0FBF1F201FB120141B94FF4C8715A
:10BE5000B0FBF1F201FB120008B100207047012095
:10BE6000704700001CB507A2D2E90012CDE900120C
:10BE700007226946F4F7FFFA08B100201CBD012033
:10BE80001CBD00005AA50683100301001CB50178F3
:10BE9000102909D0112907D0122905D0012903D072
:10BEA000022901D0032914D14178032911D18178C5
:10BEB00004290ED1B0F80710ADF800100721FDF7E6
:10BEC0009FFCADF80400022201A96846F4F7D3FAFA
:10BED00008B100201CBD01201CBD00001CB507A23C
:10BEE000D2E90012CDE9001207226946F4F7C3FA3D
:10BEF00008B100201CBD01201CBD00005AA506830E
:10BF0000150001001CB507A2D2E90012CDE900120C
:10BF100007226946F4F7AFFA08B100201CBD0120E2
:10BF20001CBD00005AA50683160001001CB507A21F
:10BF3000D2E90012CDE9001205226946F4F79BFA16
:10BF400008B100201CBD01201CBD00005AA50C83B7
:10BF5000550000001CB507A2D2E90012CDE900127D
:10BF600005226946F4F787FA08B100201CBD0120BC
:10BF70001CBD00005AA506835500000001785A290F
:10BF800008D14178A52905D1C178832902D100794A
:10BF9000562801D00020704701207047F7F774FC45
:10BFA000FBF7FEFEF9F77AFFF9F7B4FEFAF772F83D
:10BFB000FAF78EF8F9F78AFEFAF720F8FAF7A6F8FA
:10BFC000FAF704F8F9F746FEFAF73CF801F0AAFF91
:10BFD0000F4C002204212046F7F708FC4FF4FA70BA
:10BFE000F7F708FA012204212046F7F7FFFB40F695
:10BFF000B830F7F7FFF9F5F7CDF906A0FCF71AFF0F
:10C0000000F044F8F9F7C4FE00F052F8FEE7000033
:10C01000000400484D61696E426F6172642048659A
:10C020006C6C6F2056323032355F303532300D0A4D
:10C0300000000000427862F30701027862F30F21EA
:10C04000C278807862F3174160F31F6100EE101A26
:10C050007047002A04D0521E02D48B5C8354FAE746
:10C06000704710B5EFF3058111B16FF0050403E0DF
:10C07000002408B102F0F0F8204610BDEFF305806F
:10C0800008B102F0B5BE02F0ADBE0000EFF30580CE
:10C0900010B16FF0050070470448016811B14FF00E
:10C0A000FF30704701210160002070473C070010FD
:10C0B00010B5EFF3058010B16FF0050010BD084812
:10C0C0000168012902D04FF0FF3010BD054A002160
:10C0D00082F8141D0221016002F06EF9002010BDEB
:10C0E0003C0700100BE000E0F8B514464FF00005E7
:10C0F000EFF3058212BB08B301B3A4B1D4E9023255
:10C1000063B1542A1AD32269C2B1676900FB01F6F0
:10C11000B74213D3009502F037FB07E072B92269EA
:10C1200062B9626952B9002202F00DFB050005D028
:10C130000CB1216800E0002102F02CF82846F8BD7F
:10C1400070B505464FF00004EFF3058050BB0DB10C
:10C15000686800E00020C10701D0012600E0002649
:10C1600000071FD46DB1D5E9021021B1542819D3AD
:10C170001EB1042002E020B114E0012002F0D6FA42
:10C1800005E00EB1042000E0012002F0C4FA040032
:10C1900008D00DB1296800E0002101F0FBFF0EB1CD
:10C1A00044F00104204670BDF8B5144603460E461F
:10C1B0004FF00005EFF3058098BB93B39E423DD846
:10C1C0004CB1A0680028E06803D0542836D3012081
:10C1D00002E008B132E00020012B05D010B3184670
:10C1E000A26802F078FA20E040B10320009000221B
:10C1F00011460120A36802F0C7FA04E003220021DF
:10C20000012002F0A0FA050018D086B100231A46DA
:10C21000194602F031FB012809D0284601F0CEFF73
:10C2200000250BE0184602F039FA050006D00CB1E3
:10C23000216800E00021284601F0ACFF2846F8BD47
:10C240002DE9FF410B464FF00005EFF30581039503
:10C2500049BB40B38027182100244AB3166806B1B1
:10C26000344696691EB13146761E382E02D21679B2
:10C27000F60703D0002004B0BDE8F081566906B18E
:10C28000B708D2F808C0BCF1000F0DD0D5685C2DFE
:10C2900018D312693AB136B18DE806103A462146F4
:10C2A00002F066FD03900DE0D6685EB912694AB9E6
:10C2B00003AACDE90012BAB2214602F029FD0128F5
:10C2C00000D003950398D6E72DE9F04782468846CB
:10C2D0003CA0FCF7AFFD0125DFF810913BE000BF6B
:10C2E0000AEB050001888678C4784FBA23463246A7
:10C2F00039463FA0FCF79EFD6FF4714010FA87F0BD
:10C30000092821D2DFE800F005080B0E1114171AD6
:10C310001D0089F800401BE089F8014018E089F809
:10C32000024015E089F8034012E089F804400FE06C
:10C3300089F805400CE089F8064009E089F80740D3
:10C3400006E089F8084003E0394634A0FCF772FDA6
:10C35000A819C01C85B24545C2D3082223494FF411
:10C360008810F5F76BF835490120087034A0FCF708
:10C3700061FD4C4699F8001037A0FCF75BFD617831
:10C380003CA0FCF757FDA17842A0FCF753FDE178F3
:10C3900048A0FCF74FFD21794DA0FCF74BFD6179DA
:10C3A00051A0FCF747FDA17955A0FCF743FDE179C9
:10C3B0005CA0FCF73FFD217ABDE8F04761A0FCF7E7
:10C3C00039BD00005465726D696E616C20506172F8
:10C3D000616D657465722053657474696E6773204E
:10C3E00052656365697665643A0A0000B806001014
:10C3F000506172616D2049443A20307825303458BC
:10C400002C204C656E6774683A2025642C20566198
:10C410006C75653A2025640A00000000556E6B6E4D
:10C420006F776E20506172616D657465722049444A
:10C430003A203078253034580A00000021060010D8
:10C440005570646174656420666C6173685F6461D3
:10C4500074613A0A00000000436F6E74726F6C20C2
:10C460005472616E736D697420466C61673A202561
:10C47000640A000054656D7020466972737420541C
:10C4800068726573686F6C643A202564C2B0430AB1
:10C490000000000054656D70205365636F6E64206A
:10C4A0005468726573686F6C643A202564C2B04347
:10C4B0000A000000507265737375726520546872CB
:10C4C0006573686F6C643A2025642050610A00002F
:10C4D000434F205468726573686F6C643A2025641A
:10C4E0002070706D0A000000483220546872657335
:10C4F000686F6C643A2025642070706D0A0000003B
:10C50000536D616C6C626F6172642055706C6F6109
:10C5100064204672657175656E63793A20256420E2
:10C52000730A000048656172742055706C6F616415
:10C53000204672657175656E63793A2025642073B3
:10C540000A0000004D61696E626F6172642055706F
:10C550006C6F6164204672657175656E63793A200F
:10C56000256420730A0000002DE9F0410446B0F86C
:10C5700001000D4647BAB4F80B002C4940BA04F14B
:10C580000D064880601910F8028CE81E81B2601C0C
:10C59000F4F7F8FF01464046414505D0BDE8F041BB
:10C5A000024623A0FCF746BC6FF4004038184FF059
:10C5B00001081DD0FE2807D0FF2825D0B0F5817FC7
:10C5C0002CD0394627A00FE0A5F10D0104290ADB84
:10C5D0003068F17800BA20F0FF000843FBF790FBC9
:10C5E000404627490DE027A0BDE8F041FCF722BCFA
:10C5F000122D04D9607C10B92BA0FCF71BFC2F492D
:10C6000040460870BDE8F0810E2DFBD9607B002804
:10C61000F8D1BDE8F0412AA0FCF70CBC2946304611
:10C62000FFF752FEBDE8F041FAF77CBC0C060010A3
:10C63000436865636B73756D204D69736D617463D9
:10C6400068212045787065637465643A202530322E
:10C65000582C2052656365697665643A202530322E
:10C66000580A0000556E6B6E6F776E204D657373C0
:10C670006167652049443A203078253034580A00F3
:10C6800036060010496E76616C6964203078383067
:10C690004646207061796C6F6164206C656E6774CA
:10C6A000683A2025640D0A0048656172745F636111
:10C6B0006C6C6261636B5F4F4B0A000035060010C3
:10C6C000436C6F75645F52656769737465725F630D
:10C6D000616C6C6261636B5F4F4B0A0030B595B063
:10C6E00028A1F3F799FE00282DD02221F3F7B2FEFE
:10C6F00004002AD02221601CF3F7ACFE002824D0CD
:10C70000051B6D1E2A46611C2048F3F797FE1F4843
:10C7100000241FA14455F3F7D3FE00B104702C216F
:10C7200004A8F3F76EFE0FAB10AA11A912A88DE8AA
:10C730000F0013AB14AA17A11448F3F7D1FE062873
:10C7400005D019A019E01EA017E022A015E014984A
:10C75000643009901398401E089012980790119821
:10C760000690109805900F98049002200C9004A851
:10C77000F3F7CCFD022803D119A0FCF75BFB0220E4
:10C7800015B030BD2B43434C4B3A0000340B002016
:10C790002B2D000025642F25642F25642C25643A59
:10C7A00025643A256400000050617273696E675F0A
:10C7B000756E69785F6661696C65640A00000000E7
:10C7C0004E6F7420666F756E64202B43434C4B2074
:10C7D0000A0000004E6F7420666F756E64200A00B8
:10C7E000436F6E76657273696F6E206661696C6502
:10C7F000640A00001CB504460D2215A1F3F751FE92
:10C8000058B901AB6A4616A104F10D00F3F768FEB2
:10C81000022809D014A0FCF70DFB0B2215A120461D
:10C82000F3F73FFE28B106E0DDE9000100F07EF8F5
:10C83000F3E7F9F7F7F90D2211A12046F3F731FEDE
:10C84000002803D1BDE81C40FFF730BA1CBD000032
:10C8500041542B52454144464C4153483D00000051
:10C8600025642C25640000004154204572726F72CB
:10C870000D0A000041542B56455253494F4E3F007C
:10C8800041542B4552415345464C4153480000000A
:10C8900000B593B0142102A8F3F7B3FD00200246BF
:10C8A000079002A91448F7F72BFF002207A91248A6
:10C8B000F7F704FF9DF80A109DF80900CDE9000183
:10C8C0009DF808300DA2142108A8FCF7C3FA9DF8C2
:10C8D0001E109DF81D00CDE900019DF81F300BA230
:10C8E00014210DA8FCF7B6FA08AA0DA90CA0FCF7B4
:10C8F000A1FA13B000BD0000A4310010253032644D
:10C900003A253032643A2530326400003230253026
:10C9100032642F253032642F25303264000000004D
:10C920005254432025732D25730A00002DE9F0474A
:10C930000E46804604464FF48079134F1AE02502D4
:10C940004A461149284601F0B1F92A4621460FA06E
:10C95000FCF770FA002514A0795DFCF76BFA280744
:10C96000B0F1704F02D112A0FCF764FA6D1CFF2DDC
:10C97000F1D9641CB442E2D932464146BDE8F047E1
:10C980000CA0FCF757BA0000C03D00200D0A5B5018
:10C9900061676520256C75202D2030782530386C36
:10C9A000585D3A0D0A000000253032582000000082
:10C9B0000D0A00000D0A5B5052494E545D20506133
:10C9C00067657320256C7520746F20256C75207049
:10C9D00072696E7465640D0A0000000070B5B0F8ED
:10C9E00007004FF4006142BA104C114D4E00022A6C
:10C9F00010D0012A19D12046F6F7F8FE01220821AD
:10CA00002846F6F7F3FE002231462046BDE8704086
:10CA1000F6F7ECBE01222046F6F7E8FE00220821D8
:10CA20002846F6F7E3FE0122EEE770BD0008004855
:10CA3000000400487FB501781A4C0322184B0F29D7
:10CA4000254615D2A3F19C0604F2A71405F5B77587
:10CA5000CDE90026CDE902541A79491E00EE102ACC
:10CA6000104B0246183BB8EE400AC9B2032014E04E
:10CA70000B4E04F5D5749B3E05F5BD75CDE900263A
:10CA8000CDE902545A79074B00EE102A10390246BC
:10CA9000B8EE400AC9B20C3B022000F069F87FBD35
:10CAA000B80600109C0700102DE9F041B0F807000F
:10CAB000002640BA2A4C012826D00125022826D07B
:10CAC000032828D0274F042829D0052834D0062849
:10CAD00018D0072816D1FFF7E9F8F9F7F9FFE56450
:10CAE000FAF796F80420E0706571A06F20B101F0AC
:10CAF000D9FB0A2001F0B0FB1B4A00211B48FFF7BD
:10CB00009FFBA067BDE8F081A670062001E0A5703C
:10CB10000720E070F6E70220A0700820F9E7012264
:10CB200080213846F6F762FE012210213846F6F7DA
:10CB30005DFE25710320ECE7002280213846F6F7E0
:10CB400055FE002210213846F6F750FE0520E07011
:10CB50002671FFF7ABF8E664BDE8F041FAF758B884
:10CB6000140600100008004810F20008D99D0008C3
:10CB70002DE9F05F2DED028B9A46DDE90C76DDE9BB
:10CB80000EB9F0EE408A13460C460546B94266D20D
:10CB9000D81CFFF74FFA0AEB8400B0EE408A80ED14
:10CBA000008A4FF0010809F804800BEB8400D3F8E9
:10CBB00003100160F6F720FE0146002204EB44005A
:10CBC000032D02D0022D02D00AE0294B01E0284BB0
:10CBD000243B43F8201003EB800080F8048042716E
:10CBE0000021DFED240A084611E000BF19F80030EB
:10CBF00063B10AEB800393ED000AB4EEE00AF1EEB4
:10CC000010FA01DDF0EE400A491CC9B2401CB842DE
:10CC1000ECDB49B1F4EEE80AF1EE10FA01DD022096
:10CC200000E00020307006E03270032D1BD012A10E
:10CC300012A0FCF7FFF83078022810D119480188BB
:10CC400000290CD1032D10D04FF20601BCEEC80A0A
:10CC50000180641C10EE101A4480C9B28180BDECC2
:10CC6000028B00F023B810A1E2E74FF20801EDE7D4
:10CC7000EC04001000000000483200005761726EA2
:10CC8000696E673A20416C6C2025732073656E7362
:10CC90006F727320617265206F66666C696E6521C4
:10CCA0000A000000B2060010434F000030BCBDE88F
:10CCB000C09F0000F0B587B041798DF80010D0F822
:10CCC0000720CDF80120D0F80B000125274ECDF824
:10CCD00005006C46082921D1002213461046211870
:10CCE0001B02C97843EA1263401C41EA022206286B
:10CCF000F5DB1FA103A8FCF7C1F81F4B002003A917
:10CD000001EB400211F81070527802EB0712A2F505
:10CD10004C721A54401C0728F2DBF5739DF8000092
:10CD2000092821D100221346104621181B02097937
:10CD300043EA1263401C41EA02220528F5DB0CA1FC
:10CD400003A8FCF79BF80D4B002003A901EB400260
:10CD500011F81040527802EB0412A2F54C721A54EA
:10CD6000401C0628F2DBF57307B0F0BD1406001076
:10CD7000256C6C7500000000CE060020C80600205F
:10CD800070B58188B0F807004BBA41BA45F2055535
:10CD9000581B1F4A4FF48814AB4223D008DCA3F57C
:10CDA000AA4005280CD2DFE800F00E1114171A0073
:10CDB00001281AD002281BD00B2824D02B2822D0DF
:10CDC000194614A020E0517019A013E091701FA023
:10CDD00010E0117224A00DE091712BA00AE0917275
:10CDE00032A007E0D17037A004E011713BA001E050
:10CDF00051713FA0FCF71EF82046BDE870400822A4
:10CE00000349F4F71BBB3AA0BDE87040FCF712B829
:10CE1000B8060010556E6B6E6F776E206164647299
:10CE20006573733A203078253034580A00000000CA
:10CE300074656D705F66697273745F746872657330
:10CE4000686F6C64202564200A00000074656D70B2
:10CE50005F7365636F6E645F7468726573686F6C2F
:10CE600064202564200A00006D61696E626F617242
:10CE7000645F75706C6F61645F6672657175656E15
:10CE80006379202564200A00736D616C6C626F61A8
:10CE900072645F75706C6F61645F667265717565F1
:10CEA0006E6379202564200A000000006F626A65C5
:10CEB00063745F656D69737369766974792025643D
:10CEC000200A000070726573737572655F74687212
:10CED0006573686F6C64202564200A00636F5F745B
:10CEE00068726573686F6C64202564200A00000016
:10CEF00068325F7468726573686F6C6420256420A3
:10CF00000A0000002DE9F04105468088EE1D47BA71
:10CF10000020315CFF2916D0401C2828F9DBA878B6
:10CF2000801FC4B2282C00D92824214618A0FBF762
:10CF300081FF00BFA7F5AC4010380CD0202816D0D8
:10CF4000394617A020E0C4B221461CA0FBF772FFAF
:10CF5000002CE4D0EEE714211C48F3F752FA2246E5
:10CF600031461A48F3F726FA184919A00CE0174879
:10CF7000142114300546F3F744FA22463146284678
:10CF8000F3F718FA294616A0BDE8F041FBF752BFA7
:10CF900075617274325F6C656E323A2025640A00E6
:10CFA000556E6B6E6F776E20616464726573733A51
:10CFB000203078253034580A000000007561727402
:10CFC000325F6C656E313A2025640A00C406001099
:10CFD00075617274325F535349443A2025730A00D5
:10CFE00075617274325F50617373776F72643A2047
:10CFF00025730A002DE9F041134C0F460546E668FB
:10D000002068001D00F0C8FF681C07D137B12168F7
:10D01000BDE8F0410D48091D01F00EB82068354407
:10D02000B5424560216805D2A06BBDE8F041091DFD
:10D0300000F0EABF606B091D00F0E6FFA06A8542C0
:10D0400000D2A562BDE8F08100070010C4360010D0
:10D050002DE9F041054600F0FBFF2D4CA068401C77
:10D06000A06020682B4F10B1606930B32BE02560C1
:10D07000A068012827D1002606EB860007EB800078
:10D0800000F0B4FF761C382EF6D3234800F0AEFF34
:10D090002148143000F0AAFF1F48283000F0A6FFF6
:10D0A0001D483C3000F0A2FF1B48503000F09EFFAE
:10D0B000194860631430A06305E02068E96AC06A1B
:10D0C000884200D82560606A401C60626864E86A33
:10D0D0002169884200D9206100EB800007EB8000C5
:10D0E000291D00F0A9FF00F0D3FF606900280CD0D3
:10D0F0002068E96AC06A884207D208494FF0805028
:10D100000860BFF34F8FBFF36F8FBDE8F081000061
:10D1100000070010143200107436001004ED00E017
:10D1200038B500F095FF104C2068C8B90F4800F0E2
:10D130005DFF0E48143000F059FF0C48E0601430D9
:10D1400020610A4B0020F43B009003F154021021AF
:10D150000A2001F019FB206010B105A101F01AF8B6
:10D16000BDE8384000F094BF10070020F44F0020C5
:10D17000546D72510000000030B4026C0B46002A5E
:10D180000BD0C1681144C1608468A14201D3016819
:10D19000C16030BC1846F3F70DB930BC70472DE9BB
:10D1A000F041856B174604460026026C82B1C7B178
:10D1B000E068F3F7FFF8E168206C091AE160226883
:10D1C000914202D2A168081AE060022F16D017E03F
:10D1D0002068A8B9A06801F077FE06460020A0608C
:10D1E0000EE06068F3F7E6F8216C60680844606060
:10D1F000A168884204D32068606001E005B16D1E1B
:10D200006D1CA5633046BDE8F08110B5044690F86A
:10D21000590058B101280CD002280FD0502080F3BB
:10D220001188BFF34F8FBFF36F8FFEE7206B00F0C5
:10D2300043FF2046BDE8104000F03EBF10BD000097
:10D2400010484FF4C041420706D0C01D0D4920F0E0
:10D250000700411AC1F5C0410B4A00230144C2E94D
:10D2600000030839183A21F0070111604B600B6088
:10D270000B1AC0E9001393604FF0004053605061F7
:10D2800070470000D45A002058070010144E154C67
:10D29000A6F29C474FF08058DFF84C9012E000BF98
:10D2A00000F0D6FEF068C568281D00F075FEA06885
:10D2B000401EA0606068401E606000F0E9FE2846E5
:10D2C000FFF7A3FF60680028EAD138680128F9D980
:10D2D000C9F80080BFF34F8FBFF36F8FF2E70000F4
:10D2E000B03600100007001004ED00E0002807D061
:10D2F0000021816001600B460A46C16001F0BCBAA2
:10D300007047000070B51D46049C61B1C4F8002050
:10D31000C4E90F010121204601F06AFA84F8505057
:10D320000020A06470BD2460F2E700002DE9F05FEA
:10D330008846DDE90B941546834691009A460A9E7D
:10D34000A522206BF3F756F86FF00301206B01EB79
:10D350008501084420F00707780707D0502080F3A4
:10D360001188BFF34F8FBFF36F8FFEE70025B8F131
:10D37000000F0FD05FF00000221818F8001082F89C
:10D38000341018F8001011B1401C1028F4D384F8A0
:10D39000435001E084F83450382E00D33726E6623B
:10D3A000C4E91365201D00F02CFE04F1180000F004
:10D3B00028FE2461C6F138006462A061656584F8C6
:10D3C000585052465946384600F09AFA2060B9F152
:10D3D000000F01D0C9F8004000F000B830BCBDE833
:10D3E000C09F000030B5114900E011460A68824232
:10D3F000FBD34B685C18844203D1406818444860F2
:10D40000084643681C18944209D1084C183C24680B
:10D41000A24209D052681A4442600A681268026047
:10D42000814200D0086030BD0460F9E75807001061
:10D4300070B5002441600B4D0061914206D8D11AAD
:10D440008269914206D2011D286907E09A4203D2FF
:10D45000994201D3012403E0011DE86800F0D4FDE6
:10D46000204670BD1007002010B5044600F0F0FD06
:10D47000A06B28B15FF0000400F00AFE204610BD4A
:10D480000124F9E7F1B500260098846C5CB1A16B2A
:10D49000E06B81420FD3502080F31188BFF34F8F90
:10D4A000BFF36F8FFEE7502080F31188BFF34F8FDB
:10D4B000BFF36F8FFEE7A16B81420CD294F9455008
:10D4C000002269462046FFF76AFE0646681C04D023
:10D4D0006D1C84F845503046F8BD606A0028FAD0CB
:10D4E00004F1240001F030FD0028F4D00126F2E719
:10D4F00030B589B03C4D6EE00498002806DADDE9CD
:10D500000601059A90470498002864DB069C606930
:10D5100010B1201D00F040FD03A800F0D7F802462E
:10D5200004980A2857D2DFE800F00505052D334A94
:10D5300005052D3394F8280040F0010084F82800F8
:10D540000599A069059B01442046FFF771FF68B368
:10D55000216A2046884794F8280040073BD50020E0
:10D5600000900598A169002342181946204601F051
:10D57000B5FDD8B9502080F31188BFF34F8FBFF3AA
:10D580006F8FFEE714F8280F20F00100207022E0D2
:10D5900094F8280040F0010084F828000598A06164
:10D5A00028B1811813462046FFF742FF13E05020B0
:10D5B00080F31188BFF34F8FBFF36F8FFEE794F8AE
:10D5C0002800810703D4204600F076FD03E020F018
:10D5D000010084F82800002204A9286801F074FAE8
:10D5E000002889D109B030BD100700202DE9FC4189
:10D5F0000F46054600F024FF01A800F067F8044636
:10D60000019818B101F0D8FCBDE8FC81254EAFB1FE
:10D6100030690068D0B30027291B3A46306800F013
:10D62000F9FD01F0C9FC0028EED11F494FF08050F0
:10D630000860BFF34F8FBFF36F8FE5E7A542EBD8CC
:10D6400001F0BAFCF0682746C068C468201D00F0ED
:10D65000A3FC94F82800410719D5A0692B4641196D
:10D660003A462046FFF7E4FEA8B1002003460146F3
:10D6700000902A46204601F031FD60B9502080F329
:10D680001188BFF34F8FBFF36F8FFEE707E020F0E5
:10D69000010084F82800216A20468847B4E7012762
:10D6A000BAE700001007002004ED00E00648416BD7
:10D6B000096829B1416BC968C968496881627047C6
:10D6C0004FF0FF31FAE700000007001070B5054683
:10D6D00001F088FB064E0446B068844203D200F095
:10D6E00009F8012000E0002028602046B46070BDE9
:10D6F00010070020F8B5194D20E0C068C46806681E
:10D70000201D00F049FC216A2046884794F8280033
:10D71000400713D5A0693044B04206D92461606047
:10D72000211DE86800F070FC08E000200346014677
:10D7300000903246204601F0D1FC38B1E86801681B
:10D740000029DAD12969C5E90310F8BD502080F31A
:10D750001188BFF34F8FBFF36F8FFEE710070020D4
:10D7600008484068401C4FF0500080F3118804D0F6
:10D77000BFF34F8FBFF36F8FFEE7BFF34F8FBFF342
:10D780006F8FFEE724070020074CE068016841B175
:10D79000C0680021D0F80000FFF728FFFFF7A8FEBF
:10D7A000F3E701210020F7E7100700202DE9F04101
:10D7B000044600F04DFC94F9455004F124060FE0B6
:10D7C000A06C18B12046FFF75DFE04E0606A48B126
:10D7D000304601F0B9FB08B100F0B4FD6D1E6DB22A
:10D7E000002DEDDC4FF0FF3684F8456000F050FC72
:10D7F00000F02EFC94F9445004F1100709E0206970
:10D8000048B1384601F0A0FB08B100F09BFD6D1E49
:10D810006DB2002DF3DC84F84460BDE8F04100F007
:10D8200037BC00002DE9F0410546002700F008FE56
:10D83000324E306808B9FFF703FD706905424ED1DA
:10D84000C5B3083568070ED005F00700C0F1080021
:10D850000544680707D0502080F31188BFF34F8F2D
:10D86000BFF36F8FFEE72DB37068854237D823482A
:10D87000183001460C6801E020460C466168A94258
:10D8800002D221680029F7D131688C4227D007687D
:10D890002168016060680837411B10290FD96019A1
:10D8A000420708D0502080F31188BFF34F8FBFF399
:10D8B0006F8FFEE713E041606560FFF793FD6168DD
:10D8C0007068401A7060B268904200D2B0607069AF
:10D8D00001430020C4E90001F068401CF06001F041
:10D8E0006BFB780707D0502080F31188BFF34F8F70
:10D8F000BFF36F8FFEE73846BDE8F08140070010A8
:10D9000010B5031F4FF080741C601B1F21F0010134
:10D910001960191F044B0B6014390A60091F6FF05E
:10D92000020244380A6010BD61D7000810B5134CDC
:10D93000207F062812D2DFE800F00305090B0D0F47
:10D94000112000E0102000F053F909E01220FAE75E
:10D950000220F8E70120F6E70320F4E70020207713
:10D96000207F0621401CB0FBF1F201FB1200207762
:10D97000BDE810404FF4F57000F06EBC14060010C6
:10D980000B4A10B511680B6823F010030B600949AE
:10D990004B680B6011680A6842F010020A60014689
:10D9A0000348FAF761FEBDE810406420FEF759BB5A
:10D9B0007C3B0020B03D00202DE9FF4F8B4681B01D
:10D9C000994692464FF480712948F2F71AFD0024D7
:10D9D00049E000BF27490AEB8A0045000868026851
:10D9E00022F0100202602448426802600868016860
:10D9F00041F0100101601F480199FAF735FE6420DB
:10DA0000FEF72FFB4FF00008194E24E000270CE032
:10DA100001271748F2F728FD80B2FF2805D29DF8AC
:10DA200000103154304480F8018069461248FCF7F8
:10DA30009BF90028ECD05FB1BBF1000008D0014693
:10DA40000B48F2F7E9FC18B1012005B000F01EB850
:10DA50000A20FEF706FB6D1ED8D2054907A0FBF78A
:10DA6000E9F9641CE4B24C45B4D30020EDE70000B2
:10DA7000340700207C3B0020B03D002054696D65D8
:10DA80006F75745F213A2025730A000030BCBDE831
:10DA9000C08F00002DE9FF4F81B08A464FF480719E
:10DAA0003C48DDF838B0F2F7ACFC00266DE0049895
:10DAB000394900EB800047000868026822F0100234
:10DAC00002603648426802600868016841F010014F
:10DAD000016031480199FAF7C7FD6420FEF7C1FAE9
:10DAE0004FF0000837E00025DFF8A8902C460CE046
:10DAF00001252848F2F7B8FC80B2FF2805D29DF82E
:10DB0000002009F800204844447069462348FCF787
:10DB10002BF90028ECD0DDB11E4DA14620A12846EE
:10DB2000F2F77AFC04000AD084F80090BAF1000001
:10DB30001AD001462846F2F76FFCE0B914E02846F7
:10DB4000F2F792FC82B229461248521CF2F732FCDC
:10DB50000A20FEF786FA7F1EC5D2B8F1000F0ED05C
:10DB6000012005B000F026B8039830B101462846E0
:10DB7000F2F752FC08B14FF00108A51CCEE70549A9
:10DB800008A0FBF757F9761CF6B25E458FD300204C
:10DB9000E7E70000340800207C3B0020B03D002077
:10DBA0000D0A000054696D656F75745F213A202578
:10DBB000730A000030BCBDE8C08F000000B5A1B002
:10DBC0000B46024604A16846FBF758F96846FFF782
:10DBD000D7FE21B000BD000041542B43574A4150AD
:10DBE0003D25732C342C322C25730D0A00000000C7
:10DBF0001CB506218DF8000003208DF801000020DF
:10DC00008DF802008DF803008DF8040002208DF8D5
:10DC100005006846FBF7F4FD8DF80600000A8DF854
:10DC200007004FF47A73082269460548F7F772FD3A
:10DC30004FF4807203490248F7F70AFD1CBD00004B
:10DC4000F83A00201E0000102DE9F04115460E465E
:10DC5000044600F0E3F8DFF850804FF480570022CC
:10DC600039464046F5F7C2FD022000F089F8C4F3BA
:10DC7000074000F085F8C4F3072000F081F8E0B217
:10DC800000F07EF8002404E0305D00F079F8641CB8
:10DC9000A4B2AC42F8D3012239464046F5F7A6FDBE
:10DCA000BDE8F04100F07EB8000400482DE9F041E5
:10DCB000DFF8508014460D4606464FF48057002288
:10DCC00039464046F5F792FD032000F059F8C6F3B7
:10DCD000074000F055F8C6F3072000F051F8F0B205
:10DCE00000F04EF804E000BF00F00EF805F8010B5C
:10DCF000641EA4B2F8D239464046BDE8F041012284
:10DD0000F5F774BD000400480EB56FF07F40009039
:10DD1000012301AA02A90548F6F70AFF10B1FF2066
:10DD20008DF804009DF804000EBD0000103A00209C
:10DD300070B5044600F072F800F034F80F4E4FF45E
:10DD40008055002229463046F5F750FD202000F08E
:10DD500017F8C4F3074000F013F8C4F3072000F0ED
:10DD60000FF8E0B200F00CF8012229463046F5F732
:10DD70003DFDBDE8704000F015B80000000400480B
:10DD800001B582B06FF07F400090012301AA02A983
:10DD90000348F6F7CDFE002800D001200EBD00009C
:10DDA000103A002070B50B4D4FF4805400222146EC
:10DDB0002846F5F71BFD0520FFF7E2FFFFF7A4FF5C
:10DDC000C007FBD121462846BDE870400122F5F787
:10DDD0000DBD0000000400482DE9F0410646C0B228
:10DDE000C0F580740F461546A24200D814464FF481
:10DDF000807800BF00F012F8A2B239463046FFF733
:10DE000023FFA54207D0274426442D1B4446A542A4
:10DE1000F0D82C46EEE7BDE8F081000070B5094D62
:10DE20004FF48054002221462846F5F7DFFC0620F7
:10DE3000FFF7A6FF21462846BDE870400122F5F70E
:10DE4000D5BC000000040048F8F708FB2DE9F041BC
:10DE50002E48B0B00068C169C943C90652D4102128
:10DE600001622B48006840682A4EC0F5007085B2F8
:10DE700071888D4201D3681A02E0C1F50070284410
:10DE80000404240C37D0DFF89080FF2C24D8ADF8A0
:10DE9000504000206B46424606E00F18C7F30807C3
:10DEA000D75D1F54401C80B2A042F6D300201B4F08
:10DEB0000346199019AA6946386800F099FD0128AF
:10DEC0000AD019AA1AA9386800F09AFE002319AAE4
:10DED0006946386800F08CFD00270AE070883844F5
:10DEE000C0F308010E4818F80110FBF756FF7F1C1D
:10DEF000BFB2A742F2D375804FF4007206490348BF
:10DF0000F7F7A6FB30B0BDE8F08100007C3B0020B5
:10DF1000203D0020EC0600101E010010A00600109D
:10DF2000B03D002070B51E211648F2F76AFA154878
:10DF30004FF4807421461E30F2F763FA65002946DB
:10DF40001148F2F75EFA104A29461048FBF700FF25
:10DF50000F480068016841F0100101600D48006839
:10DF6000016841F0100101601E2206490848F7F7D8
:10DF70006FFB2246BDE87040024906481E31F7F7A4
:10DF800067BB0000000000101E010010B03D002023
:10DF9000743A0020F83A0020D0E9013201699A6011
:10DFA000D0E901235A604A68824201D182684A60FE
:10DFB000002202610868401E08600868704700007F
:10DFC000034B036003F15C00086080201060704721
:10DFD0001C500020044B036003F15C0008604FF408
:10DFE00000701060704700007852002000F10801B6
:10DFF0004FF0FF32C0E90112C160016100210160F0
:10E00000704700210161704730B50B685A1C02D07F
:10E0100000F1080202E0026904E022465468256823
:10E020009D42FAD953684B6099608A6051600861DB
:10E030000168491C016030BD42684A6093688B608A
:10E0400093685960916008610168491C01607047DC
:10E05000502080F31188BFF34F8FBFF36F8F0A49B1
:10E060004868401C486001280CD10848006810F03E
:10E07000FF0F07D0502080F31188BFF34F8FBFF3FD
:10E080006F8FFEE7704700002407002004ED00E0DA
:10E090000849486828B1401E486001D180F31188C2
:10E0A0007047502080F31188BFF34F8FBFF36F8FFD
:10E0B000FEE700002407002070B500282AD0164D86
:10E0C000A0F1080460686969084207D1502080F314
:10E0D0001188BFF34F8FBFF36F8FFEE722683AB10D
:10E0E000502080F31188BFF34F8FBFF36F8FFEE78F
:10E0F0008843606000F0A4F960686968084468605B
:10E100002046FFF76FF92869401C2861BDE8704080
:10E1100000F052BF70BD0000400700104FF0E0203B
:10E1200000210161816105494FF47A720968B1FBF0
:10E13000F2F1491E41610721016170470C0700207F
:10E1400010B5F2F789F8114910280ED300F1E0203C
:10E1500090F8F0030A78904207D2502080F311889B
:10E16000BFF34F8FBFF36F8FFEE7094800688968E0
:10E1700000F4E060884207D9502080F31188BFF393
:10E180004F8FBFF36F8FFEE710BD00002407002004
:10E190000CED00E010B5084B002200BF53F83240F0
:10E1A0001CB1521C082AF9D310BD43F8321003EBFE
:10E1B000C201486010BD0000C04E002010B5040030
:10E1C0000AD000F013F894F8460000280CD120463D
:10E1D000BDE81040FFF770BF502080F31188BFF3F7
:10E1E0004F8FBFF36F8FFEE710BD0000084A00217C
:10E1F00002EBC1035B68834206D1002042F8310084
:10E2000002EBC10148607047491C0829F0D37047F0
:10E21000C04E002070B515460E460446FFF718FFA5
:10E2200094F944100020491C01D184F8440094F969
:10E230004510491C01D184F84500FFF729FFA06B68
:10E2400028B92A46314604F1240000F099F8204606
:10E25000BDE87040FFF7AABA10B5020014D00F480D
:10E26000006B38B1502080F31188BFF34F8FBFF39C
:10E270006F8FFEE700F0E4F800211046FEF7BAFECB
:10E2800000F09AFE002807D105494FF08050086041
:10E29000BFF34F8FBFF36F8F10BD0000000700105A
:10E2A00004ED00E070B50546FFF7D2FE1E4C05B93F
:10E2B0002568281DFFF770FEA86A18B105F118003F
:10E2C000FFF76AFE606A401C60622068854207D1E1
:10E2D000291D1648FFF7B0FE6068401C606007E02B
:10E2E000A068401EA0602846FEF78FFFFFF7DEF90A
:10E2F000FFF7CEFE6069002814D02068854211D156
:10E30000206B38B1502080F31188BFF34F8FBFF3DB
:10E310006F8FFEE706494FF080500860BFF34F8FC4
:10E32000BFF36F8F70BD000000070010B036001003
:10E3300004ED00E002490A6A0260C9684160704762
:10E340000007001001490120C86170470007001054
:10E3500010B50C4650B1094909681831FFF754FE51
:10E360002046BDE810400121FEF744BE502080F356
:10E370001188BFF34F8FBFF36F8FFEE700070010C8
:10E3800070B514460D4668B10A4909681831FFF79F
:10E3900053FE0CB14FF0FF3521462846BDE87040D2
:10E3A000FEF728BE502080F31188BFF34F8FBFF3D4
:10E3B0006F8FFEE70007001030B587B0002403948C
:10E3C00005AA04A903A80494FFF7FAFDDDE90301F7
:10E3D0000094CDE90110002315A11748059A00F01B
:10E3E000C7FC164D0028E8621FD000F047FE012848
:10E3F00009D0401C19D1502080F31188BFF34F8FF2
:10E40000BFF36F8FFEE7502080F31188BFF34F8F6B
:10E41000BFF36F8F4FF0FF30A86201206861EC609E
:10E4200007B0BDE8304000F0A9B807B030BD00002B
:10E4300049444C45000000008DD200080007001040
:10E440000248016B491C016370470000000700107F
:10E45000164810B5016B11B10121C16110BD002139
:10E46000C1610169124A01E0B9B1491E01EB8103A2
:10E4700052F82330002BF7D001EB810302EB83022B
:10E4800002F1080453685B685360A34201D15B68E2
:10E490005360DA680260016110BD502080F311887A
:10E4A000BFF34F8FBFF36F8FFEE700000007001030
:10E4B000143200102DE9FF4F95B0924688468146F0
:10E4C000229E00F08FFC07464FF47A7000254643E9
:10E4D000834634E020484FF496726946006800F0A5
:10E4E000F3FA01282BD11898BDF85010401B421E9A
:10E4F000914201DA084600E0401E84B20AEB0500B2
:10E5000022466946F1F756FF281985B200210AF81C
:10E510000510514611A0FAF78DFC5046FDF766FB39
:10E5200000240AE059F824105046F1F775FF18B19D
:10E53000204619B000F01EB8641C4445F2DB00F020
:10E5400051FCB6FBFBF1C01B8842C3D306A0FAF70F
:10E5500071FC4FF0FF30ECE7A006001052656376C7
:10E560003A2025730D0A000054696D656F75740DAE
:10E570000A00000030BCBDE8C08F00001CB5374861
:10E580000168374A914207D1502080F31188BFF3C8
:10E590004F8FBFF36F8FFEE700683149491E8842F5
:10E5A00007D1502080F31188BFF34F8FBFF36F8FD7
:10E5B000FEE72C4908780190FF20087008788DF854
:10E5C00000009DF800009DF8002000F0F00090424F
:10E5D00007D0502080F31188BFF34F8FBFF36F8FA8
:10E5E000FEE79DF80000204C00F05000207007204E
:10E5F000A06005E09DF8002052008DF80020401E2C
:10E600009DF800201206F5D4A060032807D0502002
:10E6100080F31188BFF34F8FBFF36F8FFEE74FF486
:10E620004070A060019808700C482030016841F4E7
:10E6300070010160016841F070410160FFF76EFDFB
:10E6400000206060F1F7D0FD0848016841F04041CA
:10E650000160F1F7B5FD00201CBD000000ED00E0F9
:10E6600071C20F4100E400E02407002034EF00E015
:10E6700010B5502080F31188BFF34F8FBFF36F8F19
:10E6800000F0BEFB18B104494FF080500860002034
:10E6900080F3118810BD000004ED00E010B50C46B9
:10E6A00048B184420FD9502080F31188BFF34F8FB7
:10E6B000BFF36F8FFEE7502080F31188BFF34F8FB9
:10E6C000BFF36F8FFEE70222002100F03CF8002824
:10E6D00000D0846310BD38B50C4648B184420FD9D0
:10E6E000502080F31188BFF34F8FBFF36F8FFEE789
:10E6F000502080F31188BFF34F8FBFF36F8FFEE779
:10E700000221134600220091114600F03DF8002836
:10E7100000D0846338BD10B502460021012000F00E
:10E7200012F80446FEF7E2FD204610BD38B50B4650
:10E73000002200901146012000F026F80446FEF762
:10E74000D5FD204638BDF8B517460E46050013D056
:10E7500005FB06F05430FFF765F804000AD00020EE
:10E7600084F8460004F154023B46314628460094A2
:10E77000FEF7C8FD2046F8BD502080F31188BFF396
:10E780004F8FBFF36F8FFEE738B5049D18B153B1BB
:10E79000CAB181B120E0502080F31188BFF34F8FC0
:10E7A000BFF36F8FFEE7502080F31188BFF34F8FC8
:10E7B000BFF36F8FFEE7502080F31188BFF34F8FB8
:10E7C000BFF36F8FFEE739B1502080F31188BFF39C
:10E7D0004F8FBFF36F8FFEE754241C46012384F84C
:10E7E00046302B460094FEF78DFD204638BD0000D4
:10E7F00070B50D46040025D0FFF72AFCD4E90F20A0
:10E80000216802FB0011A1600021A1632168616001
:10E810000A46D4E90F01401E00FB0121E1602146B8
:10E820004FF0FF3001F8440F487004F110008DB133
:10E83000FFF7DCFB04F12400FFF7D8FBFFF728FC0F
:10E84000012070BD502080F31188BFF34F8FBFF3BC
:10E850006F8FFEE721690029F0D000F075FB0028DA
:10E86000ECD004494FF080500860BFF34F8FBFF3E6
:10E870006F8FE3E704ED00E02DE9FF4782B01D460E
:10E880008A464FF00008040003D0BAF1000F08D008
:10E8900011E0502080F31188BFF34F8FBFF36F8FCB
:10E8A000FEE7206C38B1502080F31188BFF34F8F02
:10E8B000BFF36F8FFEE7022D0AD1E06B012807D06E
:10E8C000502080F31188BFF34F8FBFF36F8FFEE7A7
:10E8D00000F07AFA454F4FF000094FF0805648B9E2
:10E8E000049838B1502080F31188BFF34F8FBFF3E5
:10E8F0006F8FFEE7FFF7ACFBA06BE16B884207D39D
:10E90000022D05D0049838B3B8F1000F27D02BE0C2
:10E91000D4F838802A4651462046FEF740FCA16CC8
:10E9200041B1022D02D1B8F1000F0FD12046FEF700
:10E93000A9FD05E0616A19B104F1240000F004FBAF
:10E9400020B13E60BFF34F8FBFF36F8FFFF7A0FB87
:10E95000012006B0BDE8F087FFF79AFB22E0684689
:10E96000FFF7E8FC4FF00108FFF792FBFFF768FDA7
:10E97000FFF76EFB94F94400401C01D184F84490E9
:10E9800094F94500401C01D184F84590FFF780FBC5
:10E9900004A9684600F082F930B12046FEF706FF70
:10E9A00000F00AFB0020D4E7FFF752FBA06BE16BFD
:10E9B000884213D1FFF76CFB04F110000499FFF7B4
:10E9C000C7FC2046FEF7F2FE00F0F6FA002891D1CF
:10E9D0003E60BFF34F8FBFF36F8F8BE7FFF758FB9E
:10E9E0002046FEF7E3FE00F0E7FA83E704ED00E0DF
:10E9F0002DE9F0471F4616468A46040003D0BAF1B7
:10EA0000000F08D011E0502080F31188BFF34F8F22
:10EA1000BFF36F8FFEE7206C38B1502080F3118870
:10EA2000BFF34F8FBFF36F8FFEE7022F0AD1E06B6A
:10EA3000012807D0502080F31188BFF34F8FBFF318
:10EA40006F8FFEE7FFF77CFB5021EFF3118081F31E
:10EA50001188BFF34F8FBFF36F8F8046A06BE16BC0
:10EA6000884207D3022F05D05FF0000088F3118899
:10EA7000BDE8F08794F94550D4F838903A465146AD
:10EA80002046FEF78CFB681C04D06D1C84F84550B2
:10EA90000120EBE7A06C012540B1022F02D1B9F1B2
:10EAA000000FF5D12046FEF7EDFC06E0606A002875
:10EAB000EED004F1240000F047FA0028E8D0002E40
:10EAC000E6D03560E4E700002DE9F747002683B083
:10EAD0008A46040003D0BAF1000F08D011E050209C
:10EAE00080F31188BFF34F8FBFF36F8FFEE7206C69
:10EAF00038B1502080F31188BFF34F8FBFF36F8F71
:10EB0000FEE700F061F9DFF8F4804FF000094FF004
:10EB1000805748B9059838B1502080F31188BFF369
:10EB20004F8FBFF36F8FFEE7FFF792FAA56BC5B16A
:10EB300051462046FEF720FB6D1EA563206950B1AB
:10EB400004F1100000F000FA28B1C8F80070BFF31B
:10EB50004F8FBFF36F8FFFF79BFA012006B0BDE820
:10EB6000F087059808B11EB106E0FFF791FA27E09B
:10EB70006846FFF7DFFB0126FFF78AFAFFF760FC24
:10EB8000FFF766FA94F94400401C01D184F84490E0
:10EB900094F94500401C01D184F84590FFF778FABC
:10EBA00005A9684600F07AF8002820460AD0FEF74A
:10EBB000FDFD00F001FA2046FEF756FC0028B3D018
:10EBC0000020CBE7FEF750FC90B104F1240005993A
:10EBD000FFF7BEFB2046FEF7E9FD00F0EDF9002847
:10EBE000A2D1C8F80070BFF34F8FBFF36F8F9BE7C0
:10EBF0002046FEF7DBFD00F0DFF995E704ED00E0CD
:10EC00002DE9F04790468946040003D0B9F1000F82
:10EC100008D011E0502080F31188BFF34F8FBFF36D
:10EC20006F8FFEE7206C38B1502080F31188BFF35E
:10EC30004F8FBFF36F8FFEE7FFF782FA5020EFF39D
:10EC4000118680F31188BFF34F8FBFF36F8FA76BCF
:10EC5000F7B194F9445049462046FEF78DFA7F1EDD
:10EC6000A763681C04D06D1C84F84450012010E098
:10EC700020690028FAD004F1100000F065F900289E
:10EC8000F4D0B8F1000FF1D00121C8F80010EDE781
:10EC9000002086F31188BDE8F08700002DE9F041DF
:10ECA0000C46050011D0C4B1FFF7D2F9174BDA6852
:10ECB0006E682068911B471C17D02F681B6A9F4203
:10ECC00019D0964217D8012410E0502080F3118803
:10ECD000BFF34F8FBFF36F8FFEE7502080F3118893
:10ECE000BFF34F8FBFF36F8FFEE70024FFF7D0F91C
:10ECF0002046BDE8F081884205D9401A20602846A8
:10ED0000FFF718FBF1E700202060DCE700070010A8
:10ED10002DE9FF5F8346DDE90E87994616468A4650
:10ED20009000FEF77FFD05001CD05C20FEF77AFD09
:10ED3000040014D00020256384F85900CDE9024076
:10ED4000CDE900874B46324651465846FEF7EEFA6B
:10ED50002046FEF77DF9012004B000F006B82846F1
:10ED6000FFF7AAF94FF0FF30F6E730BCBDE8C09FCF
:10ED7000F0B585B0DDE90B640A9DA6B1DCB15C2776
:10ED800000972663022684F85960002604AFCDE977
:10ED90000246CDE90057FEF7C9FA2046FEF758F9BA
:10EDA000049805B0F0BD502080F31188BFF34F8F59
:10EDB000BFF36F8FFEE7502080F31188BFF34F8FB2
:10EDC000BFF36F8FFEE700000548416919B1006B82
:10EDD00018B10020704701207047022070470000E2
:10EDE000000700100148C0687047000000070010CD
:10EDF00010B5FFF7A5F90148C06810BD0007001065
:10EE00002DE9F0412E4C0027206B28B1A069401C51
:10EE1000A0613846BDE8F081E668761CE66013D153
:10EE2000606B006838B1502080F31188BFF34F8FBA
:10EE3000BFF36F8FFEE7606BA16B6163A063206A15
:10EE4000401C2062FEF732FCA06ADFF87880864220
:10EE500009D3606B0068A0B1606BC068C568686862
:10EE6000864211D2A0622068C06A00EB800158F887
:10EE70002100012800D90127E0690028C9D0012715
:10EE8000C7E74FF0FF30EDE7281DFFF785F8A86AC8
:10EE900018B105F11800FFF77FF8E86A2169884288
:10EEA00000D9206100EB800108EB8100291DFFF7EC
:10EEB000C3F8E86A2168C96A8842CAD30127C8E74B
:10EEC000000700101432001070B504004FF000016C
:10EED00033D01B4D2868844207D0502080F311881E
:10EEE000BFF34F8FBFF36F8FFEE7206D38B1401E29
:10EEF0002065E36CE26A9A421FD040B11DE05020C9
:10EF000080F31188BFF34F8FBFF36F8FFEE7201D93
:10EF1000FFF742F8E06CE062C0F13800A061E06AFF
:10EF20002969884200D92861064900EB800001EB7D
:10EF30008000211DFFF780F80121084670BD000008
:10EF4000000700101432001070B5C068C46854B1D6
:10EF500004F118000646FFF71FF8144D286B50B156
:10EF60003146134815E0502080F31188BFF34F8FCE
:10EF7000BFF36F8FFEE7201DFFF70EF8E06A2969E7
:10EF8000884200D928610B4900EB800001EB80002A
:10EF9000211DFFF751F8E06A2968C96A884202D941
:10EFA0000120E86170BD002070BD00000007001066
:10EFB0009C360010143200102DE9F0472C4D00242F
:10EFC0002746286B38B1FFF743F8286B401E2863AB
:10EFD000286B40B146E0502080F31188BFF34F8F7B
:10EFE000BFF36F8FFEE7A968224E0120D1B3A6F5CB
:10EFF000916980463068E0B1F068C46804F1180097
:10F00000FEF7CAFF201DFEF7C7FFE06A29698842A4
:10F0100000D9286100EB800109EB8100211DFFF779
:10F020000BF8E06A2968C96A8842E3D3C5F81C80F6
:10F03000E0E70CB1FEF73AFBAC694CB14FEA0806C9
:10F04000FFF7DEFE00B1EE61641EF9D10020A86179
:10F05000E86938B10849012738070860BFF34F8FC6
:10F06000BFF36F8FFFF714F83846BDE8F087000054
:10F07000000700109C36001004ED00E010B586B0CB
:10F08000FEF74EF8114C2068B8B1002003900490B0
:10F0900005AA04A903A8FEF79DFFDDE903210220CC
:10F0A0008DE8070000230AA10B48059AFFF760FED0
:10F0B000606010B106B0012010BD502080F31188AF
:10F0C000BFF34F8FBFF36F8FFEE7000010070020E4
:10F0D000546D72205376630089D700082DE9FF41F3
:10F0E0001E46134602000A9D4FF0000016D0144C35
:10F0F0002768002F0FD0CDE900130292062917DAF6
:10F10000FFF762FE02284FF000030FD0002269468D
:10F110002068FFF7B1FB04B0BDE8F081502080F318
:10F120001188BFF34F8FBFF36F8FFEE72A46EEE7DC
:10F130000023324669463846FFF75AFCEBE70000E9
:10F14000100700201F1C1F1E1F1E1F1F1E1F1E1F1B
:10F150001F1D1F1E1F1E1F1F1E1F1E1F24F600081F
:10F16000000000000000000000000000000000009F
:10F170000008000030000000000000000000000057
:10F1800044F600080000000000000000000000003D
:10F1900000000000000800001C000000000000004B
:10F1A00000000000CCF50008000000000000000096
:10F1B0000000000000000000001000001800000027
:10F1C00000000000000000004CF6000800000000F5
:10F1D0000000000000000000000000000008000027
:10F1E00010000000000000000000000078F6000899
:10F1F000000000000000000000000000000000000F
:10F2000000080000280000000000000000000000CE
:10F21000C4F500080000000000000000000000002D
:10F2200000000000001000001800000000000000B6
:10F23000000000005CF60008000000000000000074
:10F240000000000000000000000800002000000096
:10F250000000000000000000F0F5000800000000C1
:10F26000C426001054000000C20E00100018000058
:10F27000DCF5000800000000682F002054000000AA
:10F28000660B00200024000004F6000800000000C7
:10F29000183100105400000018270010000A000068
:10F2A00014F6000800000000583900205400000047
:10F2B000BC2F00209C0900006CF600080000000034
:10F2C000000000000000000034F60008000000000C
:10F2D000000000000000000000000000000000002E
:10F2E0000102030406070809A0860100400D03007F
:10F2F000801A060000350C0040420F0080841E007A
:10F3000000093D0000127A000024F40000366E016E
:10F310000048E801006CDC02000000000102030468
:10F320001F1C1F1E1F1E1F1F1E1F1E1F00404040B0
:10F3300040404040404041414141414040404040C8
:10F340004040404040404040404040404005020274
:10F350000202020202020202020202020220202033
:10F36000202020202020200202020202020290908F
:10F37000909090901010101010101010101010108D
:10F3800010101010101010100202020202028888E1
:10F3900088888888080808080808080808080808ED
:10F3A00008080808080808080202020240000000D5
:10F3B0002DF300081F1D1F1E1F1E1F1F1E1F1E1FB7
:10F3C00041542B4D515454434F4E4E3D302C22341A
:10F3D000372E3130302E362E323134222C3138381F
:10F3E000332C22424154547C7365637572656D6F92
:10F3F00064653D322C7369676E6D6574686F643D3A
:10F40000686D6163736861312C74696D65737461D3
:10F410006D703D313732393335313730313030333B
:10F420007C222C2242415454266B317663634C4A31
:10F4300076735579222C22453636344631313043A5
:10F440003537353242444232393443313441444312
:10F450003535393441363733433635353242382243
:10F460000D0A000041542B4D5154545355423D3028
:10F470002C222F7379732F6B317663634C4A76732A
:10F4800055792F424154542F7468696E672F736504
:10F4900072766963652F70726F70657274792F73FD
:10F4A0006574222C310D0A00574946495F53656E39
:10F4B000645F50726573737572655F434F5F483266
:10F4C0005F44617461204641494C45442061667443
:10F4D0006572203320726574726965732E20476FE0
:10F4E000746F20574946495F524553544F52450D5A
:10F4F0000A000000574946495F53656E645F5465D2
:10F500006D70657261747572655F446174612046E7
:10F5100041494C4544206166746572203320726510
:10F5200074726965732E20476F746F20574946497E
:10F530005F524553544F52450D0A00005749464902
:10F540005F53656E645F73656E736F726C696E6531
:10F55000204641494C454420616674657220332041
:10F56000726574726965732E20476F746F205749F6
:10F5700046495F524553544F52450D0A0000000062
:10F58000574946495F53656E645F73797374656D5F
:10F590006C6576656C204641494C45442061667433
:10F5A0006572203320726574726965732E20476F0F
:10F5B000746F20574946495F524553544F52450D89
:10F5C0000A000000636C6F756400000074656D7064
:10F5D0005F7072657373757265000000636C6F75A0
:10F5E000645F6D6573736167655F717565756500EF
:10F5F00063616E5F6D6573736167655F7175657576
:10F600006500000075617274327278717565756598
:10F6100000000000756172743372787175657565EC
:10F6200000000000486967686573744C6576656C16
:10F630000000000064617461526561647953656D16
:10F6400000000000436F6D6D6F6E000063686563BE
:10F650006B5F73656E736F72000000005379737493
:10F66000656D5374617475730000000064617461AA
:10F670004D75746578000000646973706C61790081
:10F68000C0F6000800000020340700001011000838
:10F69000E8F60008000000106407000010110008E0
:10F6A000E8F6000834070020A0B30000008F00082F
:10F6B00034F700086407001074330000008F00085E
:10F6C00001FF01FF01FF01FF01FF01FF01C0BA01BE
:10F6D00002D12DD5E34139013926210A171042F113
:10F6E0000319093D1AAA018101FF01FF01FF01FF72
:10F6F00001FF01FF011C5D010101020A8907590B8D
:10F7000009112E3172031AFF0181A90C01441A3F1D
:10F710005073777010093C64640A0A011E03D00A12
:10F720005F016A69614C6F6E675C4A4C3801C9A819
:04F730000174000060
:040000050800018D61
:00000001FF
